:020000040800F2
:1000000030AE0020A1020008B9CE0008B1B100084E
:10001000C5C9000815350008D1020108000000001C
:10002000000000000000000000000000E1D900080E
:10003000995700080000000021D4000811EB0008C7
:10004000BB020008BB020008BB020008BB0200089C
:10005000BB020008BB0200089D570008BB02000855
:10006000BB020008A9570008B5570008BB020008EA
:10007000A1550008B1550008BB020008BB020008EA
:10008000BB020008BB020008BB02000839350008AB
:100090001935000829350008BB020008C1570008BF
:1000A000BB020008BB020008BB020008BB0200083C
:1000B000BB020008BB020008BB020008BB0200082C
:1000C000BB020008BB020008BB020008BB0200081C
:1000D000BB020008BB020008BB020008BB0200080C
:1000E000BB020008BB020008BB020008BB020008FC
:1000F000BB020008BB020008BB020008BB020008EC
:10010000BB020008BB020008BB020008BB020008DB
:10011000BB020008BB020008BB020008BB020008CB
:10012000BB020008C1550008D1550008E155000880
:10013000BB020008BB020008BB02000869350008CA
:100140004935000859350008BB020008BB02000809
:10015000BB020008F1550008BB020008B502010807
:10016000BB020008BB020008BB020008BB0200087B
:10017000BB020008BB020008BB0200080000000030
:10018000BB020008BB02000800F002F800F05EF8B5
:100190000AA090E8000C82448344AAF10107DA45E2
:1001A00001D100F053F8AFF2090EBAE80F0013F0D6
:1001B000010F18BFFB1A43F001031847DC68010068
:1001C000FC6801000A444FF0000C10F8013B13F0EA
:1001D000070408BF10F8014B1D1108BF10F8015BA0
:1001E000641E05D010F8016B641E01F8016BF9D193
:1001F00013F0080F1EBF10F8014BAD1C0C1B09D1EA
:100200006D1E58BF01F801CBFAD505E014F8016B5B
:1002100001F8016B6D1EF9D59142D6D370470000ED
:100220000023002400250026103A28BF78C1FBD8FF
:10023000520728BF30C148BF0B6070471FB516F08A
:100240008AFA00F0DAF81FBD10B510BD00F09AF977
:100250001146FFF7F3FF10F03DFA00F0B8F903B4D0
:10026000FFF7F2FF03BC00F0BBF900000B49D1F827
:1002700000C04A685CF8043B1068184442F8040B5C
:100280008C4528BFA1F1DC0C8A4228BFA1F1DC0219
:10029000C1F800C04A6020F0004070474C040020C4
:1002A0000948804709480047FEE7FEE7FEE7FEE70A
:1002B000FEE7FEE7FEE7FEE7FEE7FEE70448054946
:1002C000054A064B70470000E5EB0008890100086D
:1002D000308E002030AE0020309E0020309E002066
:1002E00053EA020C00F069802DE9F04B4FF0000654
:1002F000002B1FBFB3FA83F503FA05F424FA05F6C1
:100300005E4012BF1643B2FA82F502FA05F4C5F157
:1003100020051EBF22FA05FC44EA0C04203556EAEB
:10032000044C4FEA144418BF641C4FF000084FF00F
:100330000009904271EB030C39D3002919BFB1FABF
:1003400081F701FA07F6B0FA80F700FA07F6C7F16D
:1003500020071EBF20FA07FC46EA0C062037B6FB32
:10036000F4FCA7EB0507103F07F01F0BCBF12006AD
:100370002CFA06F60CFA0BFB44BFB3460026202FDE
:10038000A4BF5E464FF0000B5BEA060C08BF4FF0BF
:10039000010B19EB0B0948EB0608ABFB027C06FBD3
:1003A00002CC0BFB03CCC01B71EB0C01C1E70B466D
:1003B000024641464846BDE8F08B13B5084318BFD6
:1003C0004FF0FF300146AFF30080BDE81C4070479E
:1003D0000B4910B5A1F17C020A4CC2E93712372152
:1003E00006E000EB104342F82130074B00FB0340CE
:1003F0000B1EA1F10101F4DC10BD0120E8E70000B3
:10040000EC030020E119D666CD0D0100032A40F26D
:10041000308010F0030C00F0158011F8013BBCF1A6
:10042000020F624498BF11F801CB00F8013B38BFBE
:1004300011F8013BA2F1040298BF00F801CB38BFCC
:1004400000F8013B11F0030300F02580083AC0F0EA
:10045000088051F8043B083A51F804CBA0E8081092
:10046000F5E7121D5CBF51F8043B40F8043BAFF3C5
:100470000080D20724BF11F8013B11F801CB48BF1F
:1004800011F8012B24BF00F8013B00F801CB48BF55
:1004900000F8012B704710B5203AC0F00B80B1E88E
:1004A0001850A0E81850B1E81850A0E81850203AA9
:1004B000BFF4F5AF5FEA027C24BFB1E81850A0E8B2
:1004C000185044BF18C918C0BDE810405FEA827CCC
:1004D00024BF51F8043B40F8043B08BF7047D207E3
:1004E00028BF31F8023B48BF11F8012B28BF20F884
:1004F000023B48BF00F8012B704702F0FF0343EABC
:10050000032242EA024200F002B84FF0000200B5B6
:10051000134694469646203922BFA0E80C50A0E826
:100520000C50B1F12001BFF4F7AF090728BFA0E8D4
:100530000C5048BF0CC05DF804EB890028BF40F8A0
:10054000042B08BF704748BF20F8022B11F0804FE2
:1005500018BF00F8012B704770477047704710B5FF
:1005600000F008F8006810BD10B5044600F002F86D
:10057000046010BD004870475404002000487047D4
:10058000540400207546FFF7F9FFAE4605006946A2
:10059000534620F00700854618B020B5FFF78EFEC1
:1005A000BDE820404FF000064FF000074FF0000874
:1005B0004FF0000BAC46ACE8C009ACE8C009ACE8B1
:1005C000C009ACE8C00921F007018D46704710B59D
:1005D0000446AFF300802046BDE81040FFF73FBE61
:1005E00001491820ABBEFEE726000200704700005C
:1005F00080B58AB008900791089820B9FFE7FF20DE
:100600008DF827009BE0079820B9FFE7FF208DF8C1
:10061000270094E0079890ED000A90ED013A90EDE4
:10062000021A90ED032A20EE030A21EE021A30EEA0
:10063000010A30EE000A8DED060A079890ED010AD6
:1006400090ED021A20EE000A21EE011A30EE010AA6
:1006500030EE001AB7EE000A8DED010A30EE410AC5
:100660008DED050A9DED060ADDED050A14F058FD35
:100670009DED011A089880ED010A079890ED000A97
:1006800090ED013A90ED024A90ED032A20EE040A23
:1006900022EE032A30EE420A30EE000A8DED040A03
:1006A0009DED040AB0EEC00AB4EE410AF1EE10FA74
:1006B0000ADBFFE7DDED040A9FED230A0FF052FF8E
:1006C000089880ED020A07E09DED040A14F026FA6E
:1006D000089880ED020AFFE7079890ED000A90ED78
:1006E000011A90ED022A90ED033A20EE030A21EE62
:1006F000021A30EE010A30EE000A8DED030A079867
:1007000090ED020A90ED031A20EE000A21EE011A84
:1007100030EE010A30EE001AB7EE000A30EE410A60
:100720008DED020A9DED030ADDED020A14F0F8FCDE
:10073000089880ED000A00208DF82700FFE79DF95A
:1007400027000AB080BD00BFDB0FC93F80B58CB069
:100750000A9009918DED080A0A9820B9FFE7FF2059
:100760008DF82F0029E19DED081AB7EE000A80EE02
:10077000010A0A9880ED040A0A994FF07E50086039
:100780000A99002048600A9988600A99C860099807
:10079000002800F00E81FFE7099801680091406889
:1007A00015F00EFF0246009801920A46019942ECAC
:1007B000101B8DED020B15F003FF9DED020B41ECBC
:1007C000110B14F0ADFB8DED040B9DF8170080F0BC
:1007D00080008DF817000498059915F0C5F9079069
:1007E000099890ED000AB5EE400AF1EE10FA2BD10F
:1007F000FFE7099890ED010AB5EE400AF1EE10FA14
:1008000022D1FFE7099890ED020AB5EE400AF1EE19
:1008100010FA19D1FFE70A9940F2C560C3F64D708E
:1008200008600A9944F62D20C3F60D4048600A99E5
:100830004AF25640CBF6393088600A9944F2AD70DE
:10084000C3F61970C860B3E09DED070A9FED5D1A0D
:10085000B4EE410AF1EE10FA08DBFFE79DED070A5E
:10086000B5EE400AF1EE10FA19DDFFE70A9945F6F8
:100870006E10C3F67F7008600A9945F20C30C3F61B
:10088000B01048600A9948F6AB00CBF6BB308860E0
:100890000A9949F28550C3F69750C86087E09DEDEC
:1008A000070A9FED491AB4EE410AF1EE10FA0ADB8D
:1008B000FFE79DED070A9FED431AB4EE410AF1EE02
:1008C00010FA19DDFFE70A9940F2C560C3F64D70D2
:1008D00008600A9944F62D20C3F60D4048600A9935
:1008E0004AF25640CBF6393088600A9944F2AD702E
:1008F000C3F61970C86059E09DED070A9FED331AE1
:10090000B4EE410AF1EE10FA0ADBFFE79DED070AAB
:100910009FED2D1AB4EE410AF1EE10FA19DDFFE752
:100920000A9940F2C560C3F64D7008600A9944F612
:100930002D20C3F60D4048600A994AF25640CBF686
:10094000393088600A9944F2AD70C3F61970C860F6
:100950002BE09DED070A9FED1D1AB4EE410AF1EE62
:1009600010FA08DBFFE79DED070AB5EE400AF1EE4D
:1009700010FA19DDFFE70A9940F2C560C3F64D7021
:1009800008600A9944F62D20C3F60D4048600A9984
:100990004AF25640CBF6393088600A9944F2AD707D
:1009A000C3F61970C860FFE7FFE7FFE7FFE7FFE75F
:1009B000FFE700208DF82F00FFE79DF92F000CB016
:1009C00080BD00BFDB0FC93FDB0F49400000B442D0
:1009D00081B000900099002088604860086001B0F4
:1009E0007047000080B52DED048BB2B030902F9190
:1009F0002E922D93309828B9FFE7FF208DF8C7007D
:100A000000F0F7BD2F9828B9FFE7FF208DF8C70049
:100A100000F0EFBD2E9828B9FFE7FF208DF8C70042
:100A200000F0E7BD40F27401C2F200014EF69E7084
:100A3000C3F6275008602D9848B9FFE730982F99E2
:100A40002E9A00F0DDFD8DF8C70000F0D2BD2D9884
:100A5000006809902D98406808902D98806807904C
:100A60009DED090AB5EE400AF1EE10FA19D1FFE743
:100A70009DED080AB5EE400AF1EE10FA11D1FFE73C
:100A80009DED070AB5EE400AF1EE10FA09D1FFE735
:100A900030982F992E9A00F0B3FD8DF8C70000F022
:100AA000A8BD2F98006806902F98406805902F9851
:100AB000806804902E98006803902E9840680290F9
:100AC0002E988068019030989DED033A90ED010AD0
:100AD00090ED022A90ED031A20EE430A9DED023AB2
:100AE00022EE032A30EE420A9DED012A21EE021A7F
:100AF00030EE410AB6EE001A20EE010A8DED270A0B
:100B000030989DED034A90ED000A90ED023A90ED89
:100B1000032A20EE040A9DED014A23EE043A30EE4A
:100B2000030A9DED023A22EE032A30EE420A20EE3D
:100B3000010A8DED260A30989DED024A90ED000ADB
:100B400090ED013A90ED032A20EE040A9DED014A52
:100B500023EE043A30EE430A9DED033A22EE032AD7
:100B600030EE020A20EE010A8DED250A30989DED47
:100B7000014A90ED000A90ED013A90ED022A20EE34
:100B8000040A9DED024A23EE043A30EE030A9DED7D
:100B9000033A22EE032A30EE420A20EE010A8DEDDE
:100BA000240A9DED060AB5EE400AF1EE10FA11D1C5
:100BB000FFE79DED050AB5EE400AF1EE10FA09D106
:100BC000FFE79DED040AB5EE400AF1EE10FA00F0E1
:100BD0009984FFE79DED060A20EE000A9DED051AB7
:100BE00021EE011A30EE010A9DED041A21EE011AE0
:100BF00030EE010A0AF0DEFA8DED2C0A9DED2C1A7A
:100C00009DED060A20EE010A8DED060A9DED2C1AD7
:100C10009DED050A20EE010A8DED050A9DED2C1AC9
:100C20009DED040A20EE010A8DED040A9DED090AEE
:100C300020EE000A9DED081A21EE011A30EE010A9D
:100C40009DED071A21EE011A30EE010A0AF0B2FA00
:100C50008DED2C0A9DED2C1A9DED090A20EE010A5E
:100C60008DED090A9DED2C1A9DED080A20EE010A72
:100C70008DED080A9DED2C1A9DED070A20EE010A64
:100C80008DED070A309890ED000A30EE000A9DEDD8
:100C9000091A20EE010A8DED210A309890ED000A24
:100CA00030EE000A9DED081A20EE010A8DED200AB3
:100CB000309890ED000A30EE000A9DED071A20EE04
:100CC000010A8DED1F0A309890ED010A30EE000AFE
:100CD0009DED091A20EE010A8DED1E0A309890ED67
:100CE000000A30EE000A8DED190A309890ED010AE5
:100CF00030EE000A8DED180A309890ED020A30EEC1
:100D0000000A8DED170A309890ED030A30EE000AC4
:100D10008DED160A309890ED000A90ED021A30EE33
:100D2000000A20EE010A8DED150A309890ED020AB6
:100D300090ED031A30EE000A20EE010A8DED140A40
:100D4000309890ED000A20EE000A8DED130A3098DD
:100D500090ED000A90ED011A20EE010A8DED120AC5
:100D6000309890ED000A90ED021A20EE010A8DED08
:100D7000110A309890ED000A90ED031A20EE010A56
:100D80008DED100A309890ED010A20EE000A8DEDED
:100D90000F0A309890ED010A90ED021A20EE010A38
:100DA0008DED0E0A309890ED010A90ED031A20EEB9
:100DB000010A8DED0D0A309890ED020A20EE000A2E
:100DC0008DED0C0A309890ED020A90ED031A20EE9A
:100DD000010A8DED0B0A309890ED030A20EE000A0F
:100DE0008DED0A0A9DED091A9DED130A21EE000A08
:100DF0009DED202A309890ED025A90ED033A22EEB4
:100E0000032A30EE420A9DED1F2A22EE052A30EE1B
:100E1000020A9DED0F2A21EE022A30EE020A9DED14
:100E2000182A9DED084A22EE044A24EE054A30EEC7
:100E3000040A9DED074A22EE042A22EE032A30EE30
:100E4000020A9DED0C2A21EE022A30EE420A9DEDA7
:100E50000A2A21EE021A30EE410A8DED230A9DED99
:100E6000210A309890ED015A90ED024A90ED033A34
:100E700020EE030A9DED081A9DED132A21EE022AA9
:100E800030EE020A9DED1F2A22EE052A30EE420ABC
:100E90009DED1E2A22EE042A30EE020A9DED0F2A55
:100EA00021EE022A30EE420A9DED0C2A21EE022AA2
:100EB00030EE020A9DED172A9DED074A22EE042A24
:100EC00022EE032A30EE020A9DED0A2A21EE021AD2
:100ED00030EE410A8DED220A9DED230A20EE000A34
:100EE0009DED221A21EE011A30EE010A0AF062F994
:100EF000B7EE006A86EE000A8DED1D0A9DED210A0F
:100F0000309890ED012A90ED021A90ED033A20EE10
:100F1000011A9DED200A20EE020A30EE412A9DEDD5
:100F2000071A9DED130A21EE000A30EE022A9DED0C
:100F30001E0A20EE030A30EE020A9DED0F2A21EE72
:100F4000022A30EE420A9DED172A9DED084A22EE54
:100F5000042A22EE032A30EE020A9DED0C2A21EE2D
:100F6000022A30EE420A9DED0A2A21EE021A30EEE4
:100F7000010A8DED1C0A9DED1D0A30EE000A8DED73
:100F80001B0A9DED1C0A30EE000A8DED1A0A9DED3C
:100F9000170ADDED0D0A30EEA02A9DED151A31EE8F
:100FA000422A9DED061A31EE021A20EE010A9DED4D
:100FB000181ADDED123A33EEA32A9DED143A32EE03
:100FC000032A9DED053A32EE432A21EE021A70EE15
:100FD000014A9DED1C3A309890ED011A90ED020AFD
:100FE000D0ED032A63EE001A9DED1D2A9DED0C7ACB
:100FF000B6EE004A8DED004A77EE445A9DED0A5A4E
:1010000035EE255A62EE055A9DED115A75EE606A6D
:1010100063EE266A75EEA66ADDED095A75EEA65AEC
:1010200061EEA51A71EEA41A62EE222A23EE011ACD
:1010300031EE621ADDED0E2ADDED104A72EEE42A81
:1010400062EE222ADDED0B4A73EEA43A63EE233AF8
:1010500072EEA32ADDED083A72EEE32A21EE221A9F
:1010600031EE211A22EE000A35EE205A22EE052A30
:101070009DED0F5A34EE455A35EE475A23EE053AA8
:1010800032EE032A9DED073A32EE432A20EE020AA1
:1010900030EE010A8DED2B0A9DED160ADDED0D2ACD
:1010A00032EEA21A9DED152A31EE421A9DED062A66
:1010B00031EE421A20EE010A9DED191ADDED126A99
:1010C00036EEA62A9DED143A32EE032A9DED053A3E
:1010D00032EE432A21EE021A30EE011A3098D0ED9A
:1010E000005AD0ED014AD0ED023A90ED032AB1EE5C
:1010F000000A24EE803A9DED0F7A37EE075A75EE1E
:10110000461ADDED0C0A30EEA05A75EE211A9DED5F
:10111000045A35EE215A23EE053A31EE031A9DEDBD
:101120001C5A65EE027A9DED1D3A74EE601A9DED33
:101130000A8A71EEC81A23EE218ADDED111A32EE09
:10114000E19A25EE099A38EE098A9DED099A38EE62
:10115000498A67EE887A31EE271A63EE233A65EE04
:10116000255A73EEA53ADDED0E5ADDED107A75EED7
:10117000E75A63EE255ADDED0B7A76EEA76A65EE47
:10118000266A75EEA65ADDED086A75EEE65A63EE3C
:10119000A53A31EE231A23EE022ADDED1A3A63EE68
:1011A000A43A32EE632A71EEA21A23EE213A34EE0B
:1011B000477A37EE607A25EE075A33EE053A9DED11
:1011C000075A33EE453A22EE032A31EE021A8DED2C
:1011D0002A1A9DED191ADDED0D0A30EEA03A9DEDAB
:1011E000152A32EE433A9DED062A32EE032A21EE0D
:1011F000021A9DED162ADDED124A34EEA43A9DED59
:10120000145A33EE053A9DED055A33EE453A22EE77
:10121000032A31EE022A309890ED001AD0ED011A1F
:10122000D0ED022AD0ED033A22EE800A9DED0F5A4E
:1012300035EE053A33EE467A9DED0C6A36EE063A07
:1012400033EE077A9DED043A33EE073A20EE030AB7
:1012500070EE025A9DED1B0A20EE620A9DED1C3ACB
:1012600023EE012A30EE420A9DED1D2A34EE467A25
:10127000DDED0A6A37EE667A62EE076A9DED117A55
:1012800070EEC77A63EE277A76EEA76ADDED097A0B
:1012900076EEE76A20EE260A30EE250A62EE211A83
:1012A00063EE233A71EEA31ADDED0E3ADDED105A2E
:1012B00073EEE53A62EE233ADDED0B5A74EEA54A81
:1012C00063EE244A73EEA43ADDED084A73EEE43A85
:1012D00061EEA31A30EE210A22EE011ADDED1A1A90
:1012E00061EEA21A31EE611A37EE207A22EE072A59
:1012F00034EE455A35EE465A23EE053A32EE032ACD
:101300009DED073A32EE432A21EE021A30EE010A31
:101310008DED290A9DED180A9DED0D7A37EE071A1D
:101320009DED152A31EE421A9DED062A31EE421A44
:1013300020EE010A9DED171ADDED122A32EEA22AE7
:101340009DED143A32EE032A9DED053A32EE432A22
:1013500021EE021A70EE013A9DED1B1A3098D0ED85
:10136000001A90ED010AD0ED020A90ED032A21EE59
:10137000022A9DED1C3A23EE001A31EE421A9DED31
:101380001D2A9DED0C5A34EE456ADDED0A4A36EE13
:10139000646A62EE064A9DED116A77EE465A63EE84
:1013A000255A74EEA54ADDED095A74EEE54A21EEA0
:1013B000241A31EE231A62EE211A63EE200A70EE2F
:1013C000E10ADDED0E1ADDED103A71EEE31A62EE80
:1013D000211ADDED0B3A72EEA32A63EE222A71EE9A
:1013E000A21ADDED082A71EEE21A60EEA10A31EED2
:1013F000201A22EE000A36EE076A22EE062A9DED3A
:101400000F6A34EE464A34EE454A23EE043A32EE91
:10141000032A9DED073A32EE432A20EE020A30EE0F
:10142000010A8DED280A9DED2B0A20EE000A9DEDA4
:101430002A1A21EE011A30EE010A9DED291A21EE39
:10144000011A30EE010A9DED281A21EE011A30EE44
:10145000010A09F0AFFE8DED2C0A9DED2C1A9DEDD1
:101460002B0A20EE010A8DED2B0A9DED2C1A9DED25
:101470002A0A20EE010A8DED2A0A9DED2C1A9DED17
:10148000290A20EE010A8DED290A9DED2C1A9DED09
:10149000280A20EE010A8DED280A40F27400C2F2FB
:1014A000000090ED000A9DED2B1A20EE011A9DED33
:1014B000270A30EE410A8DED270A90ED000A9DEDD6
:1014C0002A1A20EE011A9DED260A30EE410A8DED12
:1014D000260A90ED000A9DED291A20EE011A9DEDD5
:1014E000250A30EE410A8DED250A90ED000A9DEDAA
:1014F000281A20EE011A9DED240A30EE410A8DEDE6
:10150000240AFFE79DED271A309890ED000A90ED30
:10151000042A21EE021A30EE010A80ED000A9DED48
:10152000261A309890ED010A90ED042A21EE021A55
:1015300030EE010A80ED010A9DED251A309890EDFC
:10154000020A90ED042A21EE021A30EE010A80ED23
:10155000020A9DED241A309890ED030A90ED042ABA
:1015600021EE021A30EE010A80ED030A309890ED68
:10157000000A90ED013A90ED022A90ED031A20EE58
:10158000000A23EE033A30EE030A22EE022A30EE7E
:10159000020A21EE011A30EE010A09F00BFE8DED70
:1015A0002C0A9DED2C1A309890ED000A20EE010ACD
:1015B00080ED000A9DED2C1A309890ED010A20EE86
:1015C000010A80ED010A9DED2C1A309890ED020A77
:1015D00020EE010A80ED020A9DED2C1A309890ED64
:1015E000030A20EE010A80ED030A00208DF8C700EF
:1015F000FFE79DF9C70032B0BDEC048B80BD000051
:1016000080B5A0B01E901D911C921E9820B9FFE7D6
:10161000FF208DF87F00D3E21D9820B9FFE7FF205F
:101620008DF87F00CCE21C9820B9FFE7FF208DF8F1
:101630007F00C5E240F27401C2F2000142F60230BE
:10164000C3F6075008601D9800681B901D984068FD
:101650001A901D98806819901C98006818901C9822
:10166000406817901C98806816901E989DED183A57
:1016700090ED010A90ED022A90ED031A20EE430A44
:101680009DED173A22EE032A30EE420A9DED162A0E
:1016900021EE021A30EE410AB6EE001A20EE010ADF
:1016A0008DED100A1E989DED184A90ED000A90ED00
:1016B000023A90ED032A20EE040A9DED164A23EE2D
:1016C000043A30EE030A9DED173A22EE032A30EE7B
:1016D000420A20EE010A8DED0F0A1E989DED174A71
:1016E00090ED000A90ED013A90ED032A20EE040AF5
:1016F0009DED164A23EE043A30EE430A9DED183A6A
:1017000022EE032A30EE020A20EE010A8DED0E0AC7
:101710001E989DED164A90ED000A90ED013A90ED6D
:10172000022A20EE040A9DED174A23EE043A30EE19
:10173000030A9DED183A22EE032A30EE420A20EE0B
:10174000010A8DED0D0A9DED1B0AB5EE400AF1EE82
:1017500010FA11D1FFE79DED1A0AB5EE400AF1EE3D
:1017600010FA09D1FFE79DED190AB5EE400AF1EE36
:1017700010FA00F0AE81FFE79DED1B0A20EE000A93
:101780009DED1A1A21EE011A30EE010A9DED191A8B
:1017900021EE011A30EE010A09F00CFD8DED150A5B
:1017A0009DED151A9DED1B0A20EE010A8DED1B0A19
:1017B0009DED151A9DED1A0A20EE010A8DED1A0A0B
:1017C0009DED151A9DED190A20EE010A8DED190AFD
:1017D0001E9890ED000A30EE000A8DED0C0A1E985E
:1017E00090ED010A30EE000A8DED0B0A1E9890ED87
:1017F000020A30EE000A8DED0A0A1E9890ED030AE7
:1018000030EE000A8DED090A1E9890ED000AB1EE47
:10181000003A20EE030A8DED080A1E9890ED010AA9
:1018200020EE030A8DED070A1E9890ED020A20EEC5
:10183000030A8DED060A1E9890ED010AB2EE001A19
:1018400020EE010A8DED050A1E9890ED020A20EEA9
:10185000010A8DED040A1E9890ED000A20EE000AA0
:101860008DED030A1E9890ED010A20EE000A8DED21
:10187000020A1E9890ED020A20EE000A8DED010A80
:101880001E9890ED030A20EE000A8DED000A9DEDF2
:10189000081A9DED010A21EE000A9DED0A2A9DED30
:1018A0001B4A22EE042A30EE020A9DED022A21EEA6
:1018B000021A30EE010A9DED0B1A9DED1A2A21EE57
:1018C000021A30EE410A8DED140A9DED071A9DEDC6
:1018D000000A21EE000A9DED092A9DED1B4A22EE29
:1018E000042A30EE420A9DED032A22EE032A1E98B6
:1018F00090ED014A22EE042A30EE020A9DED0C2AF8
:101900009DED1A4A22EE042A30EE420A30EE410AD8
:101910009DED052A9DED024A22EE044A30EE040AAE
:101920009DED014A22EE042A30EE020A9DED192AAD
:1019300021EE021A30EE010A8DED130A9DED030A25
:1019400020EE030A1E9890ED021A20EE010A9DED8A
:101950000C1A9DED1B2A21EE021A30EE010A9DEDB4
:10196000061A9DED002A21EE022A30EE020A9DEDB4
:10197000092A9DED1A4A22EE042A30EE420A30EE80
:10198000410A9DED042A9DED024A22EE044A30EE02
:10199000040A9DED014A22EE042A30EE020A9DED72
:1019A000192A21EE021A30EE010A8DED120A9DED80
:1019B000020A20EE030A1E9890ED032A20EE020A86
:1019C0009DED0B1A9DED1B4A21EE041A30EE410AE3
:1019D0009DED011A21EE031A21EE021A30EE010AE2
:1019E0009DED0A1A9DED1A2A21EE021A30EE410AE7
:1019F0008DED110A9DED140A20EE000A9DED131ADB
:101A000021EE011A30EE010A9DED121A21EE011AA3
:101A100030EE010A9DED111A21EE011A30EE010A95
:101A200009F0C8FB8DED150A9DED151A9DED140A00
:101A300020EE010A8DED140A9DED151A9DED130A95
:101A400020EE010A8DED130A9DED151A9DED120A87
:101A500020EE010A8DED120A9DED151A9DED110A79
:101A600020EE010A8DED110A40F27400C2F200006E
:101A700090ED000A9DED141A20EE011A9DED100A5A
:101A800030EE410A8DED100A90ED000A9DED131A1B
:101A900020EE011A9DED0F0A30EE410A8DED0F0A7E
:101AA00090ED000A9DED121A20EE011A9DED0E0A2E
:101AB00030EE410A8DED0E0A90ED000A9DED111AEF
:101AC00020EE011A9DED0D0A30EE410A8DED0D0A52
:101AD000FFE79DED101A1E9890ED000A90ED042A84
:101AE00021EE021A30EE010A80ED000A9DED0F1A78
:101AF0001E9890ED010A90ED042A21EE021A30EEB4
:101B0000010A80ED010A9DED0E1A1E9890ED020A61
:101B100090ED042A21EE021A30EE010A80ED020A4D
:101B20009DED0D1A1E9890ED030A90ED042A21EE0A
:101B3000021A30EE010A80ED030A1E9890ED000AA9
:101B400090ED013A90ED022A90ED031A20EE000A82
:101B500023EE033A30EE030A22EE022A30EE020AA6
:101B600021EE011A30EE010A09F024FB8DED150A71
:101B70009DED151A1E9890ED000A20EE010A80EDE9
:101B8000000A9DED151A1E9890ED010A20EE010A3B
:101B900080ED010A9DED151A1E9890ED020A20EEC7
:101BA000010A80ED020A9DED151A1E9890ED030AB8
:101BB00020EE010A80ED030A00208DF87F00FFE788
:101BC0009DF97F0020B080BD84B08DED030ACDED7E
:101BD000020A9DED030A9DED021AB1EE411AB4EE20
:101BE000410AF1EE10FA07DAFFE79DED020AB1EEC5
:101BF000400A8DED010A18E09DED030A9DED021AE1
:101C0000B4EE410AF1EE10FA05DDFFE79DED020AA0
:101C10008DED000A04E09DED030A8DED000AFFE75B
:101C20009DED000A8DED010AFFE79DED010A04B06C
:101C30007047000080B541F63460C2F200000068D1
:101C400008210FF02DF980BD80B582B040F26062AE
:101C5000C2F20002002001901221132300F02CFA9E
:101C6000019802B080BD000080B5022001214FF034
:101C7000FF320FF067F980BD81B000909FED010A3F
:101C800001B070470000C84380B541F63460C2F22D
:101C90000000006810210FF003F980BD80B540F20C
:101CA0006060C2F20000C21D01200221062300F084
:101CB00003FA002080BD000080B5042001214FF010
:101CC000FF320FF03FF980BD80B58AB008900791D0
:101CD000089820B9FFE7FE208DF82700B4E00798A8
:101CE00020B9FFE7FE208DF82700ADE041F2221079
:101CF000C2F200000078C00720B1FFE7FD208DF898
:101D00002700A1E00FF0ACF941F63461C2F2000106
:101D1000086020B9FFE7FE208DF8270094E00798BF
:101D20000899C862002006907E21B622049200F035
:101D300059FA049A0120142100F054FA1E2005904B
:101D400001F0C2FA0599069800F0F2F906990846E2
:101D500000F0EEF91E2804D0FFE7FC208DF82700E4
:101D600072E00120002100F0E3F90F2804D0FFE722
:101D7000FC208DF8270067E00320019001F014F8A3
:101D80000420029001F010F842F25D02C0F6000259
:101D9000002003900121009101F034FA019841F6EE
:101DA0003541C0F6000101F07DF8029841F6894105
:101DB000C0F6000101F076F803984021AA2200F055
:101DC00011FA009A0398412100F00CFA039853216C
:101DD000082200F007FA029A0398582100F002FA4C
:101DE000029A03987D2100F0FDF9322001F06CFA8F
:101DF000009A0F21104600F0F5F90098019A102181
:101E000000F0F0F90098039A162100F0EBF9009A1F
:101E10001821104600F0E6F900981521802200F004
:101E2000E1F90A2001F050FA0099019841F22212DA
:101E3000C2F20002117000F0E3FF029800F0E0FF30
:101E400003988DF82700FFE79DF927000AB080BDB1
:101E500084B00290029820B9FFE7FE208DF80F00B1
:101E60006AE040F26061C2F20001B1F80100ADF831
:101E70000600B1F80300ADF80400B1F80500ADF8B4
:101E80000200BDF9060000EE100AB8EEC00A029882
:101E900080ED040ABDF9040000EE100AB8EEC00A95
:101EA000029880ED050ABDF9020000EE100AB8EEB6
:101EB000C00A029880ED060A029890ED040A9FED90
:101EC000201A80EE010A80ED040A029890ED050ABE
:101ED00080EE010A80ED050A029890ED060A80EE78
:101EE000010A80ED060A487C897CC00040EA511056
:101EF000ADF80000BDF90000B0F5806F07DBFFE72B
:101F0000BDF80000A0F50060ADF80000FFE7BDF9E6
:101F1000000000EE100AB8EEC00AB4EE001A20EE7F
:101F2000010AB3EE071A30EE010A029880ED0A0AA0
:101F300000208DF80F00FFE79DF90F0004B07047F7
:101F400000A0AA4584B00290029820B9FFE7FE20C5
:101F50008DF80F007AE040F26060C2F20000B0F845
:101F60000710ADF80610B0F80910ADF80410B0F87D
:101F70000B00ADF80200BDF9060000EE100AB8EE45
:101F8000C00A029880ED070ABDF9040000EE100AAD
:101F9000B8EEC00A029880ED080ABDF9020000EE12
:101FA000100AB8EEC00A029880ED090A029890ED76
:101FB000070A9FED281A80EE010A80ED070A0298B1
:101FC00090ED080A80EE010A80ED080A029890ED73
:101FD000090A80EE010A80ED090A029890ED070ACD
:101FE0009FED1D1A20EE010A80ED070A029890ED80
:101FF000080A20EE010A80ED080A029890ED090A0D
:1020000020EE010A80ED090A0298C16A91ED001ADA
:1020100090ED070A30EE410A80ED070A0298C16A86
:1020200091ED011A90ED080A30EE410A80ED080AA0
:102030000298C16A91ED021A90ED090A30EE410A48
:1020400080ED090AFE208DF80F00FFE79DF90F00D3
:1020500004B070476F12034235FA8E3C80B5012000
:1020600000F0FAFE68B9FFE70121084600F062FFC0
:1020700041F63460C2F20000006802210EF010FF49
:10208000FFE7022000F0E8FE68B9FFE70220012127
:1020900000F050FF41F63460C2F2000000680421F5
:1020A0000EF0FEFEFFE780BD80B5182001214FF045
:1020B000FF320EF047FF80BD80B586B08DF8170067
:1020C0008DF8161004928DF80F30049808B9FFE7C8
:1020D0002BE09DF817000146029120B1FFE702981E
:1020E000012805D009E00120002100F023FF04E0D1
:1020F0000220002100F01EFFFFE79DF8160040F0CF
:10210000800040F27361C2F2000108700122009267
:1021100000230193184601F097F8009B0198049959
:102120009DF80F2001F02EF8FFE706B080BD0000FB
:1021300080B586B08DF816008DF81510012001F0DD
:10214000C3F89DF816000146049120B1FFE70498FA
:10215000012805D009E00120002100F0EBFE04E099
:102160000220002100F0E6FEFFE79DF8150040F098
:10217000800040F27361C2F20001019108700122F7
:1021800000230293184601F05FF80199029B022296
:10219000184600F0F7FF9DF816000146039120B1A4
:1021A000FFE7039801280CD017E00121084600F052
:1021B000C1FE40F27360C2F2000040788DF8170053
:1021C0000BE00220012100F0B5FE40F27360C2F284
:1021D000000000788DF81700FFE79DF8170006B0A3
:1021E00080BD000080B584B08DF80F008DF80E1012
:1021F0008DF80D209DF80E0000F07F0040F2736115
:10220000C2F2000108709DF80D004870012001F035
:102210005BF89DF80F000146029120B1FFE702989C
:10222000012805D009E00120002100F083FE04E030
:102230000220002100F07EFEFFE740F27361C2F24F
:10224000000102220023184600F0FEFF9DF80F0057
:102250000146019120B1FFE70198012805D009E06E
:102260000121084600F066FE04E00220012100F092
:1022700061FEFFE704B080BD80B586B08DF8160022
:1022800004918DF80F209DF80F0020B9FFE70A2078
:102290008DF80F00FFE741F2A060C2F20000006875
:1022A00064210EF0D9FC20B1FFE7FB208DF8170068
:1022B00070E041F29C60C2F2000000680290FFE70B
:1022C0000298E0B1FFE7029800789DF81610884266
:1022D00011D1FFE702984068049988420BD1FFE7CB
:1022E00041F2A060C2F2000000680EF099FDFF20EC
:1022F0008DF817004EE0029800690290E0E7142084
:1023000000F040FE0190019858B9FFE741F2A0604B
:10231000C2F2000000680EF083FDFE208DF8170069
:1023200038E09DF80F001C2100220EF093FB01996C
:1023300088600198806870B9FFE7019800F02CFD73
:1023400041F2A060C2F2000000680EF069FDFF20BB
:102350008DF817001EE09DF816000199087004988A
:10236000019948609DF80F000199087341F29C6142
:10237000C2F200010868019A10610198086041F2F8
:10238000A060C2F2000000680EF04AFD00208DF847
:102390001700FFE79DF9170006B080BD82B00190DD
:1023A0008DF80310019802B07047000084B08DF8DA
:1023B0000B00019141F29C60C2F2000000680090A5
:1023C000FFE70098A8B1FFE7009800789DF80B1090
:1023D00088420AD1FFE7009840680199884204D1F9
:1023E000FFE700988068039006E00098006900907D
:1023F000E7E700200390FFE7039804B07047000070
:1024000082B000900098C068022809D1FFE70098C8
:1024100081680220042908BF03208DF8070008E026
:10242000009880680438B0FA80F040098DF8070001
:10243000FFE79DF8070002B07047000083B08DF8F9
:1024400007009DF80700022803DBFFE70020029049
:1024500018E09DF807000146009120B1FFE70098C1
:10246000012806D00BE040F63C40C2F2000002908A
:1024700008E040F66440C2F20000029002E0002052
:102480000290FFE7029803B07047000080B586B065
:102490008DF8160004910392029341F22010C2F2CB
:1024A00000000078C00720B9FFE7FD208DF8170075
:1024B00037E0039820B9FFE7FE208DF8170030E0E1
:1024C00041F2A060C2F20000006864210EF0C4FB7B
:1024D00020B1FFE7FB208DF8170022E09DF81600E1
:1024E0000499FFF763FF019041F2A060C2F200007F
:1024F00000680EF095FC019820B9FFE7FC208DF8EC
:1025000017000EE001980399029B00220EF042FA98
:1025100000900098002818BF4FF0FF308DF817008A
:10252000FFE79DF9170006B080BD000080B596B0AA
:1025300041F22010C2F200000078C00720B1FFE78E
:10254000FD208DF85700A7E040F2B440C2F2000031
:102550006821FDF7DAFF00201490FFE714980128A6
:1025600009DCFFE79DF8500000F01CFBFFE7149822
:1025700001301490F2E741F2E001C2F2000142F2B0
:102580009D30C0F60000086000200EF0B5FB01464B
:1025900041F2A060C2F200000160006820B9FFE7CC
:1025A000FF208DF8570077E041F22011C2F20001C0
:1025B00007910120089008700AA803902821FDF7D0
:1025C000A4FF0399089A002009900F900A900B909D
:1025D000109011920C900D9012920E220292139272
:1025E0000E9040F63C40C2F20000019003F048FD1E
:1025F000019804F043FC099842F2AD72C0F6000263
:10260000062100F06FF8099942F62D32C0F600025B
:102610000592084600F066F8059A0899099800F0B6
:1026200061F8059A09980221049100F05BF801987D
:10263000032103F04FFC029A039908980F920E9021
:1026400040F66440C2F20000069003F019FD0698BF
:1026500004F014FC089842F69102C0F6000208212A
:1026600000F040F8059A0999089800F03BF8059A9F
:102670000899084600F036F80499059A089800F081
:1026800031F80698112103F025FC079A089909985A
:1026900011708DF85700FFE79DF9570016B080BD07
:1026A00080B584B002908DF8071041F2E000C2F2CC
:1026B0000000006858B1FFE741F2E000C2F20000FC
:1026C000026802989DF807109047039006E0029870
:1026D0009DF80710FFF762FE0390FFE7039804B030
:1026E00080BD000082B08DF806008DF805100092C4
:1026F00041F22010C2F200000078C00720B9FFE7C5
:10270000FD208DF807002AE0009820B9FFE7FE20A1
:102710008DF8070023E09DF80600022804DBFFE7A0
:10272000FF208DF807001AE09DF805000D2804DB56
:10273000FFE7FF208DF8070011E000989DF80610D4
:1027400040F2B443C2F20003342211FB02319DF87F
:10275000052041F8220000208DF80700FFE79DF9D1
:10276000070002B07047000080B584B08DF80E00FD
:1027700002918DF8072041F22010C2F2000000788B
:10278000C00720B9FFE7FD208DF80F0009E09DF894
:102790000E0002999DF80720FFF76EFD8DF80F00DF
:1027A000FFE79DF90F0004B080BD000080B598B030
:1027B00000200E90FFE70E98012867DCFFE79DF8E8
:1027C0003800FFF73BFE0D900D9808B9FFE759E080
:1027D000FFE70D98002103F04BFD002851D0FFE7E3
:1027E0000D98002111AA0FAB03F06CFD002847D112
:1027F000FFE7139818B9FFE71198019002E01298CB
:102800000190FFE701980C9011A8FFF7F9FD8DF8F2
:102810002F000C989DF82F10FFF742FF0A909DF8AB
:1028200038000A99FFF7C2FD0990099838B3FFE70D
:102830000020089007900690059004900390029065
:102840009DF82F008DF808000C9803900A980490CA
:1028500015988DF81400149838B9FFE702A80D30C8
:10286000159A0FA9FDF7D2FDFFE705F023FA0890AE
:10287000099802A900231A460EF06CF9FFE7FFE75A
:10288000A7E7FFE70E9801300E9094E718B080BDDF
:1028900080B598B000200E90FFE70E98012867DC05
:1028A000FFE79DF83800FFF7C9FD0D900D9808B9B6
:1028B000FFE759E0FFE70D98012103F0D9FC00285C
:1028C00051D0FFE70D98012111AA0FAB03F0FAFCDC
:1028D000002847D1FFE7139818B9FFE71198019036
:1028E00002E012980190FFE701980C9011A8FFF701
:1028F00087FD8DF82F000C989DF82F10FFF7D0FE64
:102900000A909DF838000A99FFF750FD0990099840
:1029100038B3FFE7002008900790069005900490D8
:10292000039002909DF82F008DF808000C980390FA
:102930000A98049015988DF81400149838B9FFE798
:1029400002A80D30159A0FA9FDF760FDFFE705F00D
:10295000B1F90890099802A900231A460EF0FAF876
:10296000FFE7FFE7A7E7FFE70E9801300E9094E737
:1029700018B080BD80B592B0844614988DF846C0DA
:102980008DF8451010920F938DF83B0041F2201006
:10299000C2F200000078C00720B9FFE7FD208DF8E3
:1029A00047009EE09DF84600022804DBFFE7FF2079
:1029B0008DF8470095E00F9870B9FFE79DF8450046
:1029C000022809D0FFE79DF84500032804D0FFE75F
:1029D000FE208DF8470084E09DF83B00092804DBC9
:1029E000FFE7FF208DF847007BE09DF84600FFF7EA
:1029F00025FD0D900D9820B9FFE7FE208DF84700CA
:102A00006FE0002001900C900B900A9009900890C4
:102A10000790069005909DF8450001460291032815
:102A20001FD80299DFE801F002080F1610980590F0
:102A300000200790089018E0109806900420079056
:102A40000020089011E010980590002007900220C7
:102A500008900AE010980690042007900220089041
:102A600003E0FF208DF847003BE09DF83B00099014
:102A700000208DF828000F9868B1FFE79DF83B0013
:102A8000012808DBFFE705A818300F999DF83B20C7
:102A9000FDF7BCFCFFE70D9803F01EFD90B1FFE7CA
:102AA0000D9805A901F1180204AB03F03DFA8DF869
:102AB0000F009DF80F0020B9FFE700208DF84700B8
:102AC0000FE0FFE79DF8460005A900F00FF920B1DF
:102AD000FFE700208DF8470003E0FF208DF8470056
:102AE000FFE79DF9470012B080BD000080B584B0BB
:102AF0008DF80E000291029820B9FFE7FE208DF8B4
:102B00000F000EE09DF80E0002990A684B1D09792E
:102B1000EC46CCF800100021FFF72CFF8DF80F00D9
:102B2000FFE79DF90F0004B080BD000080B58CB0B8
:102B300000200B90FFE70B98012831DCFFE70B9892
:102B40008DF82B009DF82B00FFF778FC0990099871
:102B500008B9FFE720E0FFE79DF82B0000F044F8FC
:102B6000C8B9FFE7099803F0B7FC08B9FFE712E01E
:102B70009DF82B0001A900F063F808B9FFE70AE00F
:102B8000099801A901F118026B4603F0CDF908B1CB
:102B9000FFE700E0E0E7FFE70B9801300B90CAE7A2
:102BA0000CB080BD81B08DF803009DF803000228B1
:102BB00001DBFFE715E09DF8030000EBC01041F6D4
:102BC0003861C2F2000101EBC0020020C2F800042B
:102BD0009DF8032002EBC21201EBC201C1F804040C
:102BE000FFE701B07047000081B08DF802009DF84A
:102BF0000200022804DBFFE701208DF803001AE041
:102C00009DF8020000EBC01041F63861C2F20001ED
:102C100001EBC000D0F800049DF8022002EBC212C4
:102C200001EBC201D1F80414401AB0FA80F0400957
:102C30008DF80300FFE79DF8030001B07047000026
:102C4000B0B584B08DF80E0002919DF80E000128F9
:102C500003DCFFE7029820B9FFE700208DF80F00A2
:102C600040E09DF80E0000EBC01141F63860C2F262
:102C7000000000EBC10001900198D0F80004019918
:102C8000D1F80414884204D1FFE700208DF80F002A
:102C900028E0029900910198D0F8043400EB431227
:102CA0005B01C0585368D2F808C0D2F80CE0146930
:102CB00055694D610C61C1F80CE0C1F808C04B606A
:102CC00008609069D269CA6188610198D0F80404EB
:102CD000013000F01F000199C1F8040401208DF8B3
:102CE0000F00FFE79DF80F0004B0B0BDF0B585B050
:102CF0008DF8120003919DF81200012803DCFFE714
:102D0000039820B9FFE700208DF8130040E09DF8FC
:102D1000120000EBC01141F63860C2F2000000EB77
:102D2000C10002900298D0F80004013000F01F00AA
:102D3000019001980299D1F80414884204D1FFE768
:102D400000208DF8130023E0029ED6F8000406EB65
:102D500040114701039A0092D2F810E054691568B7
:102D600050689368D2F80CC0F5514C61C1F810E07E
:102D7000C1F80CC08B6048609069D269CA618861F3
:102D800001980299C1F8000401208DF81300FFE7B3
:102D90009DF8130005B0F0BD80B582B00190019898
:102DA0000FF062FC02B080BD80B582B08DF80600E5
:102DB0009DF8060001460091052815D80099DFE826
:102DC00001F0031313070B0F062005F0F7F90FE0CE
:102DD0000A2005F0F3F90BE0172005F0EFF907E002
:102DE000092005F0EBF903E0FF208DF8070003E070
:102DF00000208DF80700FFE79DF9070002B080BDB5
:102E000080B582B08DF806009DF80600014600915D
:102E1000052815D80099DFE801F0031313070B0FFD
:102E2000062005F0D5F90FE00A2005F0D1F90BE0F6
:102E3000172005F0CDF907E0092005F0C9F903E0F6
:102E4000FF208DF8070003E000208DF80700FFE762
:102E50009DF9070002B080BD80B582B08DF80600F4
:102E60009DF80600072804DBFFE700208DF8070027
:102E700013E09DF8062046F66001C0F6010101EB63
:102E8000C200406831F8321004F0E4FE0138B0FAB4
:102E900080F040098DF80700FFE79DF8070002B0B9
:102EA00080BD000083B08DF80A000191019820B91F
:102EB000FFE7FE208DF80B0038E09DF80A00072898
:102EC00004DBFFE7FF208DF80B002FE09DF80A10D0
:102ED00046F66000C0F6010030F83100ADF802009F
:102EE00000208DF80100FFE79DF801000F2819DC94
:102EF000FFE7BDF802009DF80110C840C00750B1BF
:102F0000FFE701989DF8012040F21C51C2F2000138
:102F100041F8220006E0FFE79DF8010001308DF83E
:102F20000100E1E700208DF80B00FFE79DF90B00A1
:102F300003B0704780B582B08DF806008DF805109B
:102F40009DF80600072804DBFFE7FF208DF8070047
:102F500014E09DF8062046F66001C0F6010101EB81
:102F6000C200406831F832109DF8052002F00102DD
:102F700004F088FE00208DF80700FFE79DF90700A8
:102F800002B080BD80B582B0019001980FF0CAF800
:102F900002B080BD86B08DF816008DED040A9DF854
:102FA0001600052804DBFFE7FF208DF817008CE0F2
:102FB0009DED040AB7EE001AB4EE410AF1EE10FAE4
:102FC00004DDFFE74FF07E500490FFE79DED040A1B
:102FD000B5EE400AF1EE10FA03DAFFE700200490A4
:102FE000FFE79DF8161046F69800C0F6010050F86D
:102FF00031100968C96A03919DED040A03990131F2
:1030000001EE101AB8EE411A20EE010ABCEEC00A19
:103010008DED020A9DF8161000EBC100808860B9A2
:10302000FFE702989DF8162046F69801C0F60101C8
:1030300051F832100968486343E09DF8161046F6CF
:103040009800C0F6010000EBC100808804280DD173
:10305000FFE702989DF8162046F69801C0F6010198
:1030600051F8321009688863019028E09DF8161025
:1030700046F69800C0F6010000EBC10080880828E1
:103080000DD1FFE702989DF8162046F69801C0F68C
:10309000010151F832100968C86300900CE00298F1
:1030A0009DF8162046F69801C0F6010151F832103D
:1030B000096808640090FFE700980190FFE7019815
:1030C000FFE700208DF81700FFE79DF9170006B015
:1030D0007047000080B582B08DF806009DF80600AC
:1030E000052804DBFFE7FF208DF8070010E09DF8BE
:1030F000062046F69800C0F6010000EBC20150F829
:103100003200898807F082FA00208DF80700FFE777
:103110009DF9070002B080BD80B582B08DF8060031
:103120009DF80600052804DBFFE7FF208DF8070067
:1031300010E09DF8062046F69800C0F6010000EB6E
:10314000C20150F83200898807F046FB00208DF854
:103150000700FFE79DF9070002B080BD82B08DF83F
:1031600003009DF8030030B9FFE740F62070C2F27B
:103170000000019002E000200190FFE7019802B0FA
:103180007047000080B584B08DF80E000291ADF854
:1031900006208DF805309DF80E00012804DBFFE7BE
:1031A000FF208DF80F0029E09DF80E00FFF7D6FFF5
:1031B0000090009820B9FFE7FF208DF80F001DE078
:1031C0009DF80500C00760B1FFE700980299BDF8BF
:1031D000062005F0F1FF002818BF01208DF80F0030
:1031E0000CE000980299BDF80620142305F0BCFEFF
:1031F000002818BF01208DF80F00FFE79DF90F0090
:1032000004B080BD82B08DF806008DF805100092E4
:10321000009820B9FFE7FE208DF8070010E0009825
:103220009DF8062040F26451C2F2000101EB421108
:103230009DF8052041F8220000208DF80700FFE7E7
:103240009DF9070002B0704780B584B08DF80E007C
:103250000291ADF806208DF805309DF80E0001288A
:1032600004DBFFE7FF208DF80F0029E09DF80E003A
:10327000FFF774FF0090009820B9FFE7FF208DF85A
:103280000F001DE09DF80500C00760B1FFE7009842
:103290000299BDF8062006F0DDFC002818BF0120C9
:1032A0008DF80F000CE000980299BDF80620142359
:1032B00006F0A2F8002818BF01208DF80F00FFE7E4
:1032C0009DF90F0004B080BD80B586B004900DF06C
:1032D000ABFA01464FF47A70B0FBF1F0039004981A
:1032E0000399B0FBF1F002900DF060FA0146481C22
:1032F000019198B1FFE70198022820D3FFE70198D8
:1033000002280FD0FFE701980338022806D3FFE711
:1033100001986FF00041884215D1FFE7FF208DF83A
:10332000170014E0029818B1FFE70298009002E03D
:1033300001200090FFE700980DF0F2F903E00498F7
:1033400004F03AFAFFE700208DF81700FFE79DF937
:10335000170006B080BD000080B58AB00DF064FA99
:10336000079010F07BFF079A4FF47A710191B1FB3F
:10337000F2F1484306904EF21800CEF2000002909F
:103380000068059010F06AFF019A01460298079BB9
:10339000B2FBF3F25143049100680390069804993C
:1033A000884215D1FFE704984FF47A72504305998B
:1033B00051434EF21402CEF2000212680132B1FB08
:1033C000F2F1401A00F57A7000210991089014E09A
:1033D00004984FF47A725043039951434EF2140209
:1033E000CEF2000212680132B1FBF2F1401A00F590
:1033F0007A70002109910890FFE7089809990AB0AE
:1034000080BD000083B08DF807009DF807000146DD
:10341000009120B1FFE70098012806D00BE041F2AF
:103420005000C2F20000029008E041F29800C2F29F
:103430000000029002E000200290FFE7029803B033
:103440007047000080B582B0019001980068006864
:10345000C00600282AD5FFE7FFE70020009001986A
:10346000006800680090019800684068009000982B
:10347000FFE701980CF0C6FC00EBC00140F2885059
:10348000C2F2000000EB8100006A70B1FFE7019812
:103490000CF0B8FC00EBC00140F28850C2F2000012
:1034A00000EB8100006A8047FFE7FFE702B080BDC4
:1034B00082B08DF806008DF805100092009820B9B2
:1034C000FFE7FE208DF8070020E09DF806000128A8
:1034D00005DCFFE79DF80500092804DBFFE7FF2076
:1034E0008DF8070012E000989DF8061001EBC1026C
:1034F00040F28851C2F2000101EB82019DF80520E3
:1035000041F8220000208DF80700FFE79DF9070031
:1035100002B07047FFE7FEE780B540F63C40C2F2DC
:10352000000003F011F880BD80B540F63C40C2F2C7
:10353000000003F009F880BD80B540F63C40C2F2BF
:10354000000003F001F880BD80B540F66440C2F28F
:10355000000002F0F9FF80BD80B540F66440C2F281
:10356000000002F0F1FF80BD80B540F66440C2F279
:10357000000002F0E9FF80BD82B00090009820B901
:10358000FFE703208DF807001DE00098006846F271
:103590000041C4F20001884204D1FFE700208DF809
:1035A000070010E00098006846F60001C4F2000130
:1035B000884204D1FFE701208DF8070003E00320D3
:1035C0008DF80700FFE79DF8070002B07047000084
:1035D00082B001908DF80310019800699DF80310E6
:1035E00000EB4100407A02B07047000082B00190C9
:1035F0008DF80310019800699DF8031000EB41005D
:10360000007A02B07047000080B588B006908DF84F
:10361000171006989DF81710FFF7E8FF8DF81600B1
:1036200006989DF81710FFF7D3FF8DF815009DF849
:10363000160010280FD1FFE7069890F8240000F03C
:1036400001008DF81400069890F82A0000F001009F
:103650008DF8130027E09DF8160011280FD1FFE721
:10366000069890F8250000F001008DF814000698E7
:1036700090F82B0000F001008DF8130012E006987E
:10368000C08C9DF81610C84000F001008DF81400A1
:103690000698808D9DF81610C84000F001008DF846
:1036A0001300FFE7FFE79DF815000146039140B1C5
:1036B000FFE70398012815D0FFE70398022824D0DC
:1036C0002AE09DF814100020C907029021B9FFE7F5
:1036D0009DF813000290FFE7029800F001008DF8BA
:1036E0001F001DE09DF814100020C907019031B1A2
:1036F000FFE79DF8130080F001000190FFE70198BB
:1037000000F001008DF81F000AE09DF8140000F0A1
:1037100001008DF81F0003E000208DF81F00FFE777
:103720009DF81F0008B080BD82B001908DF8031095
:1037300000208DF80200019890F84000012807D180
:10374000FFE79DF8020040F001008DF80200FFE75E
:10375000019890F85400012807D1FFE79DF8020076
:1037600040F002008DF80200FFE7019890F8640035
:10377000012807D1FFE79DF8020040F004008DF812
:103780000200FFE79DF803109DF802000840401A70
:10379000B0FA80F0400902B07047000080B586B0F2
:1037A0008DED050ACDED040A03909DED030AB8EEF8
:1037B000400A9FED151A20EE010A11F0AFFE9FEDB1
:1037C000131A20EE010AB0EEC00A9DED051A30EE84
:1037D000010A8DED020A9DED020A9DED041AB4EE78
:1037E000410AF1EE10FA05DDFFE79DED040A8DEDCB
:1037F000010A04E09DED020A8DED010AFFE79DED4F
:10380000010A06B080BD00BF6F12833ACDCC4C3E9A
:1038100080B592B010900F910E92109818B1FFE7FA
:103820000F9820B9FFE7FE208DF847009FE10E9822
:10383000109A059211685268401A4FF000010691E3
:10384000914112F012FF05990246069800EE102AE7
:103850009FEDC91A80EE010A81ED020A0E99109AB5
:103860005060116030B9FFE7109880680CF07AFD65
:1038700060B914E01098806812F0A2FE41EC100BC1
:1038800051EC100B0CF046FD48B1FFE7109890ED9D
:10389000020AB5EE400AF1EE10FA07DCFFE71099D4
:1038A00041F26F20C3F683208860FFE7109890ED07
:1038B000020A9FEDB21AB4EE410AF1EE10FA07DAED
:1038C000FFE7109941F26F20C3F603208860FFE7FD
:1038D000109890ED020A9FEDAA1AB4EE410AF1EE9B
:1038E00010FA07DDFFE710994CF6CD40C3F64C50B7
:1038F0008860FFE710980F9909780E9A00F0A2FAF5
:103900001098007C01460491012804D0FFE7049838
:10391000052806D00EE010990020886110994861B2
:1039200042E00F984068109948610F98806810999C
:10393000886139E0109890ED0C1A90EDB70A30EEDE
:10394000410A8DED0D0A9DED0D0A11F03FFD8DED43
:103950000C0A9DED0D0A11F0E1FD8DED0B0A9DEDB8
:103960000C0A0F9890ED011A90ED022A20EE010A40
:103970009DED0B1A21EE021A30EE410A109880EDEF
:10398000050A9DED0B0A0F9890ED011A90ED022AA1
:1039900020EE010A9DED0C1A21EE021A30EE010A0A
:1039A000109880ED060AFFE71098007C014603910D
:1039B00006284BD80399DFE801F004040D1E3304F8
:1039C000080010990020C86140E00F98C068109965
:1039D000C8613BE0109901F59C70D1ED021A91EDA0
:1039E0000C0AD1EDB70A9FED6A1A09F09DFA1098FA
:1039F00080ED070A2AE0109901F59C70D1ED021ABA
:103A000091ED0C0AD1EDB70A9FED601A30EE010A74
:103A10009FED5F1A09F088FA109880ED070A15E00B
:103A2000109890ED0D0A8DED020A0E989FED550A43
:103A3000DFED550AFFF7B2FEB0EE401A9DED020A27
:103A400020EE010A109880ED070AFFE7109B03F1B2
:103A5000120003F1140103F1380293F911309FEDC4
:103A60004D0A08F0B1FF00208DF82B00FFE79DF80C
:103A70002B00109991F91110884274DAFFE7109821
:103A80009DF82B1000EB8100806B099010999DF838
:103A90002B2001EB421000F5C67001EB021191EDF5
:103AA000A80A07F0C3FB8DED080A1098007C0146B8
:103AB000019170B3FFE701980138052804D3FFE7AF
:103AC0000198062817D027E010999DF82B20C2EB0B
:103AD000021001EB8000483001EB820292ED0E0AE9
:103AE000DDED080AD1ED021A9FED291A09F01CFA42
:103AF0008DED070A10E010989DF82B1000EB810067
:103B000090ED0E0A9FED241A80EE010A8DED070A52
:103B100002E000200790FFE710989DF82B1000EBC3
:103B2000411000F503709DED070A07F07FFB109828
:103B30009DF82B1000EB810080EDA30A10999DF8F1
:103B40002B0001EB800000F52370C968D1ED1F0A3E
:103B5000B1EE600A00F0DEFAFFE79DF82B000130BD
:103B60008DF82B0083E700208DF84700FFE79DF9D3
:103B7000470012B080BD00BF00007A446F12033AC4
:103B8000CDCC4C3D9A99193FCDCC4C3FAB611C3FFD
:103B9000000000000000FA4300C0DA4580B58AB09A
:103BA000089007918DED060A089820B9FFE7FE20DE
:103BB0008DF82700F0E0FEF7B9FC07980899C86077
:103BC000089900200874079890F860000146039156
:103BD00006282ED80399DFE801F0040B12181F2CD9
:103BE000250008990420487400208DF8170024E06F
:103BF00008990420487401208DF817001DE00899E9
:103C0000022048748DF8170017E0089904204874C2
:103C100003208DF8170010E00899042048748DF8EF
:103C200017000AE008990120487405208DF8170054
:103C300003E0FC208DF82700AEE0089900204860E2
:103C40000860089988608DF81600FFE79DF8160057
:103C5000089991F91110884251DAFFE708989DF808
:103C60001610C1EB011100EB810048309DED060AF2
:103C7000079901F120020021029109F0CDFA08987C
:103C80009DF8161000EB411000F5C6709DED060A78
:103C90000799D1ED190A07F025FB08989DF8161031
:103CA00000EB411000F503709DED060A0799D1ED78
:103CB0001A0A07F017FB029808999DF8162001EBE5
:103CC0000211C1F8A00208999DF8162001EB02111B
:103CD000C1F8A40208999DF8162001EB0211C1F861
:103CE0009C0208999DF8162001EB0211C1F8A80268
:103CF000FFE79DF8160001308DF81600A6E708983A
:103D000000F59C709DED060A079901F14002002123
:103D1000019109F081FA089812309DF8171008F007
:103D2000A5FF01980899C8610899886108994861B8
:103D30008DF81500FFE79DF81500089991F911100D
:103D400088420FDAFFE708989DF8151000EB810113
:103D50000020C1F88C02FFE79DF8150001308DF8B6
:103D60001500E8E700200490FFE70498089991F90E
:103D7000111088420CDAFFE70898C068049900EB3C
:103D8000C10008F0F5F8FFE7049801300490ECE773
:103D900000208DF82700FFE79DF927000AB080BDBD
:103DA00080B586B00590059808B9FFE748E0002087
:103DB0008DF81300FFE79DF81300059991F9111094
:103DC00088421CDAFFE705989DF8131000EB81008C
:103DD000006A0390039808B9FFE70AE00398059981
:103DE0009DF8132001EB820191EDA30A08F05CF924
:103DF000FFE79DF8130001308DF81300DBE700208A
:103E00008DF80B00FFE79DF80B00059991F9111053
:103E1000884215DAFFE705989DF80B1000EB81004A
:103E2000006A0190019820B1FFE7019807F002FFB6
:103E3000FFE7FFE79DF80B0001308DF80B00E2E78C
:103E400006B080BD80B586B004908DF80F10029248
:103E5000049820B9FFE7FE208DF8170068E09DF870
:103E60000F000499097C884204D1FFE700208DF8F7
:103E700017005DE09DF80F0004281CD1FFE70498AF
:103E8000007C042817D0FFE70298FCF7A1FAFCF7A2
:103E9000EDF900EBD07121F00101411A0120002958
:103EA00018BF4FF0FF3000EE100AB8EEC00A0498B9
:103EB00080ED0D0AFFE700208DF80700FFE79DF871
:103EC0000700049991F91110884229DAFFE7049854
:103ED0009DF80710C1EB011100EB8100483009F09B
:103EE00067FA04989DF8071000EB411000F5C670C2
:103EF0009FED110A8DED000A07F092FA9DED000A80
:103F000004989DF8071000EB411000F5037007F0CE
:103F100087FAFFE79DF8070001308DF80700CEE72C
:103F20009DF80F000499087400208DF81700FFE732
:103F30009DF9170006B080BD0000000080B586B076
:103F4000049000208DF80F00FFE79DF80F00049902
:103F500091F91110884245DAFFE70498C0689DF88E
:103F60000F1000EBC10008F02DF90498C0689DF80F
:103F70000F1000EBC10007F097FF02900298049920
:103F80009DF80F2001EB8201086204989DF80F1044
:103F900000EB8100006A01900298C0B1FFE704982D
:103FA0009DF80F1000EB0111DDF808C0DCF80800E7
:103FB000DCF80C20DCF81030DCF814C0C1F8A8C222
:103FC000C1F8A432C1F8A022C1F89C0203E0FE208F
:103FD0008DF817000AE0FFE79DF80F0001308DF81B
:103FE0000F00B2E700208DF81700FFE79DF91700DA
:103FF00006B080BD84B003908DED020ACDED010ABC
:10400000039890ED000A9DED021A30EE010A8DED45
:10401000000A9DED010AB5EE400AF1EE10FA26DD28
:10402000FFE79DED000A9DED011AB4EE410AF1EEA5
:1040300010FA09DBFFE79DED011A9DED000A30EE55
:10404000410A8DED000A11E09DED000AB5EE400A2F
:10405000F1EE10FA09DAFFE79DED011A9DED000A75
:1040600030EE010A8DED000AFFE7FFE7FFE7009859
:104070000399086004B0704785B08DED040ACDED5A
:10408000030A8DED021A9DED040A9DED031A30EE30
:10409000410A8DED010A9DED020AB5EE400AF1EEEE
:1040A00010FA32DDFFE79DED020AB0EE001A80EE55
:1040B000010A8DED000A9DED010A9DED001AB4EE96
:1040C000410AF1EE10FA09DDFFE79DED021A9DEDC0
:1040D000010A30EE410A8DED010A15E09DED010A5D
:1040E0009DED001AB1EE411AB4EE410AF1EE10FA5C
:1040F00009DAFFE79DED021A9DED010A30EE010A93
:104100008DED010AFFE7FFE7FFE79DED010A05B02E
:104110007047000083B002908DED010ACDED000ADA
:10412000029890ED000A9DED001AB4EE410AF1EEFE
:1041300010FA04DDFFE7009802990860FFE7029893
:1041400090ED000A9DED011AB4EE410AF1EE10FA6D
:1041500004DAFFE7019802990860FFE703B07047AF
:1041600080B584B00290029820B9FFE7FF208DF857
:104170000F0017E0029800F09FF88DF807009DF8F7
:104180000700029981F840009DF80700029981F824
:1041900054009DF80700029981F8640000208DF812
:1041A0000F00FFE79DF90F0004B080BD80B586B019
:1041B0000490049820B9FFE7FF208DF8170074E001
:1041C0000498FFF7CDFF0498143000F011FC049818
:1041D0001C3000F031FA04982E3000F00DF90498EC
:1041E000303000F055FCFFF7B7F812F03EFA00EE61
:1041F000100A9FED301A8DED021A80EE010A049824
:1042000080ED000AFFF7A8F8049A03929368D26839
:10421000C01A914112F029FA9DED021A0146039845
:1042200000EE101A80EE010A80ED010AFFF794F803
:104230000A460499CA608860049890F840000328F0
:104240000CDCFFE7049890F85400032806DCFFE735
:10425000049890F86400042807DBFFE7049800F056
:10426000D3F8FD208DF817001FE0049890F8402047
:1042700040F22431C2F20001019101EB02114968C0
:1042800088470199049890F8542001EB021189683D
:1042900088470199049890F8642001EB0211C968DD
:1042A000884700208DF81700FFE79DF9170006B03A
:1042B00080BD00BF0024744980B586B00490002002
:1042C0000390FFE7039803283FDCFFE704980069A9
:1042D000039910F811008DF80B009DF80B000146B2
:1042E000019103282CD80199DFE801F016200C0277
:1042F000049800F0EFFB20B1FFE703208DF81700D2
:1043000027E01DE0049800F0CBFB20B1FFE702207E
:104310008DF817001DE013E0049800F0D3FB20B1E6
:10432000FFE700208DF8170013E009E0049800F083
:10433000C1FB20B1FFE701208DF8170009E0FFE77E
:10434000FFE7039801300390BCE705208DF81700C4
:10435000FFE79DF8170006B080BD000083B0019014
:104360000091019818B1FFE7009820B9FFE7FF20FE
:104370008DF80B0006E000980199086100208DF887
:104380000B00FFE79DF90B0003B0704782B000906F
:10439000009820B9FFE7FF208DF8070003E0002018
:1043A0008DF80700FFE79DF9070002B07047000095
:1043B00082B00090009820B9FFE7FF208DF8070039
:1043C00003E000208DF80700FFE79DF9070002B029
:1043D0007047000082B00090009820B9FFE7FF20EE
:1043E0008DF8070003E000208DF80700FFE79DF936
:1043F000070002B07047000081B0009000990020D3
:10440000087001B07047000082B00090009820B999
:10441000FFE7FF208DF807000AE00099002081F8EF
:104420004400009981F85800009981F86600FFE780
:104430009DF9070002B0704780B584B002900298E1
:1044400020B9FFE7FF208DF80F0035E0029900202A
:10445000C864029988640190FFE701980D2827D865
:10446000FFE7019946F6E010C0F60100405C8DF8C8
:10447000030002989DF80310FFF756F998B1FFE783
:1044800002989DF80410FFF7BFF858B1FFE70199B3
:1044900040F20400C2F2000000EBC1004168029843
:1044A0008847FFE7FFE7FFE7019801300190D4E775
:1044B00000208DF80F00FFE79DF90F0004B080BDCC
:1044C00080B584B00290029820B9FFE7FF208DF8F4
:1044D0000F0059E00299012081F858000298B0F9C4
:1044E0001E1000EE101AB8EEC00A90ED011A20EE70
:1044F000010A016991ED091A20EE010A80ED170AFF
:104500000298B0F9201000EE101AB8EEC00A90ED33
:10451000011A20EE010A016991ED091A20EE010A43
:1045200080ED180A00200190FFE701980D2827D898
:10453000FFE7019946F6E010C0F60100405C8DF8F7
:10454000030002989DF80310FFF7EEF898B1FFE71B
:1045500002989DF80410FFF757F858B1FFE701994A
:1045600040F20400C2F2000000EBC1004168029872
:104570008847FFE7FFE7FFE7019801300190D4E7A4
:1045800000208DF80F00FFE79DF90F0004B080BDFB
:1045900080B584B00290029820B9FFE7FF208DF823
:1045A0000F0045E00299002081F868000190FFE7C4
:1045B00001980D2827D8FFE7019946F6E010C0F6CC
:1045C0000100405C8DF8030002989DF80310FFF78E
:1045D000ABF898B1FFE702989DF80410FFF714F8C4
:1045E00058B1FFE7019940F20400C2F2000000EB6D
:1045F000C100416802988847FFE7FFE7FFE701989D
:1046000001300190D4E70299C88C8885029991F80D
:10461000240000F0010081F82A00029991F8250099
:1046200000F0010081F82B0000208DF80F00FFE75B
:104630009DF90F0004B080BD81B00090009900206A
:10464000087001B07047000081B0009000980169C7
:1046500091ED0B1A90ED120A20EE010A80ED120A7C
:104660000098016991ED0B1A90ED130A20EE010AF2
:1046700080ED130A002001B07047000081B0009067
:10468000002001B07047000081B0009000980169DF
:1046900091ED0A1A90ED130A30EE410A80ED130AEB
:1046A000002001B07047000081B00090002001B0F0
:1046B0007047000081B000900098016991ED0C1ADC
:1046C00090ED120A20EE010A80ED120A00980169AD
:1046D00091ED0C1A90ED130A20EE010A80ED130AF9
:1046E000002001B07047000081B0009000990120C7
:1046F00081F86800002001B07047000081B0009090
:10470000009991F86600013081F86600009991F8EF
:10471000660000F0030081F86600002001B07047D9
:1047200081B000900099032081F84400002001B07E
:104730007047000081B000900098016991ED0A1A5D
:1047400090ED130A30EE010A80ED130A002001B04B
:104750007047000081B000900098016991ED0A1A3D
:1047600090ED120A30EE410A80ED120A002001B0ED
:104770007047000081B00090002001B07047000039
:1047800081B00090002001B07047000081B000901F
:104790000098016991ED0A1A90ED120A30EE010AB3
:1047A00080ED120A002001B07047000081B0009037
:1047B0000099042081F844000099022081F8450006
:1047C000002001B07047000083B00190019820B92B
:1047D000FFE7FF208DF80B0033E001988069007E31
:1047E00001460091012812D0FFE70098022804D06A
:1047F000FFE70098032805D00EE00199002081F81A
:1048000044000EE00199022081F8440009E001997A
:10481000042081F8440004E00199002081F844005C
:10482000FFE7019988698068886401998869406810
:10483000C86401998869C068086500208DF80B007C
:10484000FFE79DF90B0003B07047000083B00190B3
:10485000019820B9FFE7FF208DF80B005BE001987D
:104860008069807E0146009101282CD0FFE70098E6
:10487000022804D0FFE70098032809D03EE0019900
:10488000002081F858000199C865019908663EE04A
:104890000199012081F8580040F20060C2F2000046
:1048A00090ED011AB1EE410A30EE410A019981ED15
:1048B000170A90ED020ABFEE081A20EE010A0198CD
:1048C00080ED180A23E00199012081F8580040F298
:1048D0000060C2F2000090ED011AB1EE410A30EE24
:1048E000410A019981ED170A90ED020ABFEE081AFC
:1048F00020EE010A019880ED180A08E001990020D5
:1049000081F858000199C86501990866FFE7002001
:104910008DF80B00FFE79DF90B0003B07047000016
:1049200084B00290029820B9FFE7FF208DF80F00B5
:1049300059E040F20060C2F200000078029900F0F5
:10494000010081F8650002988069807D014601912F
:10495000012819D0FFE70198022804D0FFE7019849
:10496000032808D018E00299012081F86700029915
:1049700081F8680018E00299012081F86700029927
:10498000002081F868000FE00299002081F867009C
:10499000029981F8680007E00299002081F8670019
:1049A000029981F86800FFE702988069C07D01469E
:1049B0000091012809D0FFE7009802280AD1FFE7FB
:1049C0000299012081F8660009E00299022081F82D
:1049D000660004E00299002081F86600FFE70020ED
:1049E0008DF80F00FFE79DF90F0004B0704700003D
:1049F00080B582B0019041F2BC60C2F2000000902C
:104A00000BF082FD00980199486001994868007890
:104A100000F001000870019901204870002002B0E8
:104A200080BD000082B00090009820B9FFE7FF2011
:104A30008DF8070003E000208DF80700FFE79DF9DF
:104A4000070002B07047000082B00090009820B9C3
:104A5000FFE7FF208DF8070003E000208DF8070036
:104A6000FFE79DF9070002B07047000082B0009098
:104A7000009820B9FFE7FF208DF8070003E0002031
:104A80008DF80700FFE79DF9070002B070470000AE
:104A900081B0009000990020087001B070470000BC
:104AA00081B00090009890F82E0000F0010001B055
:104AB0007047000081B000900098007F00F0010076
:104AC00001B0704781B000900098007D00F00100B7
:104AD00001B0704781B00090009890F8300000F06D
:104AE000010001B07047000040F28400C2F20000F3
:104AF0007047000080B584B00290029820B9FFE7AB
:104B0000FE208DF80F002BE041F22110C2F20000D0
:104B10000078C00720B1FFE7FD208DF80F001FE0EF
:104B20000CF09EFA41F63061C2F20001086020B933
:104B3000FFE7FE208DF80F0012E045F24152C0F66B
:104B40000002002001900321FEF7B2FC019841F21F
:104B50002112C2F20002012111708DF80F00FFE74F
:104B60009DF90F0004B080BD80B59CB01B901A91D8
:104B70001B994878897840EA01216FF3DF2141F2DF
:104B8000A460C2F20000199001801B9A9178D2783B
:104B9000C90841EA42116FF3DF2141801B9AD178A5
:104BA00013795279890941EA830141EA82216FF33D
:104BB000DF2181801B9A51799279490841EAC2111B
:104BC0006FF3DF21C1801B9A9179D279090941EAFB
:104BD00002116FF3DF2101811B9AD179137A527A86
:104BE000C90941EA430141EA42216FF3DF214181D2
:104BF0001B9A517A927A890841EA82116FF3DF2178
:104C000081811B9A917AD27A490941EAC201C18114
:104C10001B9A117B527B41EA02216FF3DF21018253
:104C20001B9A517B927BC90841EA42116FF3DF2145
:104C300041821B9A917BD37B127C890941EA8301D3
:104C400041EA82216FF3DF2181821B9A117C527C21
:104C5000490841EAC2116FF3DF21C182B0F90610A1
:104C600000EE101AB8EEC00A9FEDDA1A30EE010A13
:104C700030EE000A9FEDD82A80EE020AB7EE001A45
:104C800030EE410A1A9981ED010AB0F9041000EEE4
:104C9000101AB8EEC00A9FEDD13A30EE030A30EE9A
:104CA000000A9FEDCF3A80EE030A30EE410A1A99CE
:104CB00081ED020AB0F9001000EE101AB8EEC00A39
:104CC0009FEDC83A30EE030A30EE000A9FEDC63A77
:104CD00080EE030A30EE410A1A9981ED030AB0F919
:104CE000020000EE100AB8EEC00A9FEDC03A30EEA6
:104CF000030A30EE000A80EE020A30EE410A1A98EA
:104D000080ED040A1A98406811F05AFC41EC100B2F
:104D10009FEDB71B50EC111BC20F51EC100B62F34F
:104D2000DF7141EC100B51EC100B9FEDB30B53EC0A
:104D3000102B11F07EFC20B9FFE71A990020486083
:104D4000FFE71A98806811F03BFC41EC100B9FEDD7
:104D5000A81B50EC111BC20F51EC100B62F3DF715A
:104D600041EC100B51EC100B9FEDA50B53EC102BED
:104D700011F05FFC20B9FFE71A9900208860FFE777
:104D80001A98C06811F01CFC41EC100B9FED981BA9
:104D900050EC111BC20F51EC100B62F3DF7141ECB0
:104DA000100B51EC100B9FED940B53EC102B11F0EA
:104DB00040FC20B9FFE71A990020C860FFE71A9865
:104DC000006911F0FDFB41EC100B9FED891B50ECCD
:104DD000111BC20F51EC100B62F3DF7141EC100B91
:104DE00051EC100B9FED840B53EC102B11F021FCB8
:104DF00020B9FFE71A9900200861FFE71A98406878
:104E000011F0DEFB41EC100B9FED791B50EC111BF8
:104E1000C20F51EC100B62F3DF7141EC100B51EC3F
:104E2000100B9FED790B53EC102B11F017FC88B988
:104E3000FFE71A9890ED012AB7EE001ABFEE000ABC
:104E4000B5EE402AF1EE10FAC8BFB0EE410A80ED8F
:104E5000010AFFE71A98806811F0B2FB41EC100BD1
:104E60009FED631B50EC111BC20F51EC100B62F352
:104E7000DF7141EC100B51EC100B9FED630B53EC09
:104E8000102B11F0EBFB88B9FFE71A9890ED022A7E
:104E9000B7EE001ABFEE000AB5EE402AF1EE10FAA6
:104EA000C8BFB0EE410A80ED020AFFE71A98C06859
:104EB00011F086FB41EC100B9FED4D1B50EC111BCC
:104EC000C20F51EC100B62F3DF7141EC100B51EC8F
:104ED000100B9FED4D0B53EC102B11F0BFFB88B95D
:104EE000FFE71A9890ED032AB7EE001ABFEE000A0A
:104EF000B5EE402AF1EE10FAC8BFB0EE410A80EDDF
:104F0000030AFFE71A98006911F05AFB41EC100BF5
:104F10009FED371B50EC111BC20F51EC100B62F3CD
:104F2000DF7141EC100B51EC100B9FED370B53EC84
:104F3000102B11F093FB88B9FFE71A9890ED042A23
:104F4000B7EE001ABFEE000AB5EE402AF1EE10FAF5
:104F5000C8BFB0EE410A80ED040AFFE741F2A46049
:104F6000C2F20000B0F90800B0F5967F0DDDFFE752
:104F700041F2A460C2F20000B0F90800B0F5FA7F77
:104F800003DAFFE7012018905BE041F2A460C2F26F
:104F90000000B0F90800B0F5FA7F0EDBFFE741F240
:104FA000A460C2F20000B0F9080040F2DB51884270
:104FB00003DCFFE70320179040E041F2A460C2F257
:104FC0000000B0F90810002040F2DC529142169027
:104FD0002CDB1DE0000051C30060AD44000032C373
:104FE0000020AC44000052C30040AD4400005DC34B
:104FF0000000000000000000000000A09999A93FF7
:10500000000000A09999C93F000000000000F03F97
:1050100041F2A460C2F20000B0F9081040F2A462AC
:1050200000209142B8BF01201690FFE7169800F0CB
:105030000100002818BF02201790FFE7179818906A
:10504000FFE718981A99087541F2A460C2F20000AF
:10505000B0F90A00B0F5967F0DDDFFE741F2A460DC
:10506000C2F20000B0F90A00B0F5FA7F03DAFFE7F8
:10507000012015903DE041F2A460C2F20000B0F9B9
:105080000A00B0F5FA7F0EDBFFE741F2A460C2F23E
:105090000000B0F90A0040F2DB51884203DCFFE770
:1050A0000320149022E041F2A460C2F20000B0F9A3
:1050B0000A10002040F2DC52914213900EDBFFE711
:1050C00041F2A460C2F20000B0F90A1040F2A462FA
:1050D00000209142B8BF01201390FFE7139800F021
:1050E0000100002818BF02201490FFE714981590C3
:1050F000FFE715981A99487541F2A460C2F20000C2
:10510000B0F90C00B0F5967F0DDDFFE741F2A46029
:10511000C2F20000B0F90C00B0F5FA7F03DAFFE745
:10512000012012903DE041F2A460C2F20000B0F90B
:105130000C00B0F5FA7F0EDBFFE741F2A460C2F28B
:105140000000B0F90C0040F2DB51884203DCFFE7BD
:105150000320119022E041F2A460C2F20000B0F9F5
:105160000C10002040F2DC52914210900EDBFFE761
:1051700041F2A460C2F20000B0F90C1040F2A46247
:1051800000209142B8BF01201090FFE7109800F076
:105190000100002818BF02201190FFE7119812901B
:1051A000FFE712981A99887541F2A460C2F20000D4
:1051B000B0F90E00B0F5967F0DDDFFE741F2A46077
:1051C000C2F20000B0F90E00B0F5FA7F03DAFFE793
:1051D00002200F903AE041F2A460C2F20000B0F960
:1051E0000E00B0F5FA7F0EDBFFE741F2A460C2F2D9
:1051F0000000B0F90E0040F2DB51884203DCFFE70B
:1052000003200E901FE041F2A460C2F20000B0F94A
:105210000E10002040F2DC5291420D900EDBFFE7B1
:1052200041F2A460C2F20000B0F90E1040F2A46294
:1052300000209142B8BF01200D90FFE70D9800F0CB
:1052400001000E90FFE70E980F90FFE70F981A9954
:10525000C87541F2A460C2F20000B0F91000B0F5C8
:10526000967F0DDDFFE741F2A460C2F20000B0F9C5
:105270001000B0F5FA7F03DAFFE702200C903AE065
:1052800041F2A460C2F20000B0F91000B0F5FA7F5C
:105290000EDBFFE741F2A460C2F20000B0F910009B
:1052A00040F2DB51884203DCFFE703200B901FE054
:1052B00041F2A460C2F20000B0F91010002040F2E8
:1052C000DC5291420A900EDBFFE741F2A460C2F289
:1052D0000000B0F9101040F2A46200209142B8BF63
:1052E00001200A90FFE70A9800F001000B90FFE709
:1052F0000B980C90FFE70C981A99087641F2A4607D
:10530000C2F20000B0F91200B0F5967F0DDDFFE7A4
:1053100041F2A460C2F20000B0F91200B0F5FA7FC9
:1053200003DAFFE7022009903AE041F2A460C2F2FA
:105330000000B0F91200B0F5FA7F0EDBFFE741F292
:10534000A460C2F20000B0F9120040F2DB518842C2
:1053500003DCFFE7032008901FE041F2A460C2F2E3
:105360000000B0F91210002040F2DC529142079088
:105370000EDBFFE741F2A460C2F20000B0F91210A8
:1053800040F2A46200209142B8BF01200790FFE7DD
:10539000079800F001000890FFE708980990FFE7E0
:1053A00009981A99487641F2A460C2F20000B0F957
:1053B0001400B0F5967F0DDDFFE741F2A460C2F264
:1053C0000000B0F91400B0F5FA7F03DAFFE701201E
:1053D00006903DE041F2A460C2F20000B0F9140072
:1053E000B0F5FA7F0EDBFFE741F2A460C2F20000E5
:1053F000B0F9140040F2DB51884203DCFFE70320E0
:10540000059022E041F2A460C2F20000B0F914104D
:10541000002040F2DC52914204900EDBFFE741F2A3
:10542000A460C2F20000B0F9141040F2A46200209F
:105430009142B8BF01200490FFE7049800F00100FA
:10544000002818BF02200590FFE705980690FFE7A7
:1054500006981A99887641F2A460C2F20000B0F969
:105460001600B0F5967F0DDDFFE741F2A460C2F2B1
:105470000000B0F91600B0F5FA7F03DAFFE702206A
:1054800003903AE041F2A460C2F20000B0F91600C5
:10549000B0F5FA7F0EDBFFE741F2A460C2F2000034
:1054A000B0F9160040F2DB51884203DCFFE703202D
:1054B00002901FE041F2A460C2F20000B0F91610A1
:1054C000002040F2DC52914201900EDBFFE741F2F6
:1054D000A460C2F20000B0F9161040F2A4620020ED
:1054E0009142B8BF01200190FFE7019800F0010050
:1054F0000290FFE702980390FFE703981A99C87695
:1055000041F2A460C2F20000B0F916100020B1F51B
:10551000967F00900CD0FFE741F2A460C2F2000039
:10552000B0F90000B0F57A7018BF01200090FFE7D5
:1055300000981A9900F0010008701CB080BD0000AE
:1055400080B541F63060C2F20000006880210BF0A7
:10555000A7FC80BD80B582B000900020FDF752FF0F
:105560000099192205F07AFD20B9FFE700208DF897
:10557000070003E0FF208DF80700FFE79DF9070013
:1055800002B080BD80B582B00190019A80200121D7
:105590000BF0D8FC8038B0FA80F0400902B080BD32
:1055A00080B540F6AC50C2F2000001F05BFE80BD59
:1055B00080B540F68C40C2F2000001F053FE80BD81
:1055C00080B540F60C60C2F2000001F04BFE80BDD9
:1055D00080B540F6EC40C2F2000001F043FE80BD11
:1055E00080B540F64C50C2F2000001F03BFE80BD99
:1055F00080B540F66C60C2F2000001F033FE80BD61
:1056000082B001900198007810384AF6AB21CAF6B2
:10561000AA21A0FB011000090090009946F658004D
:10562000C0F60100405C0199C8650098042807D3C2
:10563000FFE701990868042262F30900886506E023
:105640000199086840F2FF3290438865FFE70198AE
:10565000806D02B07047000086B0059000208DF884
:1056600013000598806A03900598806910BBFFE7D6
:105670000398029003281BD80299DFE801F0020D7D
:105680000218059890F82F00C00720B1FFE701200D
:105690008DF81300FFE70CE00598C06AB0F1C07FF9
:1056A00004D1FFE701208DF81300FFE701E000E0DF
:1056B000FFE745E005988069B0F5005F25D1FFE779
:1056C0000398019003281ED80199DFE801F0020633
:1056D000021101208DF8130016E0059890F82F00B4
:1056E000C00720B1FFE701208DF81300FFE70BE0B2
:1056F0000598C06AB0F1C07F04D1FFE701208DF8A2
:105700001300FFE700E0FFE719E00398009003288B
:1057100004D3FFE70098032804D00EE001208DF8A1
:1057200013000BE0059890F82F00C00720B1FFE7A9
:1057300001208DF81300FFE700E0FFE7FFE7FFE738
:105740009DF8130006B0704784B003900291019257
:10575000009303980168086820F48020086000988E
:1057600003990968486003988068402809D1FFE7D9
:105770000198039909688860029803990968C860CC
:1057800008E00298039909688860019803990968FC
:10579000C860FFE704B070477047000080B5012083
:1057A00002F060F880BD000080B5082002F05AF8D1
:1057B00080BD000080B5102002F054F880BD0000CC
:1057C00080B5202002F04EF880BD000072B6FFE7E1
:1057D000FEE7000080B592B010900F91109818B1BC
:1057E000FFE70F9820B9FFE7FF208DF84700C0E1E1
:1057F000FDF7B2FD109A049213685268C01A9141E5
:1058000010F033FF0146049800EE101A9FEDDB1AEA
:1058100080EE010A80ED020AFDF79EFD0A4610990E
:105820004A60086010980F99097800F07DFA0F9887
:1058300090ED010A109890ED021A20EE010AB7EEE1
:10584000081A20EE010A8DED0E0A1098C06890ED3E
:10585000280AB5EE400AF1EE10FA72DDFFE7109863
:1058600090ED5D1A90ED600A30EE410A8DED0D0A63
:105870009DED0D0A9FEDC21AB4EE410AF1EE10FA49
:1058800009DDFFE79DED0D0A9FEDBE1A30EE010A1E
:105890008DED0D0AFFE79DED0D0A9FEDBB1AB4EEED
:1058A000410AF1EE10FA09DAFFE79DED0D0A9FEDCE
:1058B000B71A30EE010A8DED0D0AFFE7109890ED52
:1058C000051A90ED440A9DED0D2A31EE021A9DED68
:1058D0000E2A71EE020A9FEDAD1A8DED031AFEF746
:1058E000CBFB9DED031A8DED0C0A109890ED052A67
:1058F00090ED450A9DED0D3A32EE032A9DED0E3AEC
:1059000072EE030AFEF7B8FB8DED0B0A9DED0E0A51
:105910009DED0C1AB4EE410AF1EE10FA03DDFFE73B
:105920000C980E90FFE79DED0E0A9DED0B1AB4EE5C
:10593000410AF1EE10FA03DAFFE70B980E90FFE749
:10594000FFE7109814309DED0E0ADFED900AFEF788
:1059500051FB0F9890ED020A109890ED021A20EE7C
:10596000010A8DED0A0A1098C06890ED290AB5EE7B
:10597000400AF1EE10FA6BDDFFE7002009909DED83
:10598000090A9FED7F1AB4EE410AF1EE10FA09DD23
:10599000FFE79DED090A9FED7B1A30EE010A8DEDC0
:1059A000090AFFE79DED090A9FED771AB4EE410A57
:1059B000F1EE10FA09DAFFE79DED090A9FED731A7F
:1059C00030EE010A8DED090AFFE7109890ED061AF6
:1059D00090ED460A9DED092A31EE021A9DED0A2A44
:1059E00071EE020A9FED691A8DED021AFEF744FB73
:1059F0009DED021A8DED080A109890ED062A90EDA3
:105A0000470A9DED093A32EE032A9DED0A3A72EEFD
:105A1000030AFEF731FB8DED070A9DED0A0A9DEDA5
:105A2000081AB4EE410AF1EE10FA03DDFFE7089818
:105A30000A90FFE79DED0A0A9DED071AB4EE410AB0
:105A4000F1EE10FA03DAFFE707980A90FFE7FFE7A5
:105A5000109818309DED0A0ADFED4C0AFEF7CAFADD
:105A60000F9890ED020AB0EE081A80EE010A9FED41
:105A7000481A30EE010A9FED471A30EE010A1098DD
:105A800080ED060A1098007C0146019140B1FFE7C5
:105A9000019801280CD0FFE7019802285DD064E04E
:105AA00010990020C1F860011099C1F864015CE010
:105AB000109901F12000D1ED021A91ED050AD1ED06
:105AC0005D0A9FED351A8DED001A07F02DFA9DED58
:105AD000001A8DED060A109901F1D4009DED060A19
:105AE000D1ED021AD1ED5C0A07F01EFA9DED001A05
:105AF000109880ED580A109901F19800D1ED021A22
:105B000091ED060AD1ED640A07F00EFA9DED001A38
:105B10008DED050A109901F1D4009DED050AD1ED36
:105B2000021AD1ED5A0A07F0FFF9109880ED590AD0
:105B3000109901F5907091ED580A05F077FB1098D7
:105B400080ED580A109901F5A07091ED590A05F001
:105B50006DFB109880ED590A07E010990020C1F8FC
:105B600060011099C1F86401FFE700208DF847003B
:105B7000FFE79DF9470012B080BD00BF00247449C3
:105B8000DB0F4940DB0FC9C0DB0F49C0DB0FC94049
:105B900052B83E40ABAAAA3E0000000080B586B0D5
:105BA000049003918DED020A049820B9FFE7FF20CD
:105BB0008DF817007BE003980499C86004980021D1
:105BC00001910174049A02F120009DED020AD2684D
:105BD000303207F021FB049901F15C009DED020ACF
:105BE000C96801F110020121009107F015FB01992C
:105BF000049A02F198009DED020AD268703207F013
:105C00000BFB0099049A02F1D4009DED020AD268C0
:105C1000503207F001FB049901F590709DED020AE6
:105C2000C968D1ED240A05F05DFB049901F5A07067
:105C30009DED020AC968D1ED240A05F053FB0498D2
:105C4000C16891ED260A91ED281A30EE010A80ED27
:105C5000440A0499C868D0F89800C1F8140104985F
:105C6000C16891ED270A91ED291A30EE010A80ED05
:105C7000460A0499C868D0F89C00C1F81C01FCF7DA
:105C800055FC0498C06805F0CBFD0498C068083046
:105C900005F0C6FD0498C06805F058FC0498C0687B
:105CA000083005F053FC01988DF81700FFE79DF9C7
:105CB000170006B080BD000080B58CB00B900020AE
:105CC00000900A9009900890079006900B9890ED2C
:105CD000590AB1EE041A20EE010A8DED060A4FF0C2
:105CE0007E500A900B98C06806A905F0C9FC009880
:105CF000059004900390029001900B9890ED580A43
:105D0000B2EE001A20EE010A8DED010A49F69A1052
:105D1000C3F6996005900B98C068083001A905F09A
:105D2000AFFC0CB080BD000080B584B002908DF84F
:105D30000710029820B9FFE7FF208DF80F0047E019
:105D40009DF807000299097C884204D1FFE70020F2
:105D50008DF80F003CE00298203007F029FB0298F4
:105D60005C3007F025FB0298983007F021FB029881
:105D7000D43007F01DFB029800F590709FED160AD5
:105D80008DED000A05F04CFB9DED000A029800F530
:105D9000A07005F045FB0298C068083005F0D6FBFE
:105DA0000298C06805F0D2FB02981430FAF710FE92
:105DB0000299D1F8900188610299D1F87401486183
:105DC0009DF807000299087400208DF80F00FFE786
:105DD0009DF90F0004B080BD0000000080B584B0C4
:105DE0000290029820B9FFE7FF208DF80F0045E0F0
:105DF0000298C06805F04CFE0298C06805F0FCFBF4
:105E000001900198A0B1FFE70299DDF804C0DCF829
:105E10001C00DCF82020DCF82430DCF828C0C1F8B5
:105E20009CC1C1F89831C1F89421C1F89001FFE7F5
:105E30000298C068083005F02BFE0298C068083050
:105E400005F0DAFB00900098A0B1FFE70299DDF8B9
:105E500000C0DCF81C00DCF82020DCF82430DCF882
:105E600028C0C1F88CC1C1F88831C1F88421C1F8BB
:105E70008001FFE700208DF80F00FFE79DF90F007C
:105E800004B080BD83B001900091019820B9FFE774
:105E9000FF208DF80B0019E00199009B18685A68E3
:105EA0009B68C1F87031C1F86C21C1F86801019993
:105EB000009BD8681A695B69C1F87C31C1F8782108
:105EC000C1F8740100208DF80B00FFE79DF90B006D
:105ED00003B0704784B002900191029890F82000BE
:105EE0008DF803009DF80300012805D0FFE79DF819
:105EF000030002280AD1FFE7019A02980168486965
:105F00001043486100208DF80F0008E00299486AAC
:105F100040F48020486201208DF80F00FFE79DF8D3
:105F20000F0004B07047000088B0069005910492FD
:105F30000393069890F820008DF8070006980068F3
:105F4000806800900598806808B9FFE700E0FFE7E7
:105F50009DF80700012806D0FFE79DF807000228FA
:105F600040F08080FFE79DF80300400700280CD434
:105F7000FFE79DF803000007002806D4FFE79DF81F
:105F80000300C006002864D5FFE70098C0F3016055
:105F90000290029901208840039908600598806862
:105FA00068B9FFE705980168C06840EA4150069962
:105FB0000968029A01EB0211C1F880010EE005990F
:105FC0004A688868C96840EAC200084306990968B7
:105FD000029A01EB0211C1F88001FFE70598006900
:105FE00006990968029A01EB0211C1F8840105982B
:105FF000007D01280CD1FFE706980068029900EBAC
:106000000111D1F8840140F48070C1F88401FFE7E8
:106010000498406806990968029A01EB0211C1F8D8
:106020008C010498006806990968029A01EB021134
:10603000C1F8880106980068029900EB0111D1F8B7
:10604000800140F00100C1F8800100208DF81F00A0
:1060500011E00699486A40F40010486201208DF86A
:106060001F0008E00699486A40F480204862012039
:106070008DF81F00FFE79DF81F0008B07047000073
:1060800086B004900391049890F820008DF80300E6
:106090009DF80300012806D0FFE79DF803000228C1
:1060A00040F0B080FFE746F20040C4F200000190EB
:1060B0000199D1F8000240F00100C1F800020199F5
:1060C000D1F8000220F47C50C1F800020398426A23
:1060D0000199D1F8000240EA0220C1F800020398B9
:1060E000406900F01F01012088400290029A019946
:1060F000D1F81C029043C1F81C020398C069F0B9A2
:10610000FFE7029A0199D1F80C029043C1F80C0202
:10611000039A9088D168526940EA0140019901EBE5
:10612000C201C1F84002039A10889168526940EA9E
:106130000140019901EBC201C1F84402FFE7039855
:10614000C06901281ED1FFE7029A0199D1F80C021B
:106150001043C1F80C02039A90881168526940EA12
:106160000140019901EBC201C1F84002039A9089F4
:106170009168526940EA0140019901EBC201C1F8FE
:106180004402FFE70398806940B9FFE7029A01994A
:10619000D1F804029043C1F8040207E0029A019981
:1061A000D1F804021043C1F80402FFE70398006924
:1061B00040B9FFE7029A0199D1F814029043C1F85F
:1061C000140207E0029A0199D1F814021043C1F8B1
:1061D0001402FFE70398006A012808D1FFE7029A3A
:1061E0000199D1F81C021043C1F81C02FFE7019984
:1061F000D1F8000220F00100C1F8000200208DF863
:10620000170008E00499486A40F4802048620120A1
:106210008DF81700FFE79DF8170006B070470000E3
:1062200080B582B001900198FDF7A6F98DF80300C2
:106230009DF80300032819D0FFE79DF8030040F202
:10624000B442C2F20002342110FB0120006B60B1A5
:10625000FFE79DF8030040F2B442C2F2000234218D
:1062600010FB0120006B8047FFE7FFE702B080BD15
:1062700084B00390029100200190039890F82000D0
:106280008DF803009DF80300012805D0FFE79DF875
:106290000300022812D1FFE7029838B9FFE70398FC
:1062A0000068C06800F00300019006E003980068F1
:1062B000006900F003000190FFE7FFE7019804B0D8
:1062C0007047000086B004900391029201930498F5
:1062D00090F820008DF803009DF80300012806D0F7
:1062E000FFE79DF80300022840F0E880FFE70398ED
:1062F00080B9FFE704980068C068800748B9FFE7E5
:106300000499486A40F40010486201208DF8170093
:10631000DDE00FE0049800680069800748B9FFE7F6
:106320000499486A40F40010486201208DF8170073
:10633000CDE0FFE704980068039900EB0110D0F866
:10634000B00100F00400029988600298806858B992
:10635000FFE704980068039900EB0110D0F8B00142
:10636000400D029908600AE004980068039900EB68
:106370000110D0F8B001C00802994860FFE7049806
:106380000068039900EB0110D0F8B00100F00200A2
:106390000299C86004980068039900EB0110D0F8D6
:1063A000B40100F00F00082804D3FFE70299082089
:1063B00008610BE004980068039900EB0110D0F825
:1063C000B40100F00F0002990861FFE7049800682B
:1063D000039900EB0110D0F8B40180B2000A0299D1
:1063E000886104980068039900EB0110D0F8B401AB
:1063F000000C0299486104980068039900EB0110B1
:10640000D0F8B8010199087004980068039900EB6E
:106410000110D0F8B801000A01994870049800688A
:10642000039900EB0110D0F8B801000C01998870B5
:1064300004980068039900EB0110D0F8B801000E31
:106440000199C87004980068039900EB0110D0F816
:10645000BC010199087104980068039900EB0110D0
:10646000D0F8BC01000A01994871049800680399AA
:1064700000EB0110D0F8BC01000C01998871049860
:106480000068039900EB0110D0F8BC01000E0199DF
:10649000C871039838B9FFE704980168C86840F0EC
:1064A0002000C86006E004980168086940F02000F8
:1064B0000861FFE700208DF8170008E00499486A9A
:1064C00040F48020486201208DF81700FFE79DF816
:1064D000170006B07047000083B0029000200190C2
:1064E000029890F820008DF803009DF80300012821
:1064F00005D0FFE79DF80300022822D1FFE70298AC
:10650000006880684001002804D5FFE70198013049
:106510000190FFE70298006880680001002804D518
:10652000FFE7019801300190FFE70298006880685A
:10653000C000002804D5FFE7019801300190FFE773
:10654000FFE7019803B0704780B58AB0099000203A
:1065500008900998006840690790099800684068A9
:106560000690099800688068059009980068C068DE
:106570000490099800680069039009980068806990
:1065800002909DF81C00C007002800F09480FFE7EF
:106590009DF81400C00758B3FFE70998016801206F
:1065A00088609DF814008007002804D5FFE709984B
:1065B00000F0D2FC1BE09DF814004007002805D530
:1065C000FFE7089840F4006008900FE09DF8140081
:1065D0000007002805D5FFE7089840F48050089090
:1065E00003E0099800F090FCFFE7FFE7FFE7FFE713
:1065F0009DF81500C00760B3FFE7099801684FF4E4
:10660000807088609DF815008007002804D5FFE79A
:10661000099800F0EFFC1BE09DF8150040070028EA
:1066200005D5FFE7089840F4005008900FE09DF86A
:1066300015000007002805D5FFE7089840F48040C2
:10664000089003E0099800F0ADFCFFE7FFE7FFE7E3
:10665000FFE79DF81600C00760B3FFE709980168DF
:106660004FF4803088609DF816008007002804D51C
:10667000FFE7099800F00EFD1BE09DF816004007AB
:10668000002805D5FFE7089840F4004008900FE087
:106690009DF816000007002805D5FFE7089840F48C
:1066A0008030089003E0099800F0CCFCFFE7FFE79A
:1066B000FFE7FFE7FFE79DF81C000007002810D563
:1066C000FFE79DF81000C006002809D5FFE70898ED
:1066D00040F400700890099801681020C860FFE736
:1066E000FFE79DF81C00400700280FD5FFE79DF845
:1066F00010000007002808D5FFE709980168082066
:10670000C860099800F0F2FAFFE7FFE79DF81C0067
:10671000800700280BD5FFE709980068C06880074C
:1067200020B1FFE7099800F009FBFFE7FFE79DF8BC
:106730001C004006002810D5FFE79DF80C00C0069D
:10674000002809D5FFE7089840F480600890099870
:10675000016810200861FFE7FFE79DF81C00800634
:1067600000280FD5FFE79DF80C000007002808D58A
:10677000FFE70998016808200861099800F006FB06
:10678000FFE7FFE79DF81C00C00600280BD5FFE7D8
:10679000099800680069800720B1FFE7099800F0B8
:1067A0001DFBFFE7FFE79DF81E00800700280FD5BF
:1067B000FFE79DF81800C006002808D5FFE70998F4
:1067C000016810204860099800F030FBFFE7FFE700
:1067D0009DF81E00C00778B1FFE79DF8180000077C
:1067E000002808D5FFE70998016808204860099843
:1067F00000F078FCFFE7FFE79DF81D000006002889
:1068000040F18D80FFE79DF818004007002840F117
:106810008180FFE79DF81D00C00750B1FFE79DF89C
:106820000800C00728B1FFE7089840F00100089071
:10683000FFE79DF81D00800700280BD5FFE79DF8B6
:1068400008008007002805D5FFE7089840F00200FF
:106850000890FFE79DF81D00400700280BD5FFE7D3
:106860009DF808004007002805D5FFE7089840F08C
:1068700004000890FFE79DF81D000007002848D598
:10688000FFE79DF8080010F0700F42D0FFE7029874
:1068900000F0700001460191102814D0FFE7019824
:1068A000202815D0FFE70198302816D0FFE701987F
:1068B000402817D0FFE70198502818D0FFE701982B
:1068C000602819D01DE0089840F00800089019E0F1
:1068D000089840F01000089014E0089840F020005C
:1068E00008900FE0089840F0400008900AE00898EF
:1068F00040F08000089005E0089840F4807008900F
:1069000000E0FFE709980168886920F0700088615D
:10691000FFE7FFE70998016804204860FFE708984F
:1069200048B1FFE7089A0999486A104348620998F4
:10693000FFF776FCFFE70AB080BD000080B584B0A9
:106940000290029820B9FFE701208DF80F00E0E0E7
:10695000029890F8200020B9FFE7029800F0DEF8D6
:10696000FFE702980168086840F00100086001F044
:10697000A1F90190FFE7029800684068C007A8B934
:10698000FFE701F097F90199401A0B280DD3FFE7B3
:106990000299486A40F4003048620299052081F863
:1069A000200001208DF80F00B3E0E4E702980168B1
:1069B000086820F00200086001F07CF90190FFE710
:1069C0000298006840688007002815D5FFE701F0AD
:1069D00071F90199401A0B280DD3FFE70299486A13
:1069E00040F4003048620299052081F8200001201F
:1069F0008DF80F008DE0E3E70298007E012807D1B3
:106A0000FFE702980168086840F08000086006E02F
:106A100002980168086820F080000860FFE702988B
:106A2000407E012807D1FFE702980168086840F01E
:106A30004000086006E002980168086820F0400005
:106A40000860FFE70298807E012807D1FFE70298DF
:106A50000168086840F02000086006E002980168BC
:106A6000086820F020000860FFE70298C07E012837
:106A700007D1FFE702980168086820F0100008605D
:106A800006E002980168086840F010000860FFE71F
:106A90000298007F012807D1FFE702980168086883
:106AA00040F00800086006E002980168086820F0DD
:106AB00008000860FFE70298407F012807D1FFE740
:106AC00002980168086840F00400086006E0029837
:106AD0000168086820F004000860FFE7029B19685D
:106AE0005A689868D3F80CC040EA0C00D3F810C07C
:106AF00040EA0C005B691843013A1043C8610299EF
:106B000000204862029A012182F820108DF80F00BF
:106B1000FFE79DF80F0004B080BD000080B596B07F
:106B200015900020149013901290119010901598C9
:106B3000006846F20041C4F2000188425CD1FFE7E0
:106B400040F25C50C2F2000001680131016000684F
:106B5000012812D1FFE7FFE700200F9043F6400025
:106B6000C4F20200016841F000710160006800F0A9
:106B700000700F900F98FFE7FFE7FFE700200E90EF
:106B800043F63000C4F20200016841F008010160E0
:106B9000006800F008000E900E98FFE703201090A8
:106BA0000221119100210991129113900920149052
:106BB00040F60040C4F2020010A900F06FFE099AEE
:106BC000132006900521089101F00CFB069801F0B6
:106BD000FFFA0899099A1420079001F003FB07981F
:106BE00001F0F6FA0899099A15200A9001F0FAFACC
:106BF0000A9801F0EDFA77E01598006846F6000172
:106C0000C4F2000188426ED1FFE7FFE700200D903B
:106C100043F64000C4F20200016841F08061016067
:106C2000006800F080600D900D98FFE740F25C5026
:106C3000C2F200000168013101600068012812D130
:106C4000FFE7FFE700200C9043F64000C4F202008B
:106C5000016841F000710160006800F000700C9064
:106C60000C98FFE7FFE7FFE700200B9043F63000AA
:106C7000C4F20200016841F002010160006800F006
:106C800002000B900B98FFE76020109002201190FB
:106C9000002004901290032013900920149040F2D9
:106CA0000040C4F2020010A900F0F8FD049A3F2051
:106CB00001900521039101F095FA019801F088FAFD
:106CC0000399049A4020029001F08CFA029801F096
:106CD0007FFA0399049A4120059001F083FA059800
:106CE00001F076FAFFE7FFE716B080BD80B582B00D
:106CF00001900198FCF740FC8DF803009DF803001B
:106D0000032819D0FFE79DF8030040F2B442C2F215
:106D10000002342110FB0120C06960B1FFE79DF83B
:106D2000030040F2B442C2F20002342110FB012001
:106D3000C0698047FFE7FFE702B080BD80B582B041
:106D400001900198FCF718FC8DF803009DF80300F2
:106D5000032819D0FFE79DF8030040F2B442C2F2C5
:106D60000002342110FB0120806960B1FFE79DF82B
:106D7000030040F2B442C2F20002342110FB0120B1
:106D800080698047FFE7FFE702B080BD80B582B031
:106D900001900198FCF7F0FB8DF803009DF80300CB
:106DA000032819D0FFE79DF8030040F2B442C2F275
:106DB0000002342110FB0120406A60B1FFE79DF81A
:106DC000030040F2B442C2F20002342110FB012061
:106DD000406A8047FFE7FFE702B080BD80B582B020
:106DE00001900198FCF7C8FB8DF803009DF80300A3
:106DF000032819D0FFE79DF8030040F2B442C2F225
:106E00000002342110FB0120006A60B1FFE79DF809
:106E1000030040F2B442C2F20002342110FB012010
:106E2000006A8047FFE7FFE702B080BD80B582B00F
:106E300001900198FCF7A0FB8DF803009DF803007A
:106E4000032819D0FFE79DF8030040F2B442C2F2D4
:106E50000002342110FB0120806A60B1FFE79DF839
:106E6000030040F2B442C2F20002342110FB0120C0
:106E7000806A8047FFE7FFE702B080BD80B584B03D
:106E80000290029890F8200001282FD1FFE7029984
:106E9000022081F8200002980168086820F00100B3
:106EA000086000F007FF0190FFE702980068406863
:106EB000C007A8B1FFE700F0FDFE0199401A0B28BA
:106EC0000DD3FFE70299486A40F400304862029906
:106ED000052081F8200001208DF80F000FE0E4E785
:106EE0000299002048628DF80F0008E00299486A74
:106EF00040F40020486201208DF80F00FFE79DF864
:106F00000F0004B080BD000080B582B001900198F0
:106F1000FCF732FB8DF803009DF80300032819D01D
:106F2000FFE79DF8030040F2B442C2F200023421B0
:106F300010FB0120C06860B1FFE79DF8030040F23C
:106F4000B442C2F20002342110FB0120C068804725
:106F5000FFE7FFE702B080BD80B582B001900198E5
:106F6000FCF70AFB8DF803009DF80300032817D0F7
:106F7000FFE79DF803003421414340F2B440C2F2E0
:106F80000000405858B1FFE79DF803003421414309
:106F900040F2B440C2F2000040588047FFE7FFE7EC
:106FA00002B080BD80B582B001900198FCF7E4FA90
:106FB0008DF803009DF80300032819D0FFE79DF822
:106FC000030040F2B442C2F20002342110FB01205F
:106FD000006960B1FFE79DF8030040F2B442C2F2DD
:106FE0000002342110FB012000698047FFE7FFE722
:106FF00002B080BD80B582B001900198FCF7BCFA68
:107000008DF803009DF80300032819D0FFE79DF8D1
:10701000030040F2B442C2F20002342110FB01200E
:10702000406860B1FFE79DF8030040F2B442C2F24D
:107030000002342110FB012040688047FFE7FFE792
:1070400002B080BD80B582B001900198FCF794FA3F
:107050008DF803009DF80300032819D0FFE79DF881
:10706000030040F2B442C2F20002342110FB0120BE
:10707000406960B1FFE79DF8030040F2B442C2F2FC
:107080000002342110FB012040698047FFE7FFE741
:1070900002B080BD80B582B001900198FCF76CFA17
:1070A0008DF803009DF80300032819D0FFE79DF831
:1070B000030040F2B442C2F20002342110FB01206E
:1070C000806860B1FFE79DF8030040F2B442C2F26D
:1070D0000002342110FB012080688047FFE7FFE7B2
:1070E00002B080BD80B582B001900198FCF744FAEF
:1070F0008DF803009DF80300032819D0FFE79DF8E1
:10710000030040F2B442C2F20002342110FB01201D
:10711000C06A60B1FFE79DF8030040F2B442C2F2DA
:107120000002342110FB0120C06A8047FFE7FFE71F
:1071300002B080BD80B584B002900298806D01904D
:1071400000F0B8FD0090029890F8350002280DD0AC
:10715000FFE7029980204865FFE70299002081F847
:107160003400FFE701208DF80F0055E00298016818
:10717000086820F01600086002980168486920F04D
:10718000800048610298006C20B9FFE70298806C8B
:1071900038B1FFE702980168086820F0080008602D
:1071A000FFE702980168086820F001000860FFE727
:1071B000029800680068C007C8B1FFE700F07AFDD8
:1071C0000099401A062811D3FFE70299202048654C
:1071D0000299032081F83500FFE70299002081F829
:1071E0003400FFE703208DF80F0015E0E0E7029878
:1071F000C16D3F208840019988600299012081F883
:107200003500FFE70299002081F83400FFE7FFE72F
:1072100000208DF80F00FFE79DF80F0004B080BD3F
:1072200082B00090009890F83500022807D0FFE760
:1072300000998020486501208DF807000EE0009934
:10724000052081F8350000980168086820F00100E9
:107250000860FFE700208DF80700FFE79DF80700B2
:1072600002B0704780B586B005900020039040F2D0
:107270000000C2F20000006848F2B511C1F64E31BC
:10728000A0FB0110800A02900598806D0190019882
:107290000068049004980599C96DC840000700284B
:1072A0001AD5FFE70598006800684007002812D546
:1072B000FFE705980168086820F004000860059859
:1072C000C16D08208840019988600599486D40F09B
:1072D00001004865FFE7FFE704980599C96DC840BC
:1072E000C007A0B1FFE705980068406900060028C4
:1072F0000CD5FFE70598C16D012088400199886091
:107300000599486D40F002004865FFE7FFE70498E3
:107310000599C96DC8404007002814D5FFE70598B6
:1073200000680068800700280CD5FFE70598C16D4C
:1073300004208840019988600599486D40F0040058
:107340004865FFE7FFE704980599C96DC840C00686
:10735000002847D5FFE70598006800680007002867
:107360003FD5FFE70598C16D1020884001998860DE
:10737000059800680068400300281AD5FFE70598C3
:10738000006800680003002809D4FFE70598006C36
:1073900020B1FFE70598016C8847FFE708E00598F2
:1073A000806C20B1FFE70598816C8847FFE7FFE715
:1073B00016E0059800680068C005002807D4FFE7BC
:1073C00005980168086820F008000860FFE7059844
:1073D000006C20B1FFE70598016C8847FFE7FFE7E5
:1073E000FFE7FFE704980599C96DC84080060028AB
:1073F00040F18D80FFE7059800680068C00600280E
:1074000040F18480FFE70598C16D202088400199F4
:107410008860059890F83500052834D1FFE7059875
:107420000168086820F0160008600598016848693E
:1074300020F0800048610598006C20B9FFE70598AE
:10744000806C38B1FFE705980168086820F00800F3
:107450000860FFE70598C16D3F208840019988606A
:107460000599012081F83500FFE70599002081F892
:107470003400FFE70598006D20B1FFE70598016D26
:107480008847FFE77BE00598006800684003002814
:107490001AD5FFE70598006800680003002809D4A2
:1074A000FFE70598406C20B1FFE70598416C8847DD
:1074B000FFE708E00598C06B20B1FFE70598C16BB6
:1074C0008847FFE7FFE720E0059800680068C005EF
:1074D000002811D4FFE705980168086820F0100023
:1074E00008600599012081F83500FFE70599002023
:1074F00081F83400FFE7FFE70598C06B20B1FFE794
:107500000598C16B8847FFE7FFE7FFE7FFE70598AE
:10751000406DA0B3FFE70598406DC00730B3FFE7AB
:107520000599052081F8350005980168086820F064
:1075300001000860FFE70398013003900299884238
:1075400001D9FFE707E0FFE7059800680068C0077A
:107550000028F0D1FFE70599012081F83500FFE709
:107560000599002081F83400FFE7FFE70598C06C1B
:1075700020B1FFE70598C16C8847FFE7FFE706B039
:1075800080BD000080B586B004900020039000F01C
:1075900091FB0290049820B9FFE701208DF81700B5
:1075A000A3E00498406A08B1FFE7FFE704990220CE
:1075B00081F83500FFE70499002081F83400FFE7E7
:1075C00004980168086820F001000860FFE704984B
:1075D00000680068C00790B1FFE700F06BFB0299FC
:1075E000401A06280AD3FFE7049920204865049929
:1075F000032081F835008DF8170076E0E7E704985E
:10760000006800680390039848F23F01CFF2100130
:1076100008400390049900914868D1F808C0CB68ED
:107620000A6940EA0C00184310434A6910438A690A
:107630001043CA691043096A014303980843039041
:107640000498406A042808D1FFE70499C86A096BC6
:107650000143039808430390FFE7039804990968DE
:1076600008600498006840690390039820F00700C0
:1076700003900498416A0398084303900498406A71
:1076800004281AD1FFE70498816A039808430390FD
:107690000498C06A80B1FFE70498FDF7DDFF50B1A0
:1076A000FFE70499402048650499012081F83500DE
:1076B0008DF8170019E0FFE7FFE7039804990968C0
:1076C00048610498FDF79CFF01900498C16D3F202C
:1076D000884001998860049900204865049A012136
:1076E00082F835108DF81700FFE79DF8170006B0F7
:1076F00080BD000080B588B0069005910492039388
:1077000000208DF80B000698806D0190FFE7069829
:1077100090F83400012804D1FFE702208DF81F0003
:1077200045E00699012081F83400FFE7FFE706985D
:1077300090F8350001282BD1FFE70699022081F847
:10774000350006990020486506980599049A039B20
:10775000FDF7FAFF0698C16D3F20884001998860C7
:1077600006980168086840F0160008600698006CEA
:1077700038B1FFE706980168086840F00800086023
:10778000FFE706980168086840F00100086009E01A
:10779000FFE70699002081F83400FFE702208DF80A
:1077A0000B00FFE79DF80B008DF81F00FFE79DF829
:1077B0001F0008B080BD000080B584B0039000F0C9
:1077C00079FA0290039801900198013048B1FFE7DF
:1077D00040F26430C2F20000017801980844019040
:1077E000FFE7FFE700F066FA0299401A0199884224
:1077F00001D2FFE7F6E704B080BD000080B582B09B
:10780000ADF8060000208DF80500FFE79DF80500A3
:107810000F2824DCFFE7BDF806009DF80510C840DE
:10782000C007A8B1FFE79DF8051040F21C50C2F256
:10783000000050F8210050B1FFE79DF8051040F21C
:107840001C50C2F2000050F821008047FFE7FFE71C
:10785000FFE79DF8050001308DF80500D6E702B07E
:1078600080BD000080B582B0ADF8060043F614403C
:10787000C4F201000068BDF8061008420CD0FFE712
:10788000BDF8060043F61441C4F201010860BDF8DA
:107890000600FFF7B3FFFFE702B080BD8EB00D908A
:1078A0000C9100200A90099008900B90FFE70B982C
:1078B0000F2800F2CC81FFE70B99012088400A9045
:1078C0000C9800680A990840099009980A9988421A
:1078D00040F0B881FFE70C98406800F003000128F1
:1078E00007D0FFE70C98406800F0030002282FD172
:1078F000FFE70D98806808900B984100032000FA7C
:1079000001F10898884308900C98C0680B994900C9
:1079100000FA01F108980843089008980D998860CA
:107920000D98406808900B99012000FA01F1089821
:10793000884308900C984068C0F300100B9900FA37
:1079400001F108980843089008980D994860FFE7EE
:107950000C98406800F00300032818D0FFE70D984A
:10796000C06808900B984100032000FA01F10898C4
:10797000884308900C9880680B99490000FA01F13F
:1079800008980843089008980D99C860FFE70C987C
:10799000406800F00300022826D1FFE70D980B99FC
:1079A0006FF0030202EA51010844006A08900B9844
:1079B00000F0070081000F2000FA01F108988843C9
:1079C00008900C9800690B9901F00701890000FAF2
:1079D00001F108980843089008980D990B9B02EA5A
:1079E000530211440862FFE70D98006808900B9855
:1079F0004100032000FA01F10898884308900C9890
:107A0000406800F003000B99490000FA01F1089862
:107A10000843089008980D9908600C9880798007B1
:107A2000002800F00E81FFE7FFE70020079043F6F3
:107A30004400C4F20200016841F480410160006822
:107A400000F4804007900798FFE70B9820F00300B0
:107A500043F60801C4F20101405808900B9800F069
:107A6000030081000F2000FA01F108988843089074
:107A70000D980021C4F20201884203D1FFE70020E3
:107A800006905EE00D9840F20041C4F20201884287
:107A900003D1FFE70120059050E00D9840F600016A
:107AA000C4F20201884203D1FFE70220049042E0C1
:107AB0000D9840F60041C4F20201884203D1FFE76D
:107AC0000320039034E00D9841F20001C4F202015A
:107AD000884203D1FFE70420029026E00D9841F28E
:107AE0000041C4F20201884203D1FFE70520019062
:107AF00018E00D9841F60001C4F20201884203D15A
:107B0000FFE7062000900AE00D9941F60042C4F21A
:107B100002020820914208BF07200090FFE700986A
:107B20000190FFE701980290FFE702980390FFE7BA
:107B300003980490FFE704980590FFE705980690E6
:107B4000FFE70698C0B20B9901F00301890000FA23
:107B500001F108980843089008980B9921F0030157
:107B600043F60802C4F20102885043F60840C4F20A
:107B700001000068089009990898884308900C98BB
:107B80008079C006002805D5FFE7099908980843C1
:107B90000890FFE7089843F60841C4F20101086025
:107BA00043F60C40C4F20100006808900999089857
:107BB000884308900C9880798006002805D5FFE757
:107BC0000999089808430890FFE7089843F60C4184
:107BD000C4F20101086043F60440C4F201000068E9
:107BE000089009990898884308900C988079800734
:107BF000002805D5FFE70999089808430890FFE792
:107C0000089843F60441C4F20101086043F60040BD
:107C1000C4F2010000680890099908988843089008
:107C20000C988079C00728B1FFE7099908980843A4
:107C30000890FFE7089843F60041C4F2010108608C
:107C4000FFE7FFE7FFE70B9801300B902FE60EB040
:107C50007047000082B00190ADF8021001980069F1
:107C6000BDF80210084204D0FFE701208DF80100A2
:107C700003E000208DF80100FFE79DF8010002B04D
:107C80007047000082B00190ADF802108DF801201D
:107C90009DF8010028B1FFE7BDF802000199886155
:107CA00005E0BDF80200000401998861FFE702B019
:107CB0007047000048F25060C2F200000068704750
:107CC00080B58EB00C900C9820B9FFE701208DF89C
:107CD000370043E10C9890F83D0040B9FFE70C995C
:107CE000002081F83C000C9800F03CF9FFE70C996B
:107CF000242081F83D000C980168086820F00100FC
:107D000008600C980168086840F4004008600C980E
:107D10000168086820F40040086000F0BDFB0A908C
:107D20000C98406848F2A061C0F2010188420BD86B
:107D3000FFE70A9948F28042C0F21E0200209142F9
:107D400038BF012009900AE00A9940F60012C0F2FB
:107D50003D020020914238BF01200990FFE70998B9
:107D6000012804D1FFE701208DF83700F6E00A98DA
:107D70004DF68361C4F21B31A0FB0110800C0B9007
:107D80000C980068406820F03F000B9908430C995C
:107D9000096848600C980068006A20F03F0008906D
:107DA0000C98406848F2A061C0F20101884204D8F2
:107DB000FFE70B98013007900EE00B984FF4967197
:107DC000484344F6D351C1F26201A0FB01010120F6
:107DD00000EB91100790FFE70898079908430C996A
:107DE000096808620C980068C0694CF6FF71884306
:107DF00006900C98406848F2A061C0F201018842E8
:107E00001FD8FFE70A9801380C9949684900B0FB70
:107E1000F1F001306FF31F30032803D8FFE704208F
:107E200005900BE00A9801380C9949684900B0FBAD
:107E3000F1F001306FF31F300590FFE705980490D3
:107E40004CE00C98806868B9FFE70A9801380C99F3
:107E5000496801EB4101B0FBF1F001306FF31F30D5
:107E600003900DE00A9801380C9949681922514392
:107E7000B0FBF1F00130042161F31F300390FFE704
:107E80000398000518B9FFE70120029023E00C9841
:107E9000806868B9FFE70A9801380C99496801EBD6
:107EA0004101B0FBF1F001306FF31F3001900DE0A4
:107EB0000A9801380C99496819225143B0FBF1F036
:107EC0000130042161F31F300190FFE7019840F475
:107ED00000400290FFE702980490FFE7069804999B
:107EE00008430C990968C8610C980068006820F084
:107EF000C0000C9B1968DA691B6A1A4310430860BA
:107F00000C980068806848F2FF3188430C9A116829
:107F1000D36812691A43104388600C980068C068DF
:107F200020F0FF000C9B19685A699B691A431043A3
:107F3000C8600C980168086840F0010008600C995E
:107F4000002008640C9A202182F83D100C990863E7
:107F50000C9981F83E008DF83700FFE79DF8370057
:107F60000EB080BD80B590B00F9000200E900D90A7
:107F70000C900B900A900F98006845F60041C4F2EF
:107F80000001884240F08980FFE7FFE70020099068
:107F900043F63000C4F20200016841F004010160C0
:107FA000006800F0040009900998FFE7FFE700204F
:107FB000089043F63000C4F20200016841F001016C
:107FC0000160006800F0010008900898FFE74FF496
:107FD00000700A90122002900B90002003900C90E9
:107FE000032004900D90042005900E9040F60000B0
:107FF000C4F202000AA90691FFF750FCDDF808C0A0
:10800000039B049A059806994FF4807ECDF828E0EA
:10801000CDF82CC00C930D920E900020C4F20200FB
:10802000FFF73CFCFFE70020079043F64000C4F256
:108030000200016841F400010160006800F40000E2
:1080400007900798FFE740F68C40C2F200000190CD
:1080500046F24001C4F2020101604FF0C06141608C
:1080600000218160C1604FF48062026141618161E1
:10807000C16101624162FFF785FA18B1FFE7FDF7C0
:10808000A5FBFFE7FFE70F9840F68C41C2F2000125
:1080900081630F988863FFE7FFE710B080BD0000A1
:1080A00040F26430C2F20000027848F25061C2F23D
:1080B00000010868104408607047000080B543F66E
:1080C0000041C4F20201086840F4007008600868CA
:1080D00040F480600860086840F480700860032005
:1080E00000F09AF80F2000F005F800F03BF80020AF
:1080F00080BD000080B582B0009040F20000C2F266
:108100000000006840F26431C2F200010A784FF4C6
:108110007A71B1FBF2F1B0FBF1F001F0F3FE20B1A6
:10812000FFE701208DF8070018E000980F280DD810
:10813000FFE700994FF0FF30002200F053F800985D
:1081400040F26831C2F20001086003E001208DF8BE
:10815000070003E000208DF80700FFE79DF8070007
:1081600002B080BD80B582B0FFE70020019043F6E9
:108170004400C4F20200016841F4804101600068DB
:1081800000F4804001900198FFE7FFE70020009095
:1081900043F64000C4F20200016841F080510160E2
:1081A000006800F0805000900098FFE76FF0010039
:1081B0000F21002200F016F802B080BD80B582B019
:1081C0008DF807009DF9070008F000F902B080BDA6
:1081D00080B582B08DF807009DF9070008F012F90C
:1081E00002B080BD80B586B08DF81700049103926F
:1081F0000020029008F01EF902909DF917000190EE
:1082000002980499039A04F059FE0146019808F077
:1082100019F906B080BD000080B582B001900198C8
:1082200008F054F902B080BD80B584B0029001918D
:10823000029820B9FFE701208DF80F0021E1019895
:1082400043F60041C4F20201096801F007018842C7
:1082500012D9FFE7019943F60040C4F20200017011
:10826000006800F007000199884204D0FFE7012070
:108270008DF80F0005E1FFE70298007880070028DD
:108280002AD5FFE7029800784007002809D5FFE7C4
:1082900043F60801C4F20201086840F4E0500860A7
:1082A000FFE7029800780007002809D5FFE743F6AA
:1082B0000801C4F20201086840F460400860FFE76A
:1082C00043F60801C4F20201086820F0F000029AA7
:1082D000926810430860FFE702980078C007002802
:1082E0006ED0FFE702984068012811D1FFE743F6FE
:1082F0000000C4F20200006800F400310020B0EB7E
:10830000514F04D1FFE701208DF80F00B9E02CE0B8
:1083100002984068022805D0FFE7029840680328C9
:1083200011D1FFE743F60000C4F20200006800F03C
:1083300000710020B0EB516F04D1FFE701208DF8F0
:108340000F009EE010E043F60000C4F20200006857
:1083500000F002010020B0EB510F04D1FFE7012033
:108360008DF80F008DE0FFE7FFE743F60801C4F248
:108370000201086820F00300029A52681043086066
:10838000FFF798FC0090FFE743F60800C4F20200F4
:10839000006800F00C0002994968B0EB810F0ED024
:1083A000FFE7FFF787FC0099401A41F289318842C4
:1083B00004D3FFE703208DF80F0062E0E4E7FFE756
:1083C000019843F60041C4F20201096801F0070177
:1083D000884212D2FFE7019943F60040C4F202003E
:1083E0000170006800F007000199884204D0FFE79F
:1083F00001208DF80F0044E0FFE702980078400765
:1084000000280CD5FFE743F60801C4F20201086812
:1084100020F4E050029AD26810430860FFE7029807
:108420000078000700280DD5FFE743F60801C4F2E5
:108430000201086820F46040029A126940EAC20012
:108440000860FFE700F04CF843F60801C4F20201AF
:108450000968C9B20A0946F64001C0F60101895C03
:10846000C84040F20001C2F20001086040F26830EA
:10847000C2F200000068FFF73DFE00208DF80F00FB
:10848000FFE79DF80F0004B080BD000040F200003F
:10849000C2F200000068704780B5FFF7F7FF43F6AF
:1084A0000801C4F202010968C1F3822246F65001B4
:1084B000C0F60101895CC84080BD000080B5FFF7AF
:1084C000E5FF43F60801C4F20201096889B24A0BCC
:1084D00046F65001C0F60101895CC84080BD00002D
:1084E00080B586B00020059004900390029043F67A
:1084F0000800C4F20200006800F00C00014601917F
:1085000040B1FFE7019804280AD0FFE70198082846
:108510000CD04FE042F20040C0F2F40002904FE075
:1085200041F60030C0F2B700029049E043F6040083
:10853000C4F20200016801F03F01059100684002A9
:10854000002813D5FFE743F60400C4F202000068D8
:10855000C0F3881041F60031C0F2B701A0FB010161
:10856000059A0023F7F7BCFE049012E043F60400DE
:10857000C4F202000068C0F3881042F20041C0F269
:10858000F401A0FB0101059A0023F7F7A9FE04906E
:10859000FFE743F60400C4F20200006800F4403133
:1085A000022000EBD130039004980399B0FBF1F066
:1085B000029005E042F20040C0F2F4000290FFE7B2
:1085C000029806B080BD000080B586B00490049883
:1085D00020B9FFE701208DF8170050E304980078D8
:1085E000C007002800F0A580FFE743F60800C4F2AA
:1085F0000200006800F00C00042813D0FFE743F6E7
:108600000800C4F20200006800F00C0008281ED127
:10861000FFE743F60400C4F20200006840020028AD
:1086200015D5FFE743F60000C4F20200006800F42D
:1086300000310020B0EB514F08D0FFE704984068AC
:1086400020B9FFE701208DF8170018E370E0FFE77D
:1086500004984068B0F5803F09D1FFE743F6000178
:10866000C4F20201086840F48030086020E00498F9
:108670004068B0F5A02F0DD1FFE743F60001C4F22A
:108680000201086840F480200860086840F48030E7
:1086900008600CE043F60001C4F20201086820F40F
:1086A00080300860086820F480200860FFE7FFE75A
:1086B000FFE704984068E8B1FFE7FFF7FBFA039093
:1086C000FFE743F60000C4F20200006800F4003146
:1086D0000020B0EB514F0CD1FFE7FFF7EBFA039905
:1086E000401A652804D3FFE703208DF81700C6E27F
:1086F000E7E71CE0FFF7DEFA0390FFE743F6000030
:10870000C4F20200006800F400310020B0EB514FC9
:108710000CD0FFE7FFF7CEFA0399401A652804D37F
:10872000FFE703208DF81700A9E2E7E7FFE7FFE77F
:10873000FFE7049800788007002840F19680FFE763
:1087400043F60800C4F20200006810F00C0F13D0CA
:10875000FFE743F60800C4F20200006800F00C00D6
:1087600008282CD1FFE743F60400C4F20200006899
:108770004002002823D4FFE743F60000C4F20200C1
:10878000006800F002010020B0EB510F09D0FFE7B4
:108790000498C068012804D0FFE701208DF8170075
:1087A0006DE243F60001C4F20201086820F0F8000F
:1087B000049A126940EAC2000860FFE754E0049896
:1087C000C06870B3FFE70021C4F2472101200860B0
:1087D000FFF770FA0390FFE743F60000C4F20200CF
:1087E000006800F002010020B0EB510F0CD1FFE750
:1087F000FFF760FA0399401A032804D3FFE7032028
:108800008DF817003BE2E7E743F60001C4F20201EE
:10881000086820F0F800049A126940EAC200086073
:1088200021E00021C4F2472100200860FFF742FA4E
:108830000390FFE743F60000C4F20200006800F076
:1088400002010020B0EB510F0CD0FFE7FFF732FA26
:108850000399401A032804D3FFE703208DF817007B
:108860000DE2E7E7FFE7FFE7FFE70498007800077E
:1088700000284BD5FFE70498406918B3FFE740F69E
:108880008061C4F2472101200860FFF713FA0390CA
:10889000FFE743F67400C4F20200006800F0020132
:1088A0000020B0EB510F0CD1FFE7FFF703FA03995B
:1088B000401A032804D3FFE703208DF81700DEE1F8
:1088C000E7E722E040F68061C4F24721002008601B
:1088D000FFF7F0F90390FFE743F67400C4F20200DB
:1088E000006800F002010020B0EB510F0CD0FFE750
:1088F000FFF7E0F90399401A032804D3FFE70320A8
:108900008DF81700BBE1E7E7FFE7FFE70498007881
:108910004007002840F1CE80FFE700208DF80700D7
:1089200043F64000C4F202000068C000002815D4DD
:10893000FFE7FFE70020009043F64000C4F202008A
:10894000016841F080510160006800F080500090A3
:108950000098FFE701208DF80700FFE747F20000CD
:10896000C4F200000068C005002822D4FFE747F2E7
:108970000001C4F20001086840F480700860FFF74D
:1089800099F90390FFE747F20000C4F20000006885
:10899000C00500280CD4FFE7FFF78CF90399401AB3
:1089A000032804D3FFE703208DF8170067E1EAE707
:1089B000FFE7FFE704988068012809D1FFE743F645
:1089C0007001C4F20201086840F0010008601FE075
:1089D0000498806805280DD1FFE743F67001C4F2C2
:1089E0000201086840F004000860086840F00100D7
:1089F00008600CE043F67001C4F20201086820F040
:108A000001000860086820F004000860FFE7FFE745
:108A1000FFE704988068F8B1FFE7FFF74BF9039090
:108A2000FFE743F67000C4F20200006800F00201A4
:108A30000020B0EB510F0ED1FFE7FFF73BF9039990
:108A4000401A41F28931884204D3FFE703208DF8B0
:108A5000170014E1E5E71EE0FFF72CF90390FFE7AC
:108A600043F67000C4F20200006800F0020100202A
:108A7000B0EB510F0ED0FFE7FFF71CF90399401A36
:108A800041F28931884204D3FFE703208DF81700B3
:108A9000F5E0E5E7FFE79DF80700012809D1FFE7CA
:108AA00043F64001C4F20201086820F080500860DB
:108AB000FFE7FFE704988069002800F0DC80FFE70B
:108AC00043F60800C4F20200006800F00C00082819
:108AD00000F08580FFE70498806902285CD1FFE7F9
:108AE0006021C4F2472100200860FFF7E3F80390FB
:108AF000FFE743F60000C4F20200006800F00071D6
:108B00000020B0EB516F0CD0FFE7FFF7D3F80399CB
:108B1000401A032804D3FFE703208DF81700AEE0C6
:108B2000E7E70499C869D1F820C04B6A8A6A40EA2D
:108B30000C0040EA8310D2034FF6FF739A43A2F56C
:108B400080321043C96A40EA016043F60401C4F26E
:108B5000020108606021C4F2472101200860FFF78C
:108B6000A9F80390FFE743F60000C4F20200006892
:108B700000F000710020B0EB516F0CD1FFE7FFF760
:108B800099F80399401A032804D3FFE703208DF8CE
:108B9000170074E0E7E721E06021C4F247210020DC
:108BA0000860FFF787F80390FFE743F60000C4F280
:108BB0000200006800F000710020B0EB516F0CD093
:108BC000FFE7FFF777F80399401A032804D3FFE77C
:108BD00003208DF8170052E0E7E7FFE74AE004982A
:108BE0008069012804D1FFE701208DF8170046E0D5
:108BF00043F60400C4F20200006802900498806901
:108C0000012831D0FFE7029800F480000499C96977
:108C1000884229D1FFE7029800F03F000499096AD1
:108C2000884221D1FFE7029847F6C07108400499B5
:108C3000496AB0EB811F17D1FFE7029800F440307A
:108C40000499896AC9034FF6FF729143A1F58031F7
:108C5000884209D1FFE7029800F070600499C96A60
:108C6000B0EB016F04D0FFE701208DF8170006E09C
:108C7000FFE7FFE7FFE700208DF81700FFE79DF80B
:108C8000170006B080BD000080B582B00190019849
:108C900004F0F8FD8DF803009DF8030002281BD0B6
:108CA000FFE7019804F0EEFD014640F26450C2F285
:108CB000000000EB4110806968B1FFE7019804F003
:108CC000E1FD014640F26450C2F2000000EB4110A9
:108CD00080698047FFE7FFE702B080BD80B584B0C0
:108CE0000290029820B9FFE701208DF80F0071E093
:108CF0000298406A60B9FFE702984068B0F5827F49
:108D000001D1FFE703E002990020C861FFE705E019
:108D100002990020086102994861FFE7029900204A
:108D20008862029890F8510040B9FFE7029900204C
:108D300081F85000029800F051F8FFE702990220F4
:108D400081F8510002980168086820F0400008602E
:108D5000029A019211685068D2F808C0D36800F4F2
:108D600082700CF4044C604403F4006318441369EB
:108D700003F002031844536903F001031844936994
:108D800003F400731844D36903F038031844136ADA
:108D900003F080031843926A02F400521043086003
:108DA000029A508B00F004001168526A02F010021F
:108DB0001044486002980168C86920F40060C861E6
:108DC000029900204865029A012182F851108DF81D
:108DD0000F00FFE79DF80F0004B080BD80B590B094
:108DE0000F9000200E900D900C900B900A900F9811
:108DF000006843F20001C4F20101884240F0B280F1
:108E0000FFE7FFE70020099043F64400C4F20200A8
:108E1000016841F480510160006800F480500990BD
:108E20000998FFE7FFE70020089043F63000C4F2FE
:108E30000200016841F002010160006800F00200D8
:108E400008900898FFE7FFE70020079043F63000FE
:108E5000C4F20200016841F001010160006800F005
:108E6000010007900798FFE718200A900220019060
:108E70000B90002005900C90032002900D9005208F
:108E800003900E9040F20040C4F202000AA904913F
:108E9000FEF704FDDDF804C0029A03980499059BCF
:108EA0004FF0800ECDF828E0CDF82CC00C930D9239
:108EB0000E900020C4F20200FEF7F0FC059940F687
:108EC000EC40C2F20000069046F24042C4F20202B8
:108ED00002604FF0C06242608160C1604FF4806206
:108EE000026141618161C16101624162FEF74AFB39
:108EF00018B1FFE7FCF76AFCFFE7FFE70F9840F6C1
:108F0000EC41C2F20001C1640F988863FFE740F6AC
:108F10004C50C2F20000009046F25841C4F20201E7
:108F200001604FF0C0614160402181600021C1605B
:108F30004FF48062026141618161C16101624162FD
:108F4000FEF720FB18B1FFE7FCF740FCFFE7FFE767
:108F50000F9840F64C51C2F2000181640F9888636B
:108F6000FFE7FFE710B080BD80B588B0069005919F
:108F7000ADF812200393069890F85100012804D010
:108F8000FFE702208DF81F0011E1059820B1FFE7EF
:108F9000BDF8120020B9FFE701208DF81F0006E19F
:108FA00006984068B0F5827F16D1FFE70698806882
:108FB00090B9FFE70699042081F851000698059AB8
:108FC000BDF812300399EC46CCF80010114600F0C1
:108FD00065FB8DF81F00EAE0FEF76CFE0290FFE7EC
:108FE000069890F85000012804D1FFE702208DF880
:108FF0001F00DCE00699012081F85000FFE7FFE741
:109000000699042081F851000699002048650599C9
:10901000069A9163BDF81210069A9187BDF8121056
:10902000069AD18706990863069988860699C886A4
:10903000069908640699486406988068B0F5004F60
:109040000DD1FFE706980168086820F0400008602D
:1090500006980168086820F480400860FFE70698D9
:109060000068006800F04000402807D0FFE706983D
:109070000168086840F040000860FFE70698C06893
:10908000D0BBFFE7FFE70698C08FA0B3FFE70698C5
:1090900000688068C00778B1FFE706980068007B29
:1090A0000699896B08700699886B01308863069968
:1090B000C88F0138C8871DE0FEF7FCFD0299401AF1
:1090C0000399884204D3FFE70398013018B9FFE7FA
:1090D000039870B9FFE70699012081F85100FFE776
:1090E0000699002081F85000FFE703208DF81F004B
:1090F0005DE0FFE7C7E739E0FFE70698C08FA0B360
:10910000FFE7069800688068C00778B1FFE7069817
:109110000068C0680699896B08800699886B0230E0
:1091200088630699C88F0138C8871DE0FEF7C2FD25
:109130000299401A0399884204D3FFE7039801304B
:1091400018B9FFE7039870B9FFE70699012081F885
:109150005100FFE70699002081F85000FFE7032047
:109160008DF81F0023E0FFE7C7E7FFE706980399A4
:10917000029A04F0AFFA20B1FFE706992020486573
:10918000FFE70699012081F85100FFE706990020CA
:1091900081F85000FFE70698406D20B1FFE70120FD
:1091A0008DF81F0003E000208DF81F00FFE79DF8F9
:1091B0001F0008B080BD000080B584B0029001910E
:1091C000ADF80220029890F85100012804D0FFE782
:1091D00002208DF80F00B7E0019820B1FFE7BDF83D
:1091E000020020B9FFE701208DF80F00ACE00298E3
:1091F0008068A0B9FFE702984068B0F5827F0ED181
:10920000FFE70299042081F851000298019ABDF805
:109210000230114600F014FC8DF80F0094E0FFE7D7
:10922000029890F85000012804D1FFE702208DF841
:109230000F0089E00299012081F85000FFE7FFE765
:109240000299042081F85100029900204865019993
:10925000029A9163BDF80210029A9187BDF802103C
:10926000029AD18702990864029948640299888613
:109270000299C88602988068B0F5004F0DD1FFE7CB
:1092800002980168086820F04000086002980168B0
:10929000086820F480400860FFE70298C16C4DF236
:1092A000B940C0F6000008640298C16C4DF201504C
:1092B000C0F60000C8630298C16C4DF28540C0F64C
:1092C0000000C8640298C16C00200865029B196800
:1092D0009A6BD86C0C31DB8FFEF70CFA78B1FFE794
:1092E0000299486D40F010004865FFE702990020A0
:1092F00081F85000FFE701208DF80F0024E002986C
:109300000068006800F04000402807D0FFE702989E
:109310000168086840F040000860FFE7FFE7029935
:10932000002081F85000FFE702980168486840F08B
:109330002000486002980168486840F001004860D9
:1093400000208DF80F00FFE79DF80F0004B080BDEE
:1093500080B582B00190019804F094FA8DF8030072
:109360009DF8030002281BD0FFE7019804F08AFA59
:10937000014640F26450C2F2000000EB4110406828
:1093800068B1FFE7019804F07DFA014640F26450AD
:10939000C2F2000000EB411040688047FFE7FFE7A2
:1093A00002B080BD80B582B00190019804F06AFAE5
:1093B0008DF803009DF8030002281BD0FFE70198F9
:1093C00004F060FA014640F26450C2F2000000EB83
:1093D0004110006968B1FFE7019804F053FA0146B3
:1093E00040F26450C2F2000000EB41100069804777
:1093F000FFE7FFE702B080BD80B588B00690059119
:10940000ADF812200393FEF755FC0290BDF8120050
:10941000ADF80600069890F85100012804D0FFE747
:1094200002208DF81F0034E1059820B1FFE7BDF858
:10943000120020B9FFE701208DF81F0029E1FFE7A6
:10944000069890F85000012804D1FFE702208DF81B
:109450001F001EE10699012081F85000FFE7FFE799
:109460000699032081F85100069900204865059966
:10947000069A1163BDF81210069A9186BDF8121073
:10948000069AD18606998863069988870699C887BF
:10949000069948640699086406988068B0F5004FFC
:1094A0000DD1FFE706980168086820F040000860C9
:1094B00006980168086840F480400860FFE7069855
:1094C0000068006800F04000402807D0FFE70698D9
:1094D0000168086840F040000860FFE70698C0682F
:1094E000B0F5006F51D1FFE70698406828B1FFE75B
:1094F000BDF8060001280ED1FFE706980168006B51
:109500000088C8600699086B023008630699C88E07
:109510000138C886FFE7FFE70698C08EA0B3FFE7D3
:10952000069800688068800700280ED5FFE7069837
:109530000168006B0088C8600699086B02300863F8
:109540000699C88E0138C8861DE0FEF7B3FB029964
:10955000401A0399884204D3FFE70398013018B9F1
:10956000FFE7039870B9FFE70699012081F85100E1
:10957000FFE70699002081F85000FFE703208DF8EF
:109580001F0086E0FFE7C7E750E00698406828B173
:10959000FFE7BDF8060001280ED1FFE70698016835
:1095A000006B007808730699086B01300863069910
:1095B000C88E0138C886FFE7FFE70698C08EA0B3C3
:1095C000FFE7069800688068800700280ED5FFE74F
:1095D00006980168006B007808730699086B0130E3
:1095E00008630699C88E0138C8861DE0FEF762FB45
:1095F0000299401A0399884204D3FFE70398013087
:1096000018B9FFE7039870B9FFE70699012081F8C0
:109610005100FFE70699002081F85000FFE7032082
:109620008DF81F0035E0FFE7C7E7FFE706980399CD
:10963000029A04F0C1F820B1FFE70699202048659E
:10964000FFE70698806870B9FFE7FFE70020009009
:1096500006980068C06800900698006880680090CE
:109660000098FFE7FFE70699012081F85100FFE726
:109670000699002081F85000FFE70698406D20B160
:10968000FFE701208DF81F0003E000208DF81F0088
:10969000FFE79DF81F0008B080BD000080B58CB0CA
:1096A000DDF838C00A9009910892ADF81E3001200B
:1096B0000390FEF7FFFA04900A9890F851008DF895
:1096C00017000A9840680690BDF81E00ADF81C000F
:1096D0009DF81700012812D0FFE70698B0F5827FA9
:1096E00009D1FFE70A98806828B9FFE79DF81700BD
:1096F000042804D0FFE702208DF82F009BE1099891
:1097000038B1FFE7089820B1FFE7BDF81E0020B987
:10971000FFE701208DF82F008DE1FFE70A9890F810
:109720005000012804D1FFE702208DF82F0082E1CC
:109730000A99012081F85000FFE7FFE70A9890F8A6
:109740005100042805D0FFE70A99052081F851004F
:10975000FFE70A990020486508990A9A9163BDF8C5
:109760001E100A9AD187BDF81E100A9A918709998E
:109770000A9A1163BDF81E100A9AD186BDF81E1010
:109780000A9A91860A9908640A9948640A980068B6
:10979000006800F04000402807D0FFE70A98016801
:1097A000086840F040000860FFE70A98C068B0F51C
:1097B000006F40F08180FFE70A98406828B1FFE71A
:1097C000BDF81C0001280ED1FFE70A980168006B64
:1097D0000088C8600A99086B023008630A99C88E2D
:1097E0000138C886FFE7FFE70A98C18E0120019083
:1097F00039B9FFE70A98C08F002818BF01200190EF
:10980000FFE70198C007002855D0FFE70A980068D5
:1098100080688007002818D5FFE70A98C08EA0B19D
:10982000FFE70398012810D1FFE70A980168006B51
:109830000088C8600A99086B023008630A99C88ECC
:109840000138C88600200390FFE70A980068806806
:10985000C007A8B1FFE70A98C08F88B1FFE70A9850
:109860000068C0680A99896B08800A99886B023081
:1098700088630A99C88F0138C88701200390FFE7E1
:10988000FEF718FA0499401A0E99884212D3FFE79E
:109890000E98013070B1FFE70A99012081F851005C
:1098A000FFE70A99002081F85000FFE703208DF8B8
:1098B0002F00C0E098E782E00A98406828B1FFE7EF
:1098C000BDF81C0001280ED1FFE70A980168006B63
:1098D000007808730A99086B013008630A99C88EEA
:1098E0000138C886FFE7FFE70A98C18E0120009083
:1098F00039B9FFE70A98C08F002818BF01200090EF
:10990000FFE70098C007002858D0FFE70A980068D2
:1099100080688007002818D5FFE70A98C08EA0B19C
:10992000FFE70398012810D1FFE70A980168006B50
:10993000007808730A99086B013008630A99C88E89
:109940000138C88600200390FFE70A980068806805
:10995000C007A8B1FFE70A98C08F88B1FFE70A984F
:109960000068C0680A99896B08700A99886B013091
:1099700088630A99C88F0138C88701200390FFE7E0
:10998000FEF798F90499401A0E99884204D3FFE72C
:109990000E98013018B9FFE70E9870B9FFE70A99E1
:1099A000012081F85100FFE70A99002081F850005A
:1099B000FFE703208DF82F003DE095E7FFE70A98C9
:1099C0000E99049A03F0F8FE68B1FFE70A99202087
:1099D0004865FFE70A99002081F85000FFE7012061
:1099E0008DF82F0027E00A98806870B9FFE7FFE73D
:1099F000002002900A980068C06802900A980068E7
:109A0000806802900298FFE7FFE70A99012081F839
:109A10005100FFE70A99002081F85000FFE70A98FB
:109A2000406D20B1FFE701208DF82F0003E00020FA
:109A30008DF82F00FFE79DF82F000CB080BD0000CF
:109A400080B588B0069005910492ADF80E30069866
:109A500090F851008DF807000698406802909DF834
:109A60000700012812D0FFE70298B0F5827F09D1E4
:109A7000FFE70698806828B9FFE79DF807000428EB
:109A800004D0FFE702208DF81F00DFE0059838B111
:109A9000FFE7049820B1FFE7BDF80E0020B9FFE70B
:109AA00001208DF81F00D1E0FFE7069890F85000E4
:109AB000012804D1FFE702208DF81F00C6E00699B7
:109AC000012081F85000FFE7FFE7069890F8510069
:109AD000042805D0FFE70699052081F85100FFE72B
:109AE0000699002048650599069A1163BDF80E1085
:109AF000069A9186BDF80E10069AD1860499069AA8
:109B00009163BDF80E10069A9187BDF80E10069A63
:109B1000D1870699086406994864069890F8510020
:109B200004280FD1FFE70698C16C4DF2B940C0F68A
:109B3000000008640698C16C4DF20150C0F60000A8
:109B4000C8630EE00698C16C4DF2E940C0F6000013
:109B500008640698C16C4DF24D60C0F60000C86301
:109B6000FFE70698C16C4DF28540C0F60000C8645E
:109B70000698C16C00200865069B19689A6BD86C22
:109B80000C31DB8FFDF7B6FD78B1FFE70699486D24
:109B900040F010004865FFE70699002081F850006A
:109BA000FFE701208DF81F0050E006980168486823
:109BB00040F0010048600698816C00200864069916
:109BC000896CC8630699896CC8640699896C0865B4
:109BD000069B1A68196B986C0C32DB8EFDF78AFDB8
:109BE00078B1FFE70699486D40F010004865FFE73F
:109BF0000699002081F85000FFE701208DF81F0032
:109C000024E006980068006800F04000402807D073
:109C1000FFE706980168086840F040000860FFE729
:109C2000FFE70699002081F85000FFE706980168D9
:109C3000486840F02000486006980168486840F095
:109C40000200486000208DF81F00FFE79DF81F000C
:109C500008B080BD80B584B002900191ADF80220BB
:109C6000029890F85100012804D0FFE702208DF8F7
:109C70000F00A1E0019820B1FFE7BDF8020020B974
:109C8000FFE701208DF80F0096E0FFE7029890F8BB
:109C90005000012804D1FFE702208DF80F008BE06F
:109CA0000299012081F85000FFE7FFE702990320A5
:109CB00081F851000299002048650199029A1163C8
:109CC000BDF80210029A9186BDF80210029AD18660
:109CD0000299886302994864029908640299888706
:109CE0000299C88702988068B0F5004F0DD1FFE750
:109CF00002980168086820F0400008600298016836
:109D0000086840F480400860FFE70298816C4DF2DB
:109D1000D140C0F6000008640298816C4DF2A55055
:109D2000C0F60000C8630298816C4DF28540C0F611
:109D30000000C8640298816C00200865029B1A68C4
:109D4000196B986C0C32DB8EFDF7D4FC78B1FFE711
:109D50000299486D40F010004865FFE70299002025
:109D600081F85000FFE701208DF80F0024E00298F1
:109D70000068006800F04000402807D0FFE7029824
:109D80000168086840F040000860FFE7FFE70299BB
:109D9000002081F85000FFE702980168486840F011
:109DA0002000486002980168486840F0020048605E
:109DB00000208DF80F00FFE79DF80F0004B080BD74
:109DC00080B582B00190019803F05CFD8DF803002E
:109DD0009DF80300022815D0FFE79DF8030041011C
:109DE00040F26450C2F20000405850B1FFE79DF8C5
:109DF0000300410140F26450C2F200004058804725
:109E0000FFE7FFE702B080BD80B582B00190019806
:109E100003F038FD8DF803009DF8030002281BD0E5
:109E2000FFE7019803F02EFD014640F26450C2F2B4
:109E3000000000EB4110C06868B1FFE7019803F033
:109E400021FD014640F26450C2F2000000EB4110D7
:109E5000C0688047FFE7FFE702B080BD80B582B0F1
:109E60000190019803F00EFD8DF803009DF80300AA
:109E700002281BD0FFE7019803F004FD014640F2E1
:109E80006450C2F2000000EB4110806868B1FFE747
:109E9000019803F0F7FC014640F26450C2F2000062
:109EA00000EB411080688047FFE7FFE702B080BD0C
:109EB00080B582B00190019803F0E4FC8DF80300B6
:109EC0009DF8030002281BD0FFE7019803F0DAFC9D
:109ED000014640F26450C2F2000000EB41104069BC
:109EE00068B1FFE7019803F0CDFC014640F26450F1
:109EF000C2F2000000EB411040698047FFE7FFE736
:109F000002B080BD80B582B00190019804F0D6FD0A
:109F100002B080BD85B003900291FFE7039890F8EE
:109F20003C00012804D1FFE702208DF813007EE0F9
:109F30000399012081F83C00FFE7FFE70399022025
:109F400081F83D000398006840680190039800681C
:109F500080680090019820F07000019002980168DC
:109F60000198084301900198039909684860039893
:109F700000680021C4F2010188423CD0FFE7039849
:109F80000068B0F1804F36D0FFE70398006840F2D8
:109F90000041C4F2000188422DD0FFE70398006819
:109FA00040F60001C4F20001884224D0FFE7039884
:109FB000006840F60041C4F2000188421BD0FFE770
:109FC0000398006840F20041C4F20101884212D0B7
:109FD000FFE70398006844F20001C4F201018842DF
:109FE00009D0FFE70398006841F60001C4F20001C0
:109FF00088420ED1FFE7009820F080000090029880
:10A0000041680098084300900098039909688860A7
:10A01000FFE70399012081F83D00FFE70399002045
:10A0200081F83C00FFE700208DF81300FFE79DF862
:10A03000130005B07047000080B582B00090009812
:10A0400020B9FFE701208DF807003FE0009890F865
:10A050003D0040B9FFE70099002081F83C000098DE
:10A0600000F038F8FFE70099022081F83D000099E0
:10A0700051F8040B04F0C0FD0099012081F846005E
:10A08000FFE70099012081F83E00009981F83F0028
:10A09000009981F84000009981F84100FFE7FFE74F
:10A0A0000099012081F84200009981F8430000994D
:10A0B00081F84400009981F84500FFE700990120EC
:10A0C00081F83D0000208DF80700FFE79DF80700AC
:10A0D00002B080BD83B002900298006840F6004153
:10A0E000C4F20001884212D1FFE7FFE7002001908F
:10A0F00043F64000C4F20200016841F0080101602B
:10A10000006800F0080001900198FFE71BE002984A
:10A11000006844F20041C4F20101884212D1FFE715
:10A12000FFE70020009043F64400C4F202000168FB
:10A1300041F400310160006800F4003000900098A4
:10A14000FFE7FFE7FFE703B07047000080B586B088
:10A150000490039100208DF80B00FFE7049890F81D
:10A160003C00012804D1FFE702208DF81700ABE086
:10A170000499012081F83C00FFE7FFE704990220E1
:10A1800081F83D000498006880680190019820F0F3
:10A1900077000190019820F47F4001900198049984
:10A1A00009688860039800680090002872D0FFE773
:10A1B000009810286ED0FFE7009820286AD0FFE7AB
:10A1C0000098302866D0FFE70098402855D0FFE778
:10A1D0000098502837D0FFE70098602840D0FFE76C
:10A1E000009870280BD0FFE70098B0F5805F05D08D
:10A1F000FFE70098B0F5005F16D052E055E00498F4
:10A200000068039B5A689968DB6804F0E3FD0498D2
:10A21000006880680190019840F0770001900198F3
:10A2200004990968886040E004980068039B5A68B4
:10A230009968DB6804F0CEFD04980168886840F4F2
:10A240008040886031E004980068039A5168D268C1
:10A2500004F0ACFF04980068502104F0D5FD24E020
:10A2600004980068039A5168D26804F0C7FF049804
:10A270000068602104F0C8FD17E004980068039AA4
:10A280005168D26804F092FF04980068402104F0FD
:10A29000BBFD0AE0049800680399096804F0B4FD66
:10A2A00003E001208DF80B00FFE70499012081F8FD
:10A2B0003D00FFE70499002081F83C00FFE79DF88E
:10A2C0000B008DF81700FFE79DF8170006B080BD62
:10A2D00080B58AB0099000200890079006900590FC
:10A2E00004900998006840F60001C4F20001884219
:10A2F00023D1FFE7FFE70020039043F63000C4F2CC
:10A300000200016841F008010160006800F00800E7
:10A3100003900398FFE74FF48040049002200590DB
:10A320000121069103210791089040F60040C4F2F4
:10A33000020004A9FDF7B2FA56E00998006840F659
:10A340000041C4F20001884222D1FFE7FFE700206C
:10A35000029043F63000C4F20200016841F080012F
:10A360000160006800F0800002900298FFE74FF45F
:10A37000E05004900220059001210691079008907A
:10A3800041F60040C4F2020004A9FDF787FA2AE072
:10A390000998006844F20041C4F20101884221D1C9
:10A3A000FFE7FFE70020019043F63000C4F202000F
:10A3B000016841F020010160006800F02000019078
:10A3C0000198FFE740200490022005900690079036
:10A3D0000320089041F20040C4F2020004A9FDF7F6
:10A3E0005DFAFFE7FFE7FFE70AB080BD80B586B002
:10A3F00004900391029200208DF80700FFE7049873
:10A4000090F83C00012804D1FFE702208DF81700E6
:10A4100089E00499012081F83C00FFE7FFE70298FA
:10A4200000900C2800F270800099DFE801F0076DC1
:10A430006D6D206D6D6D3A6D6D6D53000498006803
:10A44000039904F0F7FC04980168886940F008005B
:10A45000886104980168886920F004008861039885
:10A4600002690498016888691043886150E0049883
:10A470000068039904F054FD04980168886940F469
:10A480000060886104980168886920F480608861B0
:10A490000398026904980168886940EA022088618B
:10A4A00036E004980068039904F0B4FD049801684C
:10A4B000C86940F00800C86104980168C86920F0C4
:10A4C0000400C8610398026904980168C8691043D0
:10A4D000C8611DE004980068039904F015FE049813
:10A4E0000168C86940F40060C86104980168C869DF
:10A4F00020F48060C8610398026904980168C86903
:10A5000040EA0220C86103E001208DF80700FFE760
:10A51000FFE70499002081F83C00FFE79DF8070061
:10A520008DF81700FFE79DF8170006B080BD00000A
:10A5300080B582B00090009820B9FFE701208DF827
:10A5400007003FE0009890F83D0040B9FFE7009910
:10A55000002081F83C00009800F038F8FFE70099EF
:10A56000022081F83D00009951F8040B04F044FBEF
:10A570000099012081F84600FFE70099012081F849
:10A580003E00009981F83F00009981F84000009951
:10A5900081F84100FFE7FFE70099012081F84200C0
:10A5A000009981F84300009981F84400009981F8EE
:10A5B0004500FFE70099012081F83D0000208DF85B
:10A5C0000700FFE79DF8070002B080BD82B0019050
:10A5D0000198006840F60001C4F20001884212D1DF
:10A5E000FFE7FFE70020009043F64000C4F20200BE
:10A5F000016841F004010160006800F0040000906F
:10A600000098FFE7FFE702B07047000080B58CB00C
:10A610000A900991099828B9FFE70A9890F83E0036
:10A6200007901CE00998042805D1FFE70A9890F8E4
:10A630003F00069010E00998082805D1FFE70A9826
:10A6400090F84000059004E00A9890F841000590C9
:10A65000FFE705980690FFE706980790FFE7079841
:10A66000012804D0FFE701208DF82F00AFE0099802
:10A6700028B9FFE70A99022081F83E001EE00998F8
:10A68000042806D1FFE70A99022081F83F000490D0
:10A6900012E00998082806D1FFE70A99022081F8FC
:10A6A0004000039005E00A99022081F841000390E0
:10A6B000FFE703980490FFE70498FFE70A98006813
:10A6C00009990122019204F069FB01980A9909682D
:10A6D0000022C4F20102914202900CD0FFE70A98D6
:10A6E00000684FF60041CBF6FE710844B0FA80F0E6
:10A6F00040090290FFE70298C00738B1FFE70A98C7
:10A700000168486C40F400404864FFE70A9800681C
:10A710000021C4F2010188423CD0FFE70A9800689A
:10A72000B0F1804F36D0FFE70A98006840F2004150
:10A73000C4F2000188422DD0FFE70A98006840F675
:10A740000001C4F20001884224D0FFE70A980068A3
:10A7500040F60041C4F2000188421BD0FFE70A988E
:10A76000006840F20041C4F20101884212D0FFE7C4
:10A770000A98006844F20001C4F20101884209D03D
:10A78000FFE70A98006841F60001C4F20001884220
:10A7900012D1FFE70A980068806800F0070008906F
:10A7A0000898062807D0FFE70A980168086840F073
:10A7B00001000860FFE706E00A980168086840F0B9
:10A7C00001000860FFE700208DF82F00FFE79DF8EB
:10A7D0002F000CB080BD000080B586B005900491BC
:10A7E000059800680499002204F0D8FA05980168D9
:10A7F00001200022C4F20102914203900CD0FFE735
:10A80000059800684FF60041CBF6FE710844B0FA97
:10A8100080F040090390FFE70398C007D8B1FFE735
:10A82000FFE705980068006A41F21111084210D153
:10A83000FFE705980068006A40F24441084207D1EA
:10A84000FFE705980168486C20F400404864FFE782
:10A85000FFE7FFE7FFE7FFE705980068006A41F2BE
:10A860001111084210D1FFE705980068006A40F214
:10A870004441084207D1FFE705980168086820F0C5
:10A8800001000860FFE7FFE7FFE7049828B9FFE74A
:10A890000599012081F83E001EE00498042806D1A5
:10A8A000FFE70599012081F83F00029012E004982B
:10A8B000082806D1FFE70599012081F840000190A2
:10A8C00005E00599012081F841000190FFE701981A
:10A8D0000290FFE70298FFE7002006B080BD00006D
:10A8E00082B00190ADF8021002B0704780B582B01E
:10A8F0000190019805F086FA8DF803009DF8030099
:10A9000003281BD0FFE79DF8030000EBC00140F2D5
:10A910008850C2F2000000EB8100006968B1FFE7D7
:10A920009DF8030000EBC00140F28850C2F2000025
:10A9300000EB810000698047FFE7FFE702B080BDC0
:10A9400080B592B01190119800680068109011982D
:10A950000068C0680F901198006840690E90002050
:10A960000D900C90109800F00F000D900D9888B984
:10A97000FFE79DF84000800600280AD5FFE79DF814
:10A980003C008006002804D5FFE7119805F05EFA28
:10A9900002E2FFE70D98002800F0C280FFE79DF873
:10A9A0003800C00738B9FFE7BDF83C0010F4907FCD
:10A9B00000F0B680FFE79DF84000C00758B1FFE700
:10A9C0009DF83D00C00730B1FFE71199486C40F099
:10A9D00001004864FFE79DF84000400700280BD5C0
:10A9E000FFE79DF83800C00730B1FFE71199486CC8
:10A9F00040F002004864FFE79DF84000800700280F
:10AA00000BD5FFE79DF83800C00730B1FFE711997B
:10AA1000486C40F004004864FFE79DF840000007E0
:10AA2000002811D5FFE79DF83C008006002805D4DA
:10AA3000FFE79DF83800C00730B1FFE71199486C77
:10AA400040F008004864FFE71198406C002866D089
:10AA5000FFE79DF84000800600280AD5FFE79DF833
:10AA60003C008006002804D5FFE7119805F0EEF9B8
:10AA7000FFE7119800684069C0F380100C901198AE
:10AA8000406C0007002804D4FFE70C9800283ED053
:10AA9000FFE7119805F03CF91198006840694006FD
:10AAA00000282FD5FFE7FFE7FFE71198006850E87F
:10AAB000050F20F040000B90FFE70B9911980268FA
:10AAC00042E805100028F0D1FFE7FFE71198C06BBE
:10AAD00098B1FFE71198C16B4FF65130C0F60000F6
:10AAE00008651198C06BFCF79BFB28B1FFE7119834
:10AAF000C06B016D8847FFE703E01198FFF7F6FE92
:10AB0000FFE703E01198FFF7F1FEFFE706E0119879
:10AB1000FFF7ECFE119900204864FFE7FFE73BE1F7
:10AB20001198006B012840F01781FFE79DF8400065
:10AB3000C006002840F11081FFE79DF83C00C006E8
:10AB4000002840F10981FFE7FFE700200A901198F3
:10AB5000006800680A901198006840680A900A9896
:10AB6000FFE71198006840694006002840F19A808C
:10AB7000FFE71198C06B00684068ADF82600BDF88B
:10AB80002600002875D0FFE7BDF826001199898DB1
:10AB900088426EDAFFE7BDF826001199C885119842
:10ABA000C06BC069B0F5807F58D0FFE7FFE7FFE7D3
:10ABB0001198006850E8030F20F480700890FFE7B8
:10ABC00008991198026842E803100028F0D1FFE7C5
:10ABD000FFE7FFE7FFE71198006850E8050F20F056
:10ABE00001000790FFE707991198026842E80510F5
:10ABF0000028F0D1FFE7FFE7FFE7FFE711980068C3
:10AC000050E8050F20F040000690FFE706991198E4
:10AC1000026842E805100028F0D1FFE7FFE711992C
:10AC2000202081F84200119900200863FFE7FFE728
:10AC30001198006850E8030F20F010000590FFE71E
:10AC400005991198026842E803100028F0D1FFE747
:10AC5000FFE71198C06BFCF76DFAFFE7119902202E
:10AC600048631198818DC28D891A89B2FFF738FE29
:10AC700017E0BDF826001199898D884210D1FFE7B1
:10AC80001198C06BC069B0F5807F08D1FFE71199BA
:10AC9000022048631198818DFFF722FEFFE7FFE74E
:10ACA000FFE779E01199888DC98D401AADF812003F
:10ACB0001198C08D00284ED0FFE7BDF81200002883
:10ACC00049D0FFE7FFE7FFE71198006850E8030F5E
:10ACD00020F490700390FFE703991198026842E80E
:10ACE00003100028F0D1FFE7FFE7FFE7FFE7119827
:10ACF000006850E8050F20F001000290FFE702997C
:10AD00001198026842E805100028F0D1FFE7FFE73C
:10AD10001199202081F84200119900200863FFE773
:10AD2000FFE71198006850E8030F20F01000019031
:10AD3000FFE701991198026842E803100028F0D15A
:10AD4000FFE7FFE71199022048631198BDF8121040
:10AD5000FFF7C6FDFFE71FE09DF840000006002852
:10AD60000AD5FFE79DF83C000006002804D5FFE760
:10AD7000119805F055FA0FE09DF8400040060028B4
:10AD80000AD5FFE79DF83C004006002804D5FFE700
:10AD9000119805F007F8FFE712B080BD80B582B0CA
:10ADA0000090009820B9FFE701208DF8070040E0EF
:10ADB0000098806908B1FFE700E0FFE7009890F88D
:10ADC000410040B9FFE70099002081F84000009859
:10ADD00000F034F8FFE70099242081F84100009842
:10ADE0000168C86820F40050C860009805F0E2F8D7
:10ADF00000980168086920F4904008610098016893
:10AE0000486920F02A00486100980168C86840F449
:10AE10000050C860009900204864009A202182F800
:10AE20004110009A82F84210009948638DF807009B
:10AE3000FFE79DF8070002B080BD000080B590B02C
:10AE40000F9000200E900D900C900B900A900F9890
:10AE5000006844F60001C4F2000188425FD1FFE7B8
:10AE6000FFE70020099043F64000C4F202000168A9
:10AE700041F480210160006800F480200990099865
:10AE8000FFE7FFE70020089043F63000C4F202001D
:10AE9000016841F004010160006800F004000890BE
:10AEA0000898FFE74FF440600A9002200B900020C2
:10AEB00004900C9003200D9007200E9040F60000A7
:10AEC000C4F202000AA9FCF7E9FC049940F6AC5070
:10AED000C2F20000059046F22802C4F202020260AB
:10AEE0004FF0006242608160C1604FF48062026195
:10AEF00041618161C16101624162FCF743FB18B1AC
:10AF0000FFE7FAF763FCFFE7FFE70F9840F6AC5165
:10AF1000C2F20001C1630F988863FFE79CE00F98BD
:10AF2000006841F20041C4F20101884240F0938080
:10AF3000FFE7FFE70020079043F64400C4F2020059
:10AF4000016841F020010160006800F020000790D6
:10AF50000798FFE7FFE70020069043F63000C4F2B1
:10AF60000200016841F040010160006800F040000B
:10AF700006900698FFE74FF484400A9002200B9059
:10AF8000002002900C9003200D9008200E9041F6B6
:10AF90000000C4F202000AA9FCF780FC029940F606
:10AFA0000C60C2F20000039046F22842C4F2020292
:10AFB00002604FF0206242608160C1604FF48062A5
:10AFC000026141618161C16101624162FCF7DAFAAB
:10AFD00018B1FFE7FAF7FAFBFFE7FFE70F9840F633
:10AFE0000C61C2F20001C1630F988863FFE740F66D
:10AFF0006C60C2F20000019046F2A041C4F202016E
:10B0000001604FF020614160402181600021C160FA
:10B010004FF48062026141618161C16101624162FC
:10B02000FCF7B0FA18B1FFE7FAF7D0FBFFE7FFE74C
:10B030000F9840F66C61C2F2000181630F9888633B
:10B04000FFE74720009005210022FDF7CBF800988C
:10B05000FDF7BEF8FFE7FFE710B080BD80B584B014
:10B0600002900191ADF80220029890F84200202849
:10B0700017D1FFE7019820B1FFE7BDF8020020B922
:10B08000FFE701208DF80F000FE002990020086310
:10B0900002980199BDF8022005F02AF88DF80F00FA
:10B0A00003E002208DF80F00FFE79DF80F0004B0C9
:10B0B00080BD000080B582B00190019804F0A2FE2E
:10B0C0008DF803009DF8030003281BD0FFE79DF8CF
:10B0D000030000EBC00140F28850C2F2000000EB18
:10B0E0008100C06868B1FFE79DF8030000EBC00174
:10B0F00040F28850C2F2000000EB8100C068804737
:10B10000FFE7FFE702B080BD80B582B001900198F3
:10B1100004F078FE8DF803009DF8030003281BD08F
:10B12000FFE79DF8030000EBC00140F28850C2F237
:10B13000000000EB8100806868B1FFE79DF8030024
:10B1400000EBC00140F28850C2F2000000EB810029
:10B1500080688047FFE7FFE702B080BD80B582B01E
:10B160000190019804F04EFE8DF803009DF8030055
:10B1700003281BD0FFE79DF8030000EBC00140F25D
:10B180008850C2F2000000EB8100406868B1FFE720
:10B190009DF8030000EBC00140F28850C2F20000AD
:10B1A00000EB810040688047FFE7FFE702B080BD09
:10B1B000FFE7FEE784B08DED030A9DED030AB6EECE
:10B1C000001A20EE010A8DED020A03980190019801
:10B1D0000090009945F6DF10C5F63770A0EB6100CE
:10B1E0000090009801909DED010A9DED021A21EE5C
:10B1F000001A21EE002AB7EE081A31EE422A20EE9C
:10B20000020A8DED010A9DED010A9DED022A22EE52
:10B21000002A22EE002A31EE421A20EE010A8DEDBC
:10B22000010A9DED010A04B07047000080B586B0A8
:10B2300004908DED030A049818B9FFE700200590EB
:10B240004CE09DED030A049890ED014A90ED022A2E
:10B2500090ED063A90ED071A23EE043A30EE430AD9
:10B2600021EE021A30EE410A8DED020A002028B9C3
:10B27000FFE7029805F09CF858B90DE002980BF032
:10B280009FF941EC100B51EC100B05F077F818B159
:10B29000FFE703980290FFE79DED020A049890ED06
:10B2A000034A90ED043A90ED052A90ED061A20EE3F
:10B2B000040A21EE031A30EE010A90ED071A21EE7E
:10B2C000021A30EE010A8DED010A04998869C861FD
:10B2D00002980499886101980590FFE79DED050AA1
:10B2E00006B080BD80B588B007908DED060ACDED23
:10B2F000050A079808B9FFE78BE0059807990860E9
:10B300000799002088610799C861079890ED000AA5
:10B31000B5EE400AF1EE10FA0EDCFFE707994FF0A8
:10B320007E50C86007990020086107994861079915
:10B330004860079988606CE09DED060A079890EDDB
:10B34000001A80EE010A8DED040A9DED041A9FEDAE
:10B35000320A80EE010A0AF0A9F98DED030A9FED89
:10B360002F0A8DED000A0AF031F8B0EE401A9DED7B
:10B37000000A31EE011A9DED033A21EE031AB7EEF1
:10B38000002A8DED012A31EE021A23EE033A31EE46
:10B39000031A8DED021A9DED031A21EE011A9DED9F
:10B3A000023A81EE031A079880ED031A079890ED90
:10B3B000031A31EE011A80ED041A0799C868486132
:10B3C0009DED031A21EE011A31EE421A31EE011AF7
:10B3D0009DED022A81EE021A079880ED011A09F00C
:10B3E000F5FFB0EE401A9DED010A31EE012A9DED08
:10B3F000031A22EE012A30EE420A21EE011A30EE43
:10B40000010A9DED021A80EE010A079880ED020AFA
:10B41000FFE708B080BD00BFDB0F4940DB0F493FAD
:10B4200080B584B002908DED010A029818B9FFE74B
:10B430000020039039E09DED010A029890ED031A77
:10B4400090ED043A90ED052A31EE031A31EE021A1E
:10B4500080EE010A8DED000A002028B9FFE7009870
:10B4600004F068FF58B911E000980BF0A9F841EC1E
:10B47000100B51EC100B04F02DFF38B1FFE70098D2
:10B480000299886100980299C86106E001980299C2
:10B49000886101980299C861FFE702989DED010A51
:10B4A000FFF7C4FE8DED030AFFE79DED030A04B02C
:10B4B00080BD000080B582B08DF806009DF80600C2
:10B4C000022804DBFFE7FF208DF8070039E09DF834
:10B4D000061040F27C60C2F2000050F8210020B15A
:10B4E000FFE700208DF807002BE08820F7F74AFDE2
:10B4F00001469DF8062040F27C60C2F2000040F850
:10B5000022109DF8061050F8210020B9FFE7FF2017
:10B510008DF8070015E09DF8061040F27C60C2F23D
:10B520000000009050F821008821F4F7EEFF009908
:10B530009DF8060051F82010087000208DF80700D3
:10B54000FFE79DF9070002B080BD000080B588B01C
:10B550000690069820B9FFE7FE208DF81F002EE028
:10B56000069800F049F80590059820B9FFE7FC20FF
:10B570008DF81F0023E005988088019008208DF841
:10B580000800FF208DF809008DF80A008DF80B00E7
:10B590008DF80C008DF80D008DF80E008DF80F0061
:10B5A000FC208DF810000598007801A9F7F79EFAA5
:10B5B000002818BF4FF0FF308DF81F00FFE79DF9FE
:10B5C0001F0008B080BD000082B08DF803009DF818
:10B5D0000300022803DBFFE70020019009E09DF84B
:10B5E000031040F27C60C2F2000050F8210001908C
:10B5F000FFE7019802B0704780B586B004900498C8
:10B6000018B9FFE70020059036E004980078FFF7AE
:10B61000DBFF0390039818B9FFE7002005902BE0AB
:10B6200000200290FFE70298039991F88410884265
:10B630001FDAFFE70398029900EB81004068019050
:10B64000019888B1FFE70198007804990978884249
:10B650000AD1FFE70198408804994988884203D1BC
:10B66000FFE70198059007E0FFE70298013002909C
:10B67000D9E700200590FFE7059806B080BD0000DF
:10B6800080B584B002900191029818B1FFE701984B
:10B6900020B9FFE7FE208DF80F0011E00298FFF7B8
:10B6A000ABFF0090009820B9FFE7FC208DF80F0059
:10B6B00006E00098019900F049F98DF80F00FFE7C6
:10B6C0009DF90F0004B080BD80B586B00490039151
:10B6D000049818B1FFE7039820B9FFE7FE208DF822
:10B6E000170090E003984178807840EA0120ADF897
:10B6F0000A00BDF80A009FED460ADFED460A102158
:10B7000006F068FE049880ED070A0399C878097965
:10B71000000140EA1110ADF80800BDF80800BBEECA
:10B720000E0AF3EE0E0A0C21009106F053FE00996A
:10B73000049880ED080A03980279407902F00F021C
:10B7400040EA0220ADF80600BDF80600BAEE080A8D
:10B75000F2EE080A06F03EFE049880ED090A03980E
:10B76000807900EE100AB8EE400A049880ED0A0ACB
:10B77000FFE7049890ED070AB5EE400AF1EE10FAE3
:10B780000ADAFFE7049890ED070A9FED231A30EEDE
:10B79000010A80ED070AECE7FFE7049890ED070A3D
:10B7A0009FED1D1AB4EE410AF1EE10FA0ADBFFE735
:10B7B000049890ED070A9FED191A30EE010A80ED0A
:10B7C000070AEAE70498C079C007C0B1FFE7049808
:10B7D00090ED071A9FED100A30EE410A80ED070A3E
:10B7E000049890ED080AB1EE400A80ED080A04982A
:10B7F00090ED090AB1EE400A80ED090AFFE700204A
:10B800008DF81700FFE79DF9170006B080BD00BF57
:10B81000DA0F49C1DA0F4941DB0FC940DB0FC9C05C
:10B8200080B586B00490049820B9FFE7FE208DF81B
:10B83000170087E004980078FFF73CFE20B1FFE78F
:10B84000FF208DF817007DE004980078FFF7BCFE1C
:10B850000390039820B9FFE7FF208DF8170071E0EF
:10B8600000200290FFE70298039991F88410884223
:10B870001BDAFFE70398029900EB8100406878B17A
:10B88000FFE70398029900EB810040684088049923
:10B890004988884204D1FFE7FD208DF8170051E068
:10B8A000FFE7029801300290DDE7039890F88400EA
:10B8B000202804DBFFE7FF208DF8170042E030204E
:10B8C000F7F760FB0190019820B9FFE7FF208DF8A2
:10B8D000170037E001983021F4F717FE0199049A18
:10B8E000106852684A600860019900200872049844
:10B8F000C079019900F00100087604984088ADF8FD
:10B90000020004980078BDF802100322F6F72CFF1D
:10B9100038B1FFE70198F7F73FFAFF208DF81700DD
:10B9200010E00198039991F8842001EB82014860AE
:10B93000039991F88400013081F8840000208DF88B
:10B940001700FFE79DF9170006B080BD80B58EB0E7
:10B950000C900B910C9818B1FFE70B9820B9FFE7FA
:10B96000FE208DF8370087E00C988088ADF818002D
:10B970000B9890ED020ADFED420A9FED421A10206B
:10B9800004F07CFEADF822000B9890ED010AFBEE6E
:10B990000E0AB3EE0E1A0C20019004F06FFE014661
:10B9A0000198ADF820100B9991ED030ADFED360AEE
:10B9B000CDED000A9FED351A04F060FEDDED000AC2
:10B9C00001460198ADF81E100B9991ED040AB1EEF5
:10B9D000041A04F053FE01460198ADF81C100B99AF
:10B9E00091ED000AFAEE080AB2EE081A04F046FEDB
:10B9F000ADF81A009DF823008DF824009DF8220070
:10BA00008DF82500BDF8200000098DF82600BDF84E
:10BA100020109DF81F0040EA01108DF827009DF8C6
:10BA20001E008DF82800BDF81C0000098DF82900C3
:10BA3000BDF81C109DF81B0040EA01108DF82A008B
:10BA40009DF81A008DF82B000C9880880290082031
:10BA50008DF80C0009980A99CDF81110CDF80D0059
:10BA60000C98007802A9F7F741F8002818BF4FF0AA
:10BA7000FF308DF83700FFE79DF937000EB080BD2D
:10BA8000DA0F49C1DA0F4941000000000000FA4313
:10BA900080B590B00E900E9820B9FFE7FE208DF88B
:10BAA0003F0077E00E980078FFF78EFD0D900D981F
:10BAB00020B9FFE7FC208DF83F006BE000200C90E0
:10BAC0000B90FFE70B980D9991F8841088421EDACD
:10BAD000FFE70D980B9900EB8100406890B1FFE7FC
:10BAE0000D980B9900EB8100406840880E994988B9
:10BAF000884207D1FFE70D980B9900EB8100406861
:10BB00000C9004E0FFE70B9801300B90DAE70C98FB
:10BB100020B9FFE7FC208DF83F003BE00E984088FD
:10BB2000ADF82A000E980078BDF82A1003AA002369
:10BB3000F6F7ACFCE0B1FFE7F7F70EFC01910090DF
:10BB4000009901980C9A13695269C91A904148F2F8
:10BB5000A162C0F20102891A70F1000004D3FFE76C
:10BB60000C9900200872FFE7FF208DF83F0011E0DC
:10BB70000C9901200872F7F7EFFB0A460C994A610D
:10BB800008610C9803A90D31FFF79EFD00208DF888
:10BB90003F00FFE79DF93F0010B080BD80B582B047
:10BBA0008DF806009DF80600022804DBFFE7FF2061
:10BBB0008DF8070039E09DF8061040F28460C2F26B
:10BBC000000050F8210020B1FFE700208DF80700A9
:10BBD0002BE04820F7F7D6F901469DF8062040F201
:10BBE0008460C2F2000040F822109DF8061050F860
:10BBF000210020B9FFE7FF208DF8070015E09DF830
:10BC0000061040F28460C2F20000009050F821005B
:10BC10004821F4F77AFC00999DF8060051F82010AD
:10BC2000087000208DF80700FFE79DF9070002B0BB
:10BC300080BD000080B58EB00C900C9820B9FFE755
:10BC4000FE208DF83700A9E00C98007800F0AAF8E3
:10BC50000B900B9820B9FFE7FC208DF837009DE092
:10BC60000B9802300A900C984088ADF81600BDF889
:10BC70001610A1F20120019104280CD3FFE70198CE
:10BC8000A0F20520042829D3FFE70198A0F209209B
:10BC9000032849D372E04FF40070069008208DF815
:10BCA0001C0000200490FFE70498032815DCFFE740
:10BCB0000A98049A00EB4200407806A9053101F881
:10BCC00012000A98049A30F8120001EB4201487001
:10BCD000FFE7049801300490E6E753E040F2FF10DC
:10BCE000069008208DF81C0004200390FFE70398BD
:10BCF000072818DCFFE70A98039A00EB4200407817
:10BD000006A9053101EB420202F8080C0A98039AD1
:10BD100030F8120001EB420101F8070CFFE703982D
:10BD200001300390E3E72DE040F2FF200690082069
:10BD30008DF81C000290FFE702980A2818DCFFE744
:10BD40000A98029A00EB4200407806A9053101EBFF
:10BD5000420202F8100C0A98029A30F8120001EB25
:10BD6000420101F80F0CFFE7029801300290E3E76F
:10BD700000208DF823008DF8240003E0FF208DF8CB
:10BD800037000BE00C98007806A9F6F7AFFE002804
:10BD900018BF4FF0FF308DF83700FFE79DF93700EF
:10BDA0000EB080BD82B08DF803009DF8030002281C
:10BDB00003DBFFE70020019009E09DF8031040F24B
:10BDC0008460C2F2000050F821000190FFE7019862
:10BDD00002B0704782B08DF805009DF8050001465D
:10BDE000009140B1FFE70098012809D0FFE70098D3
:10BDF00002280AD00EE042F21070ADF806000EE004
:10BE00004FF48040ADF8060009E047F23050ADF83D
:10BE1000060004E04FF6FF70ADF80600FFE7BDF93D
:10BE2000060002B07047000083B0ADF808008DF83E
:10BE300007109DF8070001460091022804D3FFE790
:10BE40000098022813D026E0BDF80800B0F5007F66
:10BE50000CDDFFE7BDF80800B0F5027F06DAFFE76A
:10BE6000BDF8080001388DF80B0019E014E0BDF8AA
:10BE70000800B0F5017F0DDDFFE7BDF8080040F2D6
:10BE80000A21884206DCFFE7BDF8080001388DF87A
:10BE90000B0005E000E0FFE7FF208DF80B00FFE757
:10BEA0009DF90B0003B0704780B586B004900498EC
:10BEB00018B9FFE7002005902FE004980078FFF7FD
:10BEC00071FF0390039818B9FFE70020059024E064
:10BED00000200290FFE70298039991F844108842ED
:10BEE00018DAFFE70398029900EB8100806901905E
:10BEF000019850B1FFE70198408804994988884229
:10BF000003D1FFE70198059007E0FFE702980130B1
:10BF10000290E0E700200590FFE7059806B080BD9D
:10BF200083B08DF807009DF807000146009140B1ED
:10BF3000FFE70098012809D0FFE7009802280BD0FE
:10BF40000EE00020C4F2102002900DE04AF22C0016
:10BF5000C4F29910029007E04FF07E50029003E087
:10BF60004FF07E500290FFE79DED020A03B070474C
:10BF700080B586B00490049820B9FFE7FE208DF8C4
:10BF8000170081E004980078FFF708FE20B1FFE772
:10BF9000FF208DF8170077E004980078FFF702FF84
:10BFA0000390039820B9FFE7FF208DF817006BE09E
:10BFB00000200290FFE70298039991F8441088420C
:10BFC0001BDAFFE70398029900EB8100806978B1E2
:10BFD000FFE70398029900EB81008069408804998B
:10BFE0004988884204D1FFE7FD208DF817004BE017
:10BFF000FFE7029801300290DDE7039890F84400D3
:10C000000B2804DBFFE7FF208DF817003CE05020F1
:10C01000F6F7B8FF0190019820B9FFE7FF208DF8EF
:10C02000170031E00199049A106852684A6008606C
:10C03000019818302821F4F768FA0498407901999A
:10C0400000F0010081F8280004990878498803224B
:10C05000F6F78AFB38B1FFE70198F6F79DFEFF205F
:10C060008DF8170010E00198039991F8442001EB36
:10C0700082018861039991F84400013081F84400FD
:10C0800000208DF81700FFE79DF9170006B080BD6E
:10C0900080B582B0019001989FED020A00F004F88B
:10C0A00002B080BD0000000080B58AB007A90191F0
:10C0B00001460198089180ED000A089820B9FFE731
:10C0C000FE208DF8270078E008980078FFF76AFED8
:10C0D0000690069820B9FFE7FC208DF827006CE059
:10C0E000019890ED000AB7EE001AB4EE410AF1EEA5
:10C0F00010FA04DDFFE74FF07E500790FFE701984C
:10C1000090ED000ABFEE001AB4EE410AF1EE10FA0B
:10C1100005DAFFE70020CBF680700790FFE708986C
:10C120004079C00740B1FFE7019890ED000AB1EEF9
:10C13000400A80ED000AFFE70898FFF7B5FE05907A
:10C14000059820B9FFE7FC208DF8270035E0089915
:10C1500048880979FFF768FE8DF813009DF91300F0
:10C16000B0F1FF3F04DCFFE7FF208DF8270024E05B
:10C17000019806990231039190ED000A8DED000AB5
:10C1800008980079FFF726FE9DED000A01EE100ADF
:10C19000B8EEC11A20EE010ABDEEC00A10EE100A78
:10C1A000ADF80A00BDF80A0003999DF9132021F8A3
:10C1B000120000208DF82700FFE79DF927000AB044
:10C1C00080BD000080B590B00E900E9820B9FFE7BA
:10C1D000FE208DF83F0072E00E980078FFF7E2FD38
:10C1E0000D900D9820B9FFE7FC208DF83F0066E028
:10C1F00000200C90FFE70C980D9991F844108842AC
:10C2000059DAFFE70D980C9900EB810080690B90DB
:10C210000B9800284AD0FFE70B9840880E99498870
:10C22000884243D1FFE70E990878498804AA002381
:10C23000F6F72CF9E8B1FFE7F7F78EF803910290D3
:10C24000029903980B9A136A526AC91A904140F2F4
:10C25000E932891A70F1000007D3FFE70B9900203B
:10C260000876FC208DF83F0029E0FF208DF83F0084
:10C2700025E00B9901200876F7F76EF80A460B992E
:10C280004A6208620B9804A900F008FD0B9901911D
:10C290008868CA680B69D1F814C0C1F838C04B630C
:10C2A0000A63C86200208DF83F0008E0FFE70C98A1
:10C2B00001300C909FE7FC208DF83F00FFE79DF9CF
:10C2C0003F0010B080BD000080B582B040F63C4019
:10C2D000C2F20000019046F20041C4F20001016088
:10C2E0000321416000218160C1604FF4102202618E
:10C2F0004FF4001242610176417681760122C276C6
:10C3000001774177FAF71AFB18B1FFE7F9F75EFA00
:10C31000FFE702B080BD000080B582B040F6644007
:10C32000C2F20000019046F60001C4F20001016073
:10C330000321416000218160C1604FF4102202613D
:10C340004FF4001242610176417681760122C27675
:10C3500001774177FAF7F2FA18B1FFE7F9F736FA01
:10C36000FFE702B080BD000080B58AB0FFE7002083
:10C37000099043F63000C4F20200016841F4001154
:10C380000160006800F4001009900998FFE7FFE7DA
:10C390000020089043F63000C4F20200016841F426
:10C3A00080010160006800F4800008900898FFE7B1
:10C3B0000C2000900521059100220692FBF712FF48
:10C3C0000098FBF705FF0599069A0D200190FBF7F1
:10C3D00009FF0198FBF7FCFE0599069A39200290A7
:10C3E000FBF700FF0298FBF7F3FE0599069A3A2047
:10C3F0000390FBF7F7FE0398FBF7EAFE0599069A10
:10C400003B200490FBF7EEFE0498FBF7E1FE059954
:10C41000069A45200790FBF7E5FE0798FBF7D8FE44
:10C420000AB080BD80B582B04EF6A920C0F60000EB
:10C4300046F6F012C0F601020021019104F018FE48
:10C44000019940F62C22C2F2000210604FF25120F6
:10C45000C0F6000046F69812C0F6010204F008FE8D
:10C4600002B080BD80B59AB0002019901890179046
:10C4700016901590FFE70020149043F63000C4F2A8
:10C480000200016841F002010160006800F0020052
:10C4900014901498FFE7FFE70020139043F6300054
:10C4A000C4F20200016841F040010160006800F040
:10C4B000400013901398FFE7FFE70020129043F627
:10C4C0003000C4F20200016841F00101016000681F
:10C4D00000F0010012901298FFE7FFE70020119092
:10C4E00043F63000C4F20200016841F00801016027
:10C4F000006800F0080011901198FFE7FFE70020A6
:10C50000109043F63000C4F20200016841F00401CB
:10C510000160006800F0040010901098FFE7FFE74A
:10C5200000200F9043F63000C4F20200016841F091
:10C5300080010160006800F080000F900F98FFE715
:10C54000FFE700200E9043F63000C4F202000168BD
:10C5500041F020010160006800F020000E900E986C
:10C56000FFE741F60000C4F2020001904021009173
:10C5700000220C92FBF786FB0020C4F2020003901D
:10C580001021029101220592FBF77CFB059A40F2F3
:10C590000040C4F2020006901146FBF773FB009ABC
:10C5A00001980599159216911791189115A907915F
:10C5B000FBF774F90198059A0799082315934FF42E
:10C5C0000413049316931792FBF768F90398049BDE
:10C5D000059A0799159216931792FBF75FF9029B3C
:10C5E0000398059A07991593169217921892FBF7DC
:10C5F00055F9049A059807993023159316921790C8
:10C6000040F60000C4F20200FBF748F9059A0698CC
:10C6100007991592169217921892FBF73FF90C9A08
:10C620000620089005210B91FBF7DCFD0898FBF72D
:10C63000CFFD0B990C9A09200990FBF7D3FD0998BF
:10C64000FBF7C6FD0B990C9A0A200A90FBF7CAFD6E
:10C650000A98FBF7BDFD0B990C9A17200D90FBF77C
:10C66000C1FD0D98FBF7B4FD1AB080BD80B582B056
:10C6700040F6CC60C2F20000019045F60041C4F2E1
:10C680000001016041F68021C0F2060141600021F5
:10C690008160C1604FF48042026141618161C1618A
:10C6A0000162FBF70DFB18B1FFE7F9F78FF8FFE721
:10C6B00002B080BD80B582B040F62070C2F20000AA
:10C6C000019043F20001C4F2010101604FF4827154
:10C6D000416000218160C160022202610122426149
:10C6E0004FF4007282611822C2610162416281626C
:10C6F0000A21C162FCF7F2FA18B1FFE7F9F766F810
:10C70000FFE702B080BD000080B588B00021009135
:10C71000079106910591049103910291019140F6D0
:10C720007870C2F2000044F20042C4F201020260DA
:10C730004160816041F28732C26001618161FDF731
:10C740007BFC18B1FFE7F9F741F8FFE740F6787096
:10C75000C2F20000FDF7ECFE18B1FFE7F9F736F87A
:10C76000FFE760200190002202920392059240F6BA
:10C770007870C2F2000001A9FDF738FE18B1FFE79A
:10C78000F9F724F8FFE740F67870C2F20000FDF7F1
:10C790009FFD08B080BD000080B58AB000210091E7
:10C7A00009910891079106910591049103910291D5
:10C7B000019140F6C070C2F2000040F60002C4F2DF
:10C7C00000020260416081604FF6FF72C260016149
:10C7D0008161FDF7ADFE18B1FFE7F8F7F7FFFFE75E
:10C7E00000200890099040F6C070C2F2000008A92D
:10C7F000FDF790FB18B1FFE7F8F7E8FFFFE76020CF
:10C800000190002002900390059040F6C070C2F2A3
:10C81000000001A90822FDF7E9FD18B1FFE7F8F7CC
:10C82000D5FFFFE740F6C070C2F20000FDF750FDF3
:10C830000AB080BD80B58EB0002100910D910C91A1
:10C840000B910A9109910891079106910591049124
:10C8500003910291019141F20800C2F2000040F6FA
:10C860000042C4F200020260416081604FF6FF7234
:10C87000C26001618161FDF7DFFB18B1FFE7F8F7E6
:10C88000A5FFFFE74FF480500A9041F20800C2F282
:10C8900000000AA9FDF75AFC18B1FFE7F8F796FF68
:10C8A000FFE741F20800C2F20000FDF741FE18B1B7
:10C8B000FFE7F8F78BFFFFE700200890099041F2AF
:10C8C0000800C2F2000008A9FDF724FB18B1FFE739
:10C8D000F8F77CFFFFE760200190002202920392AC
:10C8E000059241F20800C2F2000001A9FDF77EFDA9
:10C8F00018B1FFE7F8F76AFFFFE741F20800C2F25C
:10C90000000001A90422FDF771FD18B1FFE7F8F757
:10C910005DFFFFE741F20800C2F2000001A9082212
:10C92000FDF764FD18B1FFE7F8F750FFFFE741F2AC
:10C930000800C2F20000FDF7CBFC0EB080BD000085
:10C9400080B582B041F25000C2F20000019044F67E
:10C950000001C4F20001016048F2A061C0F20101CF
:10C96000416000218160C16001610C2242618161EE
:10C97000C161FEF713FA18B1FFE7F8F727FFFFE7E9
:10C9800002B080BD80B582B041F29800C2F20000D2
:10C99000019041F20041C4F2010101604FF4E13124
:10C9A000416000218160C16001610C2242618161AE
:10C9B000C161FEF7F3F918B1FFE7F8F707FFFFE7EA
:10C9C00002B080BDFFE7FEE780B58DB00DF1100C21
:10C9D000CDF808C084460298CDF82CC00A9109927F
:10C9E0008DF8233080ED030A0B9820B9FFE7FF2074
:10C9F0008DF8330035E10B98007801460191052848
:10CA000000F289800199DFE801F0034565858579A9
:10CA10009DF9230004283BD1FFE70A9890ED000A16
:10CA200090ED012A90ED021A30EE420A30EE010A32
:10CA3000099880ED000A0A9890ED000A90ED012A0D
:10CA400090ED021A30EE020A30EE010A099880EDEC
:10CA5000010A0A9890ED002A90ED011A90ED020A61
:10CA600031EE421A30EE010A099880ED020A0A9866
:10CA700090ED000A90ED012A90ED021AB1EE400A05
:10CA800030EE420A30EE010A099880ED030A00E018
:10CA9000CBE040E09DF92300042819D1FFE70A9874
:10CAA00090ED000AB1EE400A099880ED000A0A985C
:10CAB0000068099948600A980068099988600A988E
:10CAC00090ED000AB1EE400A099880ED030A00E0FB
:10CAD000ABE0FFE79DF9230002280DD1FFE70A989C
:10CAE00090ED000AB1EE400A099880ED000A0A981C
:10CAF00000680999486000E097E0FFE79DF923008E
:10CB0000012805D1FFE70A9800680999086000E04C
:10CB10008BE0FFE789E0002006908DF81700FFE723
:10CB20009DF917009DF9231088422EDAFFE702983D
:10CB300009999DF9172001EB820191ED000AB0EEF1
:10CB4000C00A80ED000A90ED000A90ED021AB4EEE2
:10CB5000410AF1EE10FA06DDFFE7029890ED000AB7
:10CB60008DED000A05E0029890ED020A8DED000AB5
:10CB7000FFE702989DED000A80ED020AFFE79DF8AD
:10CB8000170001308DF81700CAE7029890ED020AED
:10CB9000B7EE001AB4EE410AF1EE10FA21DDFFE71C
:10CBA00000208DF80F00FFE79DF90F009DF923107D
:10CBB000884215DAFFE7029890ED021A09989DF96C
:10CBC0000F1000EB810090ED000A80EE010A80ED6D
:10CBD000000AFFE79DF80F0001308DF80F00E3E732
:10CBE000FFE700208DF80E00FFE79DF90E009DF98C
:10CBF0002310884215DAFFE7029890ED031A09988E
:10CC00009DF90E1000EB810090ED000A20EE010A64
:10CC100080ED000AFFE79DF80E0001308DF80E0050
:10CC2000E3E700208DF833001BE000208DF80D00B5
:10CC3000FFE79DF80D009DF9231088420DDAFFE70C
:10CC400009999DF80D20002041F82200FFE79DF88A
:10CC50000D0001308DF80D00EBE7FF208DF833005B
:10CC6000FFE79DF933000DB080BD000083B0019057
:10CC70008DF80310019820B9FFE7FF208DF80B0015
:10CC800007E09DF803000199087000208DF80B0063
:10CC9000FFE79DF90B0003B07047000080B58AB034
:10CCA000099008910898417B807B40EA0120ADF80B
:10CCB0001E000898C17B007C40EA0120ADF81C00F2
:10CCC0000898417C807C40EA0120ADF81A00099860
:10CCD0000079FFF77FF8ADF8180009980079FFF7A1
:10CCE0001FF98DED050ABDF81E0000EE100AB8EE22
:10CCF000C00A9FED6D1A80EE010A9FED6C1A20EEBE
:10CD0000010A8DED040ABDF91C0000EE100AB8EE10
:10CD1000C00A8DED030ABDF91A00BDF91810484389
:10CD200000EE100AB8EEC00A9FED611A80EE010A0B
:10CD30008DED020A09988079C00700284CD0FFE7E2
:10CD4000BDF81E000999B1F84010401A01900198F1
:10CD5000B0F5805F05DDFFE70999486C013848644C
:10CD60000AE0019810F5805F05DAFFE70999486C41
:10CD700001304864FFE7FFE7BDF81E000999A1F8FC
:10CD8000400004980090099890ED110AB8EEC00A8E
:10CD90009FED461A20EE010A9DED001A30EE010AC1
:10CDA0009DED051A80EE010A80ED120A0999886C42
:10CDB00088609DED030A9DED051A80EE010A099831
:10CDC00080ED030A9DED020A9DED051A20EE010A91
:10CDD000099880ED040A13E0099900204864BDF821
:10CDE0001E10099AA2F840100999886404980999BC
:10CDF000886003980999C860029809990861FFE75B
:10CE0000FFE7099890ED020AB5EE400AF1EE10FA3C
:10CE10000ADAFFE7099890ED020A9FED241A30EE36
:10CE2000010A80ED020AECE7FFE7099890ED020A9B
:10CE30009FED1E1AB4EE410AF1EE10FA0ADBFFE78D
:10CE4000099890ED020A9FED1B1A30EE010A80ED61
:10CE5000020AEAE7099890F82800C007C0B1FFE786
:10CE6000099890ED021A9FED110A30EE410A80ED0B
:10CE7000020A099890ED030AB1EE400A80ED030A18
:10CE8000099890ED040AB1EE400A80ED040AFFE72C
:10CE90000898C07C00EE100AB8EE400A099880EDB0
:10CEA000050A0AB080BD00BF00000046DB0FC94084
:10CEB00000008046DB0FC9C0FFE7FEE788B007909F
:10CEC00006910592079800F0070004900498C0F1BD
:10CED0000700052803D3FFE70420019004E004982D
:10CEE000C0F107000190FFE7019803900498043017
:10CEF000062803D8FFE70020009003E004980338D9
:10CF00000090FFE70098029006980399012202FA28
:10CF100001F101390840029B984005999A40013A75
:10CF20001140084308B0704780B590B00E908DED69
:10CF30000D0ACDED0C0A8DED0B1ACDED0A1A00206D
:10CF400028B9FFE70D9803F001FA58B943E00D98AE
:10CF500009F036FB41EC100B51EC100B03F0CAF951
:10CF6000C8B3FFE7002028B9FFE70C9803F0EEF9FB
:10CF700058B930E00C9809F023FB41EC100B51EC50
:10CF8000100B03F0B7F930B3FFE7002028B9FFE733
:10CF90000B9803F0DBF958B91DE00B9809F010FB72
:10CFA00041EC100B51EC100B03F0A4F998B1FFE722
:10CFB000002028B9FFE70A9803F0C8F978B90AE019
:10CFC0000A9809F0FDFA41EC100B51EC100B03F03C
:10CFD00091F920B9FFE70E9880690F9016E19DED59
:10CFE0000D0ADDED0C0A0E98406890ED071AF7F770
:10CFF00043F88DED090A9DED090A0E98406890ED01
:10D00000001A20EE010A8DED080A0E98406890ED96
:10D01000000A9DED0C1A20EE010A8DED070A0E980C
:10D020001C309DED070AFEF701F98DED060A0E98FA
:10D0300000780146019110B3FFE70198012804D060
:10D04000FFE70198022817D01CE09DED060A0E9814
:10D0500090ED021A90ED052A30EE420A9DED0A2A63
:10D06000B4EE412AF1EE10FAC8BFB0EE421A80EEDB
:10D07000010A8DED050A05E00B98059002E00020FD
:10D080000590FFE709980E99086106980E99486186
:10D09000002028B9FFE7059803F058F970B90AE0B5
:10D0A000059809F08DFA41EC100B51EC100B03F0D0
:10D0B00021F918B9FFE700200590FFE79DED080A68
:10D0C0000E98406890ED011A90ED032A20EE010AB7
:10D0D0009DED051A21EE021A30EE410A8DED040A8B
:10D0E0000E9890ED030A9DED081A9DED0A2A21EE97
:10D0F000021A30EE010A8DED030A9DED030A0E9827
:10D10000406890ED021A20EE010A8DED020A0E9899
:10D11000406890ED020A9FED3F1AB4EE410AF1EE2D
:10D1200010FA39DDFFE7002028B9FFE7039803F084
:10D130000DF958B92FE0039809F042FA41EC100BB1
:10D1400051EC100B03F0D6F828B3FFE79DED040A6D
:10D150009DED021A30EE010AB0EEC00A0E9840684A
:10D1600090ED051AB4EE410AF1EE10FA12DCFFE779
:10D170009DED030AB0EEC00A0E98406890ED041AC7
:10D18000B4EE410AF1EE10FA04DCFFE703980E99C1
:10D19000C860FFE7FFE7FFE79DED021A9DED040A77
:10D1A00030EE010A8DED040A002028B9FFE704984B
:10D1B00003F0CCF858B925E0049809F001FA41ECE5
:10D1C000100B51EC100B03F095F8D8B1FFE70E9857
:10D1D000406890ED050A9FED0F1AB4EE410AF1EE9A
:10D1E00010FA0BDDFFE79DED040A0E984068D0EDC4
:10D1F000050AF4F7E9FC8DED040AFFE704980E999F
:10D200008861FFE70E9880690F90FFE79DED0F0A98
:10D2100010B080BDBD37863580B586B004908DF8DE
:10D220000F108DED020A0192049820B9FFE7FF204C
:10D230008DF81700B7E0002030B9FFE7019840688B
:10D2400003F084F880B90BE00198406809F0B8F960
:10D2500041EC100B51EC100B03F04CF820B9FFE738
:10D26000FF208DF817009EE0002030B9FFE70198FD
:10D27000806803F06BF880B90BE00198806809F0D2
:10D280009FF941EC100B51EC100B03F033F820B96F
:10D29000FFE7FF208DF8170085E0002030B9FFE799
:10D2A0000198C06803F052F880B90BE00198C0689B
:10D2B00009F086F941EC100B51EC100B03F01AF851
:10D2C00020B9FFE7FF208DF817006CE0002030B98F
:10D2D000FFE70198006903F039F880B90BE0019885
:10D2E000006909F06DF941EC100B51EC100B03F0E3
:10D2F00001F820B9FFE7FF208DF8170053E0002068
:10D3000030B9FFE70198406903F020F880B90BE0DD
:10D310000198406909F054F941EC100B51EC100BE5
:10D3200002F0E8FF20B9FFE7FF208DF817003AE090
:10D330000198049948609DED021AB7EE000A80EE4C
:10D34000010A8DED000A002028B9FFE7009802F0DD
:10D35000FDFF58B90EE0009809F032F941EC100BCE
:10D3600051EC100B02F0C6FF20B1FFE700980499C2
:10D37000886003E0FF208DF8170014E0049901F1A4
:10D380001C009DED020A4968D1ED060AFDF7AAFFCF
:10D390009DF80F0004990870049800F009F8002027
:10D3A0008DF81700FFE79DF9170006B080BD00005B
:10D3B00080B584B00290029820B9FFE7FF208DF875
:10D3C0000F0013E0029900200190C86002990861E3
:10D3D000029948610299886102981C309FED050A04
:10D3E000FEF71EF801988DF80F00FFE79DF90F007A
:10D3F00004B080BD0000000082B00090009820B909
:10D40000FFE7FF208DF8070005E000990020C860C5
:10D410008DF80700FFE79DF9070002B07047000094
:10D42000EFF30980BFF36F8F154B1A681EF0100FD2
:10D4300008BF20ED108A20E9F04F10602DE90900A7
:10D440004FF0500080F31188BFF34F8FBFF36F8F01
:10D4500005F0F4FC4FF0000080F31188BDE80900EE
:10D4600019680868B0E8F04F1EF0100F08BFB0EC64
:10D47000108A80F30988BFF36F8F704700BF00BF29
:10D480002412002080B582B001900198806B00903A
:10D4900000980168486820F0030048600099486DD2
:10D4A00040F0100048650099012081F85100009873
:10D4B000FBF7EAFB02B080BD80B582B00190019815
:10D4C000806B00900098FBF76DFF02B080BD0000FC
:10D4D00080B582B001900198806B00900098FCF7B5
:10D4E00093FC02B080BD000080B582B0019001982D
:10D4F000806B00900098FCF7DBFC02B080BD000060
:10D5000080B584B003900398806B0290FAF7D2FB49
:10D51000019003980068006800F48070B0F5807F87
:10D5200039D0FFE702980168486820F02000486081
:10D530000298806868B9FFE702984068B0F5827F7A
:10D5400007D1FFE702980168486820F003004860AF
:10D5500006E002980168486820F001004860FFE793
:10D560000298019A642100F0B5F820B1FFE7029912
:10D5700020204865FFE702990020C8870299012012
:10D5800081F851000298406D20B1FFE70298FBF747
:10D590007BFB04E0FFE70298FBF7DAFEFFE704B04D
:10D5A00080BD000080B584B003900398806B02902A
:10D5B000FAF780FB019003980068006800F480701F
:10D5C000B0F5807F3BD0FFE702980168486820F003
:10D5D0002000486002980168486820F00200486016
:10D5E0000298019A642100F0E7F830B1FFE7029950
:10D5F000486D40F020004865FFE70298806870B9E8
:10D60000FFE7FFE70020009002980068C0680090E4
:10D6100002980068806800900098FFE7FFE7029991
:10D620000020C8860299012081F851000298406DBF
:10D6300020B1FFE70298FBF727FB04E0FFE7029821
:10D64000FCF7BEFBFFE704B080BD000080B584B0EE
:10D6500003900398806B0290FAF72CFB01900398DB
:10D660000068006800F48070B0F5807F2BD0FFE781
:10D6700002980168486820F0200048600298019AEA
:10D68000642100F099F830B1FFE70299486D40F04D
:10D6900020004865FFE702980168486820F0030011
:10D6A000486002990020C8860299C8870299012023
:10D6B00081F851000298406D20B1FFE70298FBF716
:10D6C000E3FA04E0FFE70298FCF7C8FBFFE704B0C9
:10D6D00080BD000080B586B004900391029204984A
:10D6E0004068B0F5827F13D1FFE704988068B0F5F9
:10D6F000004F06D0FFE704988068B0F5806F07D12F
:10D70000FFE704980168086820F040000860FFE720
:10D7100004984068B0F5827F31D1FFE704988068B3
:10D72000B0F5806F15D0FFE70498039B02996A4615
:10D7300011608021002200F0BDF848B1FFE7049994
:10D74000486D40F02000486503208DF817002FE059
:10D7500014E00498039B02996A461160012100229B
:10D7600000F0A8F848B1FFE70499486D40F02000A8
:10D77000486503208DF817001AE0FFE714E00498CD
:10D78000039B02996A4611600121002200F092F881
:10D7900048B1FFE70499486D40F020004865032038
:10D7A0008DF8170004E0FFE700208DF81700FFE771
:10D7B0009DF8170006B080BD80B586B00490039137
:10D7C00002920498039B02996A4611600221012289
:10D7D00000F070F848B1FFE70499486D40F0200070
:10D7E000486503208DF8170048E040F20000C2F2BF
:10D7F000000000684AF6AB21CAF6AA21A0FB01107E
:10D8000000094DF68361C4F21B31A0FB0110800CAE
:10D810004FF47A714843019004984068B0F5827FD4
:10D8200015D1FFE70498039B02996A461160802195
:10D83000002200F03FF848B1FFE70499486D40F03E
:10D840002000486503208DF8170017E012E0FFE77D
:10D85000019808B9FFE70CE0019801380190FFE753
:10D86000049800688068C1B20020B0EBD11FEFD1EE
:10D87000FFE7FFE700208DF81700FFE79DF817008E
:10D8800006B080BD82B000900098006843F20001AD
:10D89000C4F20101884204D1FFE700208DF807009F
:10D8A00003E002208DF80700FFE79DF8070002B0B3
:10D8B0007047000080B58AB0DDF830C0089007914D
:10D8C0008DF81B20059305980190FAF7F3F90246AD
:10D8D00001980C99891A08440390FAF7EBF9029021
:10D8E000039840F20001C2F200010968C1F3CB3194
:10D8F00048430490FFE7089800688068079908404B
:10D90000401AB0FA80F040099DF81B1088425FD0A1
:10D91000FFE705980130002859D0FFE7FAF7CAF968
:10D920000299401A0399884204D2FFE7039800281D
:10D9300042D1FFE708980168486820F0E00048609D
:10D9400008984068B0F5827F13D1FFE70898806897
:10D95000B0F5004F06D0FFE708988068B0F5806FFB
:10D9600007D1FFE708980168086820F040000860C8
:10D97000FFE70898806AB0F5005F0FD1FFE7FFE787
:10D9800008980168086820F4005008600898016849
:10D99000086840F400500860FFE7FFE7089901209D
:10D9A00081F85100FFE70899002081F85000FFE757
:10D9B00003208DF827000FE0049818B9FFE7002036
:10D9C000039003E0049801380490FFE7FFE792E733
:10D9D00000208DF82700FFE79DF827000AB080BDE2
:10D9E000074B19680868B0E8F04F80F30988BFF367
:10D9F0006F8F4FF0000080F31188704700BF00BFA9
:10DA00002412002080B56FF00400002102F03CFDDC
:10DA100080BD000084B003900291039890ED000A4D
:10DA2000029890ED001A30EE010A8DED010A9DED8D
:10DA3000010AB7EE001AB4EE410AF1EE10FA1BDD4E
:10DA4000FFE79DED011AB7EE000A80EE010A8DEDA9
:10DA5000000A9DED001A039890ED000A20EE010ADD
:10DA600080ED000A9DED001A029890ED000A20EE6C
:10DA7000010A80ED000AFFE704B0704780B586B068
:10DA800004900391049828B1FFE70498B0F82001AE
:10DA900020B9FFE7FF208DF817004FE0049890EDC4
:10DAA000010A90ED471A30EE410A8DED020A049802
:10DAB000D0ED340A90ED650A9FED221AF6F7DCFAF4
:10DAC0008DED010A9DED020A0498406990ED042A4B
:10DAD000B7EE001A81EE021AB4EE410AF1EE10FA26
:10DAE00028DBFFE70398C078C00718B3FFE79DED78
:10DAF000010AB7EE001AB4EE410AF1EE10FA19DC91
:10DB0000FFE704994868C1F81C01049901F5CA703F
:10DB1000496991ED030AB8EE400ADFED0A0A80EE8A
:10DB2000800AF6F767FA0499B1F820010138A1F8E4
:10DB30002001FFE700208DF81700FFE79DF917008F
:10DB400006B080BDDB0FC94084B002908DED010AA4
:10DB5000029820B9FFE7FF208DF80F001DE0029822
:10DB6000406900780146009120B1FFE70098012844
:10DB700008D00EE0029944F20000C4F29C50C1F8B3
:10DB8000900106E002990020C4F2FA30C1F8900139
:10DB9000FFE700208DF80F00FFE79DF90F0004B0AC
:10DBA0007047000080B586B004900391049818B1C6
:10DBB000FFE7039820B9FFE7FF208DF817003BE04F
:10DBC000F5F7CAFB08F051FD00EE100A9FED1C1A94
:10DBD0008DED011A80EE010A049880ED010AF5F737
:10DBE000BBFB049A02929368D268C01A914108F074
:10DBF0003CFD9DED011A0146029800EE101A80EEE0
:10DC0000010A80ED040AF5F7A7FB0A460499CA60E9
:10DC1000886003980078049900F001000870049867
:10DC20009FED080AFFF790FF0498039900F0E2F8CF
:10DC300000208DF81700FFE79DF9170006B080BDA2
:10DC4000002474490000694380B58AB008900791A8
:10DC50008DED060A089858B1FFE7079840B1FFE735
:10DC60009DED060AB5EE400AF1EE10FA04DCFFE77E
:10DC7000FF208DF82700B9E0079840688DF817005D
:10DC8000079808994861F4F751FC00200490FFE7D9
:10DC900004989DF81710884248DAFFE7079804991E
:10DCA00001EB810100EB41003030FEF761F908988B
:10DCB0000499C1EB011100EB810000F5CC709DEDE2
:10DCC000060A079901F1740201210391FFF7A4FAF2
:10DCD00003990898049AC2EB021200EB820000F547
:10DCE00040709DED060A079A9432FFF795FA08995D
:10DCF000049801EB401000F59C609DED060A49690F
:10DD0000D1ED4D0AFDF7EEFA0899049801EB4010A9
:10DD100000F5B4609DED060A4969D1ED4E0AFDF7A4
:10DD2000E1FAFFE7049801300490B1E707986C30FE
:10DD3000FEF71EF90898406990F8700001460291BC
:10DD4000E0B1FFE7029801282FD1FFE7089800F51E
:10DD50008D609DED060A079901F1F4020121019100
:10DD6000FFF75AFA0199089800F2A4409DED060ABF
:10DD7000079A02F58A72FFF74FFA1AE0089800F541
:10DD80008D609DED060A079901F1B4020121009111
:10DD9000FFF742FA0099089800F2A4409DED060AA8
:10DDA000079AD432FFF738FA03E0FC208DF82700F9
:10DDB0001CE0089901F5CC609DED060A4969D1ED9A
:10DDC0004F0AFDF78FFA089901F5D0609DED060A1C
:10DDD0004969D1ED500AFDF785FA08990020C1F88C
:10DDE0002001C1F81C018DF82700FFE79DF92700ED
:10DDF0000AB080BD80B584B002900191029820B92C
:10DE0000FFE7FF208DF80F00C2E00298406990F80C
:10DE10002400C007002800F0AB80FFE7029890F8CC
:10DE2000180101460091032800F29C800099DFE868
:10DE300001F002205471029890ED240A9FED581AC7
:10DE400080EE010A406990ED0A1AB4EE410AF1EE43
:10DE500010FA09DDFFE70299012081F81801029903
:10DE60004868C1F81401FFE70298019900F090F9A1
:10DE70007DE0029890ED240A9FED491A80EE010A98
:10DE8000406990ED0A1AB4EE410AF1EE10FA05DA93
:10DE9000FFE70299002081F8180168E0029890EDF0
:10DEA000010A90ED451A30EE410A406990ED0B1AD7
:10DEB000B4EE410AF1EE10FA09DBFFE70299012006
:10DEC00081F810010299022081F818014FE0FFE764
:10DED0000298019900F05CF949E002990020A1F84C
:10DEE0002001029890ED340A416991ED031AB8EED1
:10DEF000412A9FED291A81EE021A30EE010A80EDC7
:10DF0000650A0299032081F8180102994868C1F84E
:10DF10001401FFE70298019900F03AF9029890ED98
:10DF2000010A90ED451A30EE410A9FED1C1AB4EE3D
:10DF3000410AF1EE10FA14DBFFE7029890ED240A93
:10DF40009FED171A80EE010AB3EE041AB4EE410AEF
:10DF5000F1EE10FA05DAFFE70299002081F81801C6
:10DF6000FFE704E00299002081F81801FFE70BE0C9
:10DF70000299002081F81801029981F81001029895
:10DF8000019900F005F9FFE700208DF80F00FFE789
:10DF90009DF90F0004B080BDDB0FC9C09A99993E6E
:10DFA00000007A4480B586B00490049820B9FFE759
:10DFB000FF208DF817005AE00498406940688DF8FA
:10DFC0000F0000200290FFE702989DF80F10884292
:10DFD0002FDAFFE704980299C1EB011100EB8100F1
:10DFE00000F5CC70FFF7E4F904980299C1EB011138
:10DFF00000EB810000F54070FFF7DAF90498029910
:10E0000000EB411000F59C609FED1B0A8DED010AAD
:10E01000FDF706FA9DED010A0498029900EB411004
:10E0200000F5B460FDF7FCF9FFE7029801300290BB
:10E03000CAE7049800F58D60FFF7BAF9049800F27A
:10E04000A440FFF7B5F9049800F5CC609FED0A0AEB
:10E050008DED000AFDF7E4F99DED000A049800F546
:10E06000D060FDF7DDF900208DF81700FFE79DF97E
:10E07000170006B080BD00BF0000000080B584B06E
:10E080000290029820B9FFE7FF208DF80F0034E0DE
:10E090000298406940688DF8070000200090FFE773
:10E0A00000989DF80710884219DAFFE70298009956
:10E0B000C1EB011100EB810000F5CC70FFF79CF97A
:10E0C00002980099C1EB011100EB810000F540704E
:10E0D000FFF792F9FFE7009801300090E0E702981F
:10E0E00000F58D60FFF788F9029800F2A440FFF771
:10E0F00083F900208DF80F00FFE79DF90F0004B0B1
:10E1000080BD000084B00290029820B9FFE7FF2094
:10E110008DF80F0038E00298406940688DF80700DC
:10E1200000200090FFE700989DF8071088421EDA53
:10E13000FFE70298009900EB81010020C1F824015B
:10E140000299009A01EB8201C1F83C010299009A00
:10E1500001EB8201C1F854010299009A01EB82019E
:10E16000C1F86C01FFE7009801300090DBE70299ED
:10E170000020C1F884010299C1F888010299C1F810
:10E180008C018DF80F00FFE79DF90F0004B0704778
:10E1900080B594B012901191129818B1FFE71198C0
:10E1A00020B9FFE7FF208DF84F0002E31298406985
:10E1B00040688DF8430012980078C007F0B9FFE777
:10E1C00000200F90FFE70F989DF8431088420FDA68
:10E1D000FFE7129840690F9901EB810100EB4100C4
:10E1E0003030FDF755FFFFE70F9801300F90EAE759
:10E1F000129840696C30FDF74BFFB7E21298007E31
:10E200000146079150B1FFE70798012800F0AA8066
:10E21000FFE70798022800F0C281A2E200200E90DA
:10E22000FFE70E989DF84310884251DAFFE71298F5
:10E230000E99C1EB011100EB810000F5CC70FFF7E6
:10E24000DBF812990E9AC2EB021001EB800000F588
:10E25000CC7001EB8202D2ED3C0AD1ED041A9FEDA5
:10E26000D71AB0EE410AFEF75FFE12980E9900EB46
:10E27000810080ED490A12980E9900EB8101D1F8D6
:10E280002401C1F8540112990E9A01EB421000F5D5
:10E29000B46001EB820191ED550AFCF7C7FF1298BB
:10E2A0000E9900EB810080ED5B0A129948690E9A85
:10E2B00002EB820300EB4300303001EB820191ED71
:10E2C0005B0AFDF7F1FEFFE70E9801300E90A8E71C
:10E2D000129901F58D6040F28452C2F2000292ED73
:10E2E000000AD1ED041AD1ED340A9FEDB41A8DED78
:10E2F000061AFEF719FE9DED061A129880ED610AC6
:10E30000129901F2A440D1ED041AD1ED430A91ED26
:10E31000610AFEF709FE129880ED620A129901F572
:10E32000D06091ED620AFCF781FF129880ED630ADC
:10E33000129948696C3091ED630AFDF7B5FE1198AA
:10E340008078C00768B1FFE71298FFF72BFE12989C
:10E35000FFF794FE1298FFF7D5FE12990120087678
:10E36000FFE702E200200D90FFE70D989DF84310B3
:10E37000884280F29680FFE71298406990F8380052
:10E3800001388DF83300129841699DF8332001EB74
:10E39000820191ED070A90ED641A20EE010A9FEDCB
:10E3A000881A80EE010A8DED0B0A129890ED640A2E
:10E3B00080EE010A40F2D050C2F2000080ED000A67
:10E3C00012990D9AC2EB021001EB800000F5CC709F
:10E3D0009DED0B0A01EB8202D2ED3C0AD1ED041A4D
:10E3E0009FED761A8DED051AFEF79EFD9DED051A3F
:10E3F00012980D9900EB810080ED490A129A0D994F
:10E40000C1EB011002EB800000F5407002EB8101CE
:10E41000D2ED041A92ED420AD1ED3C0AFEF784FDDA
:10E4200012980D9900EB810080ED4F0A12980D991A
:10E4300000EB810101F5927001F59E71FFF7EAFA98
:10E4400012980D9900EB810090ED490A90ED4F1A5A
:10E4500030EE010A80ED550A12990D9A01EB421037
:10E4600000F5B46001EB820191ED550AFCF7DEFE88
:10E4700012980D9900EB810080ED5B0A12994869B2
:10E480000D9A02EB820300EB4300303001EB820176
:10E4900091ED5B0AFDF708FEFFE70D9801300D9046
:10E4A00063E7129901F58D6040F28452C2F20002D6
:10E4B00092ED000AD1ED041AD1ED340A9FEDBF1A96
:10E4C0008DED041AFEF730FD9DED041A129880EDD3
:10E4D000610A129901F2A440D1ED041AD1ED430A68
:10E4E00091ED610AFEF720FD129880ED620A129903
:10E4F00001F5D06091ED620AFCF798FE129880ED6C
:10E50000630A129948696C3091ED630AFDF7CCFDFE
:10E5100011988078C00750B9FFE71298FFF742FDC5
:10E520001298FFF7EFFD12990020087636E041F2CD
:10E530002310C2F200000078C00770BBFFE71198FB
:10E54000C078C00748B3FFE71299022008761298F6
:10E55000407E01460391012808D0FFE70398022876
:10E5600009D0FFE7039803280BD010E0129901208F
:10E57000A1F8200110E0129948694069A1F8200132
:10E580000AE0129941F60A20A1F8200104E012994C
:10E590000020A1F82001FFE7FFE7FFE7E5E0129880
:10E5A0001199FFF76BFA00200A90FFE70A989DF88F
:10E5B0004310884280F2908004E000BF0000000019
:10E5C00000C0DA451298406990F8380001388DF89B
:10E5D0002700129841699DF8272001EB820191EDF7
:10E5E000070A90ED641A20EE010A9FED751A80EE7D
:10E5F000010A8DED080A12990A9AC2EB021001EB8A
:10E60000800000F5CC709DED080A01EB8202D2ED8E
:10E610003C0AD1ED041A9FED691A8DED021AFEF73E
:10E6200083FC9DED021A12980A9900EB810080ED9F
:10E63000490A129A0A99C1EB011002EB800000F519
:10E64000407002EB8101D2ED041A92ED420AD1ED45
:10E650003C0AFEF769FC12980A9900EB810080EDF4
:10E660004F0A12980A9900EB810101F5927001F5A9
:10E670009E71FFF7CFF912980A9900EB810090ED97
:10E68000490A90ED4F1A30EE010A80ED550A1299B1
:10E690000A9A01EB421000F5B46001EB820191EDA2
:10E6A000550AFCF7C3FD12980A9900EB810080ED32
:10E6B0005B0A129948690A9A02EB820300EB430055
:10E6C000303001EB820191ED5B0AFDF7EDFCFFE7D5
:10E6D0000A9801300A9069E7129901F58D60D1ED31
:10E6E000041AD1ED340A91ED650A9FED341A8DEDCF
:10E6F000011AFEF719FC9DED011A129880ED610ACE
:10E70000129901F2A440D1ED041AD1ED430A91ED22
:10E71000610AFEF709FC129880ED620A129901F570
:10E72000D06091ED620AFCF781FD129880ED630ADA
:10E73000129948696C3091ED630AFDF7B5FC1198A8
:10E74000C078C00760B9FFE71299012008761298D7
:10E75000D0F8D00040F28451C2F200010860FFE717
:10E7600003E0129900200876FFE7FFE7129840695E
:10E770003030FDF75FFA129840694068052806D3EB
:10E78000FFE7129840695830FDF754FAFFE71298F6
:10E7900040696C30FDF74EFA1198C07800F0010026
:10E7A00041F22311C2F20001087000208DF84F00E1
:10E7B000FFE79DF94F0014B080BD00BF00000000CE
:10E7C00000C0DA4583B001908DF80310019820B99C
:10E7D000FFE7FF208DF80B000AE09DF80300019988
:10E7E000487601990020A1F820018DF80B00FFE781
:10E7F0009DF90B0003B0704780B588B0069006986D
:10E8000020B9FFE7FF208DF81F0041E100200590AF
:10E810000699496949688DF813100390FFE703983A
:10E820009DF81310884280F28B80FFE706984069BC
:10E83000039901EB810100EB41003030FDF7C2FC90
:10E8400006984069039901EB810100EB41003030EB
:10E85000FDF72AFB02900298A0B1FFE70698039902
:10E8600000EB0111DDF808C0DCF82C00DCF83020EA
:10E87000DCF83430DCF838C0C1F82CC08B624A6256
:10E880000862FFE70699039A01EB421000F59C60CD
:10E8900001EB021191ED090AFCF7C8FC06980399F7
:10E8A00000EB810080ED350A0698039900EB8100AA
:10E8B00090ED350A9FED7B1A80EE010A80ED3C0A4F
:10E8C0000698039900EB810090ED3C0AB7EE001A20
:10E8D000B4EE410AF1EE10FA09DDFFE7069803995C
:10E8E00000EB81014FF07E50C1F8F000FFE7069881
:10E8F000039900EB810090ED3C0ABFEE001AB4EEE4
:10E90000410AF1EE10FA0ADAFFE70698039900EBE4
:10E9100081010020CBF68070C1F8F000FFE7069877
:10E92000039900EB810090ED3C1A9DED050A30EE55
:10E93000010A8DED050AFFE70398013003906EE7A9
:10E940009DED050A9DF8130001EE100AB8EEC11AFC
:10E9500080EE010A069880ED420A069840696C3004
:10E96000FDF730FC069800F18001019140696C30A0
:10E97000FDF79AFA014601985022F1F78CFD0698AE
:10E98000416991ED020A90ED321A20EE010A80ED04
:10E99000340AFFE7069890ED340AB5EE400AF1EE2E
:10E9A00010FA0ADAFFE7069890ED340A9FED3A1A5A
:10E9B00030EE010A80ED340AECE7FFE7069890EDAF
:10E9C000340A9FED351AB4EE410AF1EE10FA0ADB73
:10E9D000FFE7069890ED340A9FED311A30EE010AF8
:10E9E00080ED340AEAE7069890F8A800C00750B115
:10E9F000FFE7069890ED341A9FED270A30EE410AA2
:10EA000080ED340AFFE7069901F5CC6091ED230A09
:10EA1000FCF70CFC069880ED3B0A069890ED230A63
:10EA20009FED1E1A80EE010A80ED430A069890EDD4
:10EA3000430AB7EE001AB4EE410AF1EE10FA06DD11
:10EA4000FFE706994FF07E50C1F80C01FFE70698EA
:10EA500090ED430ABFEE001AB4EE410AF1EE10FA4F
:10EA600007DAFFE706990020CBF68070C1F80C01A9
:10EA7000FFE7069890ED090A90ED0D1A30EE410A75
:10EA800000F5D46080ED000A00208DF81F00FFE73C
:10EA90009DF91F0008B080BDDB0FC94000409C45B8
:10EAA000DB0FC9C000C0DA4580B582B0019002F02A
:10EAB000D7FA02F08BFB02B080BD000080B582B0B7
:10EAC000009000980138B0F1807F03D3FFE7012068
:10EAD000019019E0009801384EF21401CEF20001C5
:10EAE00008604FF0FF300F2101F0ACFC4EF218012E
:10EAF000CEF20001002008604EF21002CEF20002B9
:10EB0000072111600190FFE7019802B080BD00006D
:10EB100080B5F9F7C5FA05F085FB012803D0FFE7BA
:10EB200004F09CFAFFE780BD80B594B008A83021BE
:10EB3000F1F7EBFC002007900690059004900390FD
:10EB4000FFE70020029043F64000C4F20200016893
:10EB500041F080510160006800F0805002900298FE
:10EB6000FFE7FFE70020019047F20000C4F2000039
:10EB7000016841F480410160006800F48040019028
:10EB80000198FFE7012008904FF48030099002209F
:10EB90000E904FF480010F9106211091A821119140
:10EBA00012900420139008A8F9F70EFD18B1FFE7A2
:10EBB000F6F70CFEFFE70F200390022004900020E0
:10EBC00005904FF4A05006904FF48050079003A892
:10EBD0000521F9F729FB18B1FFE7F6F7F7FDFFE785
:10EBE00014B080BD4EF68851CEF20001086840F4A2
:10EBF000700008607047000083B002900191029895
:10EC00000068009002980021C4F20101884225D0DA
:10EC1000FFE70298B0F1804F20D0FFE7029840F262
:10EC20000041C4F20001884218D0FFE7029840F684
:10EC30000001C4F20001884210D0FFE7029840F6BC
:10EC40000041C4F20001884208D0FFE7029840F278
:10EC50000041C4F2010188420AD1FFE7009820F088
:10EC60007000009001984168009808430090FFE709
:10EC700002980021C4F20101884255D0FFE70298B2
:10EC8000B0F1804F50D0FFE7029840F20041C4F24B
:10EC90000001884248D0FFE7029840F60001C4F224
:10ECA0000001884240D0FFE7029840F60041C4F2DC
:10ECB0000001884238D0FFE7029840F20041C4F2D8
:10ECC0000101884230D0FFE7029844F20001C4F20B
:10ECD0000101884228D0FFE7029844F20041C4F2C3
:10ECE0000101884220D0FFE7029844F60001C4F2F7
:10ECF0000101884218D0FFE7029841F60001C4F2F2
:10ED00000001884210D0FFE7029841F60041C4F2AA
:10ED10000001884208D0FFE7029842F20001C4F2E5
:10ED2000000188420AD1FFE7009820F4407000906B
:10ED30000198C168009808430090FFE7009820F010
:10ED40008000019949690843009001988068029900
:10ED5000C862019800680299886202980021C4F292
:10ED60000101884208D0FFE7029840F20041C4F256
:10ED70000101884205D1FFE7019800690299086303
:10ED8000FFE70299086840F004000860029901203A
:10ED9000486100980299086003B0704784B00390FE
:10EDA00002910192029800F01F010120884000901A
:10EDB000009A0399086A904308620198029901F049
:10EDC0001F0100FA01F20399086A1043086204B0B7
:10EDD0007047000085B0049003910292019304985B
:10EDE00080680090009820F47F400090039802997A
:10EDF000019A41EA022101430098084300900098DB
:10EE00000499886005B0704783B002900191029820
:10EE100080680090009820F07000009001980099A0
:10EE2000084340F00700009000980299886003B002
:10EE30007047000085B0049003910498006A019027
:10EE40000499086A20F00100086204984068009064
:10EE5000049880690290029820F070000290029855
:10EE600020F0030002900398016802980843029082
:10EE7000019820F0020001900398816801980843EE
:10EE8000019004980021C4F20101884208D0FFE7F4
:10EE9000049840F20041C4F2010188420ED1FFE71C
:10EEA000019820F0080001900398C1680198084378
:10EEB0000190019820F004000190FFE704980021E0
:10EEC000C4F20101884208D0FFE7049840F20041F3
:10EED000C4F20101884213D1FFE7009820F480704A
:10EEE0000090009820F40070009003984169009809
:10EEF0000843009003988169009808430090FFE759
:10EF000000980499486002980499886103984068C1
:10EF10000499486301980499086205B0704700009D
:10EF200085B0049003910498006A01900499086ADE
:10EF300020F01000086204984068009004988069EE
:10EF40000290029820F4E0400290029820F4407071
:10EF5000029003980168029840EA0120029001980B
:10EF600020F02000019003988168019840EA011088
:10EF7000019004980021C4F20101884208D0FFE703
:10EF8000049840F20041C4F2010188420FD1FFE72A
:10EF9000019820F0800001900398C168019840EA30
:10EFA00001100190019820F040000190FFE70498C3
:10EFB0000021C4F20101884208D0FFE7049840F222
:10EFC0000041C4F20101884215D1FFE7009820F406
:10EFD00080600090009820F40060009003984169E0
:10EFE000009840EA8100009003988169009840EA07
:10EFF00081000090FFE70098049948600298049906
:10F0000088610398406804998863019804990862AC
:10F0100005B0704785B0049003910498006A019090
:10F020000499086A20F4807008620498406800908F
:10F030000498C0690290029820F070000290029833
:10F0400020F00300029003980168029808430290A0
:10F05000019820F40070019003988168019840EABB
:10F060000120019004980021C4F20101884208D0D7
:10F07000FFE7049840F20041C4F2010188420FD139
:10F08000FFE7019820F4006001900398C16801989F
:10F0900040EA01200190019820F480600190FFE790
:10F0A00004980021C4F20101884208D0FFE70498C7
:10F0B00040F20041C4F20101884215D1FFE70098F7
:10F0C00020F480500090009820F4005000900398A5
:10F0D0004169009840EA0110009003988169009806
:10F0E00040EA01100090FFE70098049948600298F8
:10F0F0000499C861039840680499C8630198049909
:10F10000086205B07047000085B004900391049830
:10F11000006A01900499086A20F4805008620498FB
:10F12000406800900498C0690290029820F4E04082
:10F130000290029820F440700290039801680298AF
:10F1400040EA01200290019820F4005001900398B9
:10F150008168019840EA0130019004980021C4F2CE
:10F160000101884208D0FFE7049840F20041C4F250
:10F17000010188420BD1FFE7009820F48040009005
:10F1800003984169009840EA81100090FFE70098D9
:10F190000499486002980499C861039840680499EA
:10F1A000086401980499086205B0704785B004901E
:10F1B000039102920498006A00900499086A20F072
:10F1C00001000862049880690190019820F0F00025
:10F1D00001900299019840EA01100190009820F0F6
:10F1E0000A00009003990098084300900198049940
:10F1F000886100980499086205B0704785B0049052
:10F20000039102920498006A00900499086A20F021
:10F2100010000862049880690190019820F4704001
:10F2200001900299019840EA01300190009820F085
:10F23000A00000900399009840EA01100090019806
:10F240000499886100980499086205B0704700002D
:10F2500080B586B0059001F00FFB4FF6A120C0F6F7
:10F26000000046F6BC12C0F601020021029101F036
:10F27000FFFE029941F69452C2F20002049210601D
:10F280004FF2A130C0F6000046F6C002C0F60102FF
:10F2900001F0EEFE0299049A50604FF24160C0F610
:10F2A000000046F6E402C0F6010201F0E1FE029918
:10F2B000049A90604FF61900C0F6000046F62C1232
:10F2C000C0F6010201F0D4FE0299049AD0604FF614
:10F2D000F900C0F6000046F65012C0F6010201F037
:10F2E000C7FE0299049A10614FF6F110C0F60000B3
:10F2F00046F67412C0F6010201F0BAFE0299049AB1
:10F3000050614FF2F160C0F6000046F60812C0F6F8
:10F31000010201F0ADFE029A049988610220039077
:10F320000A2101F097FB029A0499C861032000901A
:10F330002C2101F08FFB029A049B014600989963EF
:10F34000282101F087FB029A049B01460398596229
:10F350000421019101F07EFB029A049B014603986F
:10F360009962182101F076FB029A049B01460398EA
:10F37000D9620C2101F06EFB0199029ADDF810C0F0
:10F3800003460398CCF8303001F064FB04994863DD
:10F3900001F0C8FA01F064FE01F018FF06B080BD6C
:10F3A00080B58CB00B9001F03FFA06F086FE41EC80
:10F3B000100B9FED9D1B53EC112B51EC100B06F025
:10F3C000B9FC41EC100B51EC100B06F049FE0A9011
:10F3D0000020089001F0A4F901F012FA099040F21F
:10F3E0003060C2F20000079040F27801C2F20001E2
:10F3F000F2F76AFC0798F2F73FFC40F6E030C2F201
:10F40000000041F22411C2F20001F1F79FF90798C0
:10F41000F2F732FC0899B0EE401AB7EE000A80EE1F
:10F42000010A41F2E400C2F2000046F61422C0F6DE
:10F430000102FDF7F1FE0120F3F74CFE089842F2BD
:10F440009D31C0F60101F3F72DFD0898F3F7D8FCC4
:10F45000FFE70A99099808440990F2F725FEF2F7A8
:10F46000F3FBF2F701FCF2F719FCF2F725FC01F0CF
:10F4700003FA40F23060C2F200000690F2F7E8FCB6
:10F480000698F2F75FFD40F27860C2F20000007863
:10F49000012865D1FFE740F23061C2F2000191ED31
:10F4A000071A40F63040C2F2000090ED000A30EE3C
:10F4B000010A80ED000A91ED081A90ED010A30EE84
:10F4C000010A80ED010A91ED091A90ED020A30EE71
:10F4D000010A80ED020A40F27660C2F20000018863
:10F4E00001310180008841F28831884237DBFFE733
:10F4F00040F63040C2F2000090ED000A9FED4C1A39
:10F5000080EE010A40F27801C2F2000181ED000AAA
:10F5100090ED010A80EE010A81ED010A90ED020AE8
:10F5200080EE010A81ED020A40F27862C2F2000226
:10F530000020107040F23060C2F200000590F2F737
:10F54000C3FB0598F2F798FB40F6E030C2F20000EA
:10F5500041F22411C2F20001F1F7F8F8FFE7FFE7EA
:10F5600040F27860C2F20000007801281BD0FFE76B
:10F5700040F23060C2F2000000F1100100F11C0204
:10F5800040F6E030C2F20000049041F22413C2F2CF
:10F590000003F1F727FA049940F63020C2F2000088
:10F5A000F1F726F8FFE701F0BDF940F63021C2F28D
:10F5B000000108684A688B6840F61841C2F20001F1
:10F5C00001914B610A61C86040F23063C2F20003EE
:10F5D0000393D8691A6A5B6A8B604A60086041F6D7
:10F5E0009450C2F200000290C06A01F015FB01992C
:10F5F0000298C06A00231A4601F0ACFA0398D0EDD5
:10F600000A0A41F2E400C2F200009FED0A0ADFEDAF
:10F610000A1AB0EE611AFDF787FC0120F3F7BAFC75
:10F62000099801F097F814E70000000000407F40BF
:10F6300000409C4500002042000000000000000047
:10F6400080B586B0059001F0EFF806F036FD41EC8C
:10F65000100B9FED231B53EC112B51EC100B06F0FC
:10F6600069FB41EC100B51EC100B06F0F9FC049017
:10F67000002001F055F801F0C3F803900420F3F7DF
:10F680004BFD0220F3F748FD032001909FED160A81
:10F69000F3F780FC0198F3F71DFDFFE70499039849
:10F6A000084403909DED030AB8EE400A9FED0F1A3F
:10F6B00020EE010A05F032FFB7EE001A30EE010A23
:10F6C000B6EE001A20EE010A8DED020A9DED020A47
:10F6D0000320F3F75FFC039801F03CF8DEE700BF7E
:10F6E000000000000000594000000000A69B443BC1
:10F6F00010B58AB0099001F097F806F0DEFC41ECF5
:10F70000100B9FED431B53EC112B51EC100B06F02B
:10F7100011FB41EC100B51EC100B06F0A1FC089012
:10F72000002000F0FDFF01F06BF80790F5F7DCF921
:10F7300000F51B7140F68010C2F20000F4F70EFED7
:10F74000FFE7089907980844079041F69450C2F2E1
:10F7500000000690806B40F20061C2F200010023BD
:10F7600005931A4601F016F940F68010C2F2000027
:10F770000190F4F71BFD019A0698D2F8651040F647
:10F780002823C2F2000303931960516CD2F848C0D9
:10F79000D2F84CE0146D40F60C23C2F2000304933F
:10F7A000DC60C3F808E0C3F804C01960916DD36D44
:10F7B000D2F860C040F61C22C2F200020292C2F8E7
:10F7C00008C053601160006B01F026FA0299059B96
:10F7D0000698006B1A4601F0BDF90698406B01F0DF
:10F7E0001BFA0399059B0698406B1A4601F0B2F983
:10F7F0000698406A01F010FA0499059B0698406A41
:10F800001A4601F0A7F9079800F0A4FF99E700BF96
:10F810000000000000407F4080B58AB0099001F0F0
:10F8200003F806F04AFC41EC100B9FED2F1B53EC44
:10F83000112B51EC100B06F07DFA41EC100B51EC42
:10F84000100B06F00DFC0890002000F069FF00F09E
:10F85000D7FF0790F5F748F90690069800F5F6717E
:10F8600040F29060C2F2000005909FED210AF4F78B
:10F8700095F9059942F6F600C4F284000863FFE7A3
:10F88000089907980844079041F69450C2F2000086
:10F890000290806A40F29061C2F20001049101F589
:10F8A0003771002301931A4601F074F8019B029806
:10F8B000406A40F67011C2F2000103911A4601F04D
:10F8C00069F80498F4F73AFB00F09AFF03990246AE
:10F8D0000498F3F79DFF0498F4F762FA079800F094
:10F8E00039FFCDE700BF00BF0000000000407F40AF
:10F8F0000000FA430000000080B588B0079000F0D7
:10F9000093FF06F0DAFB41EC100B9FED351B53EC37
:10F91000112B51EC100B06F00DFA41EC100B51ECD1
:10F92000100B06F09DFB0690002000F0F9FE00F0A1
:10F9300067FF0590F5F7D8F800F5A27140F6402072
:10F94000C2F200009FED280AF6F728F9FFE70699B2
:10F9500005980844059041F69450C2F20000C06A30
:10F9600040F60041C2F2000100231A4601F012F8ED
:10F9700058B9FFE740F64020C2F2000040F60041CF
:10F98000C2F20001F6F77EFAFFE741F69450C2F2A8
:10F9900000000290006B40F6F431C2F200010391C6
:10F9A000002301931A4600F0F5FF40F64020C2F212
:10F9B00000000490F6F712FA019B04990298806AFD
:10F9C00001F5C0711A4601F0C5F803990498F5F7DE
:10F9D00001FF0498F6F770F9059800F0BBFEB6E752
:10F9E0000000000000407F400000FA4300000000DB
:10F9F00080B586B0059000F017FF06F05EFB41EC85
:10FA0000100B9FED231B53EC112B51EC100B06F048
:10FA100091F941EC100B51EC100B06F021FB049016
:10FA2000002000F07DFE00F0EBFE0390F5F75CF89F
:10FA3000014641F2E860C2F2000002909FED160A12
:10FA4000FEF702F902980221FEF7BCFEFFE70499D7
:10FA500003980844039041F69450C2F20000406BB2
:10FA600041F69051C2F20001009100231A4600F0C5
:10FA700091FF41F2E860C2F200000190FEF7BCFE87
:10FA800000990198FEF78EF8039800F063FEDEE718
:10FA90000000000000407F400000FA43000000002A
:10FAA00080B584B0039000F0BFFE06F006FB41EC89
:10FAB000100B9FED251B53EC112B51EC100B06F096
:10FAC00039F941EC100B51EC100B06F0C9FA029019
:10FAD000002000F025FE00F093FE019040F2D4508B
:10FAE000C2F20000F5F706F840F6F010C2F200008E
:10FAF000F5F730FDFFE702990198084401900A20CC
:10FB0000F5F740FD78B1FFE740F6F010C2F20000D3
:10FB1000009040F2D451C2F20001F5F725F80098A8
:10FB2000F5F718FDFFE741F69450C2F20000806B34
:10FB300040F2D451C2F2000100231A4601F00AF843
:10FB4000019800F007FED6E70000000000407F406B
:10FB500080B582B001900198806B009000990020E0
:10FB6000C8850098FAF7C2FE02B080BD80B584B0A7
:10FB70000390002002900398806B01900198006828
:10FB80004069C0B2C0090290019890F84100212854
:10FB90000AD1FFE7029838B1FFE701990020C88435
:10FBA000019800F013F9FFE7019800684069C0F37D
:10FBB00080100290019890F8420022280AD1FFE7B5
:10FBC000029838B1FFE701990020C885019800F03C
:10FBD0009FF8FFE70199486C40F0100048640198D5
:10FBE000FAF784FE04B080BD80B586B00590059814
:10FBF000806B0490059800680068C00500285AD4FE
:10FC0000FFE704990020C885FFE7FFE70498006834
:10FC100050E8030F20F480700390FFE703990498E5
:10FC2000026842E803100028F0D1FFE7FFE7FFE792
:10FC3000FFE70498006850E8050F20F001000290EB
:10FC4000FFE702990498026842E805100028F0D105
:10FC5000FFE7FFE7FFE7FFE70498006850E8050FBC
:10FC600020F040000190FFE701990498026842E803
:10FC700005100028F0D1FFE7FFE70499202081F864
:10FC800042000498006B012814D1FFE7FFE7FFE76B
:10FC90000498006850E8030F20F010000090FFE780
:10FCA00000990498026842E803100028F0D1FFE7A9
:10FCB000FFE7FFE7FFE70499002048630498006B23
:10FCC000012805D1FFE70498818DFAF709FE03E0CA
:10FCD0000498FBF7EFF9FFE706B080BD80B582B06E
:10FCE00001900198806B0090009901204863009872
:10FCF000006B012806D1FFE70098818D4908FAF7CB
:10FD0000EFFD03E00098FBF7FFF9FFE702B080BDCD
:10FD100084B00390FFE7FFE70398006850E8030F03
:10FD200020F490700290FFE702990398026842E87D
:10FD300003100028F0D1FFE7FFE7FFE7FFE7039894
:10FD4000006850E8050F20F001000190FFE70199DD
:10FD50000398026842E805100028F0D1FFE7FFE7AA
:10FD60000398006B012814D1FFE7FFE7FFE7039832
:10FD7000006850E8030F20F010000090FFE70099A2
:10FD80000398026842E803100028F0D1FFE7FFE77C
:10FD9000FFE70399202081F84200039900200863BF
:10FDA00004B0704780B582B0019001980168C868BE
:10FDB00020F04000C8600199202081F8410001989E
:10FDC000FBF7CCF9002002B080BD000082B00190AA
:10FDD000FFE7FFE70198006850E8030F20F0C0003C
:10FDE0000090FFE700990198026842E8031000289C
:10FDF000F0D1FFE7FFE70199202081F8410002B030
:10FE00007047000082B000900098006844F600013E
:10FE1000C4F20001884204D1FFE700208DF80700FA
:10FE200010E00098006841F20041C4F201018842EC
:10FE300004D1FFE701208DF8070003E003208DF8CF
:10FE40000700FFE79DF8070002B0704780B586B055
:10FE50000490002003900290049890F84200222819
:10FE600040F0A080FFE704988068B0F5805F13D170
:10FE7000FFE70498006978B9FFE70498806A029068
:10FE80000498006840686FF35F2002990880049925
:10FE9000886A0230886223E00498806A039004989C
:10FEA0008068B0F5805F08D0FFE70498806850B99B
:10FEB000FFE70498006930B9FFE7049800684068DC
:10FEC0000399087007E004980068406800F07F001C
:10FED00003990870FFE70499886A01308862FFE798
:10FEE0000499C88D0138C8850004002856D1FFE761
:10FEF00004980168C86820F02000C8600498016870
:10FF0000C86820F48070C86004980168486920F0CF
:10FF1000010048610499202081F8420004990020E2
:10FF200048630498006B012830D1FFE70499002052
:10FF30000863FFE7FFE70498006850E8030F20F02C
:10FF400010000190FFE701990498026842E803104D
:10FF50000028F0D1FFE7FFE7049800680068C006BA
:10FF600000280ED5FFE7FFE7002000900498006806
:10FF70000068009004980068406800900098FFE7CF
:10FF8000FFE70498818DFAF7ABFC03E00498FBF7D8
:10FF900091F8FFE700208DF8170007E000208DF8AA
:10FFA000170003E002208DF81700FFE79DF8170007
:10FFB00006B080BD80B586B00590059800680069E0
:10FFC00020F44050059A1168D268104308610599E1
:10FFD00088680B694A69C96918431043084304904B
:10FFE00005980068C06849F20C6188430499084389
:10FFF00005990968C86005980068406920F4407058
:020000040801F1
:10000000059A11689269104348610598006841F2A9
:100010000001C4F20101884209D0FFE70598006899
:1000200041F20041C4F20101884204D1FFE7F8F730
:1000300045FA039003E0F8F72FFA0390FFE70598DD
:10004000C069B0F5004F29D1FFE703981921A0FB43
:100050000101059A1368029353685A00DB0FF0F709
:100060003FF90299864648F21F53C5F2EB13AEFBE7
:100070000320420910014FF0640C02FB1CEC3222F9
:1000800002EBCC02A2FB0332F82303EA521300EB8B
:100090004300C2F342121044886026E003981921FD
:1000A000A0FB0101059A1368019353689A009B0F06
:1000B000F0F716F90199844648F21F52C5F2EB1287
:1000C000ACFB02304309642003FB10CC322000EB70
:1000D0000C10A0FB0202F02000EA521000EB03100B
:1000E000C2F3431210448860FFE706B080BD0000F1
:1000F00080B58AB008900791ADF81A200798089942
:100100008862BDF81A00089988850899002048641B
:10011000089A222182F842100899CA6B4FF6E931F9
:10012000C0F60001D1630899CA6B4FF6DD41C0F6F5
:10013000000111640899CA6B4FF66D31C0F60001D9
:10014000D1640899C96B086507A8059008980168EB
:10015000C06B0431059A1268BDF81A30F7F7CAFA75
:1001600058B1FFE70899102048640899202081F8C9
:10017000420001208DF827004EE0FFE700200490A8
:100180000898006800680490089800684068049027
:100190000498FFE708980069A0B1FFE7FFE7FFE7D1
:1001A0000898006850E8030F40F480700390FFE760
:1001B00003990898026842E803100028F0D1FFE78D
:1001C000FFE7FFE7FFE7FFE70898006850E8050F43
:1001D00040F001000290FFE702990898026842E8A7
:1001E00005100028F0D1FFE7FFE7FFE7FFE70898D9
:1001F000006850E8050F40F040000190FFE70199CA
:100200000898026842E805100028F0D1FFE7FFE7F0
:1002100000208DF82700FFE79DF827000AB080BD79
:1002200083B00190019890F8410021283AD1FFE76E
:1002300001988068B0F5805F13D1FFE701980069ED
:1002400078B9FFE70198006A0090009800886FF382
:100250005F200199096848600199086A02300862C4
:1002600008E0019A106A411C11620078019909683E
:100270004860FFE70199C88C0138C884000468B958
:10028000FFE701980168C86820F08000C860019805
:100290000168C86840F04000C860FFE700208DF8A2
:1002A0000B0003E002208DF80B00FFE79DF80B0028
:1002B00003B0704780B582B041F29800C2F20000EE
:1002C0000190FAF73DFB0198F3F7BCF802B080BD4E
:1002D000FFE7FEE782B041EC100B8DED000B0198BB
:1002E000C0F30A5040F2FF71401A18BF012002B05B
:1002F0007047000082B041EC100B8DED000B0198AF
:10030000C0F30A5040F2FF71401A18BF012002B03A
:100310007047000082B041EC100B8DED000B01988E
:10032000C0F30A5040F2FF71401A18BF012002B01A
:100330007047000081B000EE100A00900098C0F3F2
:10034000C750FF3818BF012001B0704781B000EEE0
:10035000100A00900098C0F3C750FF3818BF012062
:1003600001B0704781B000EE100A00900098C0F311
:10037000C750FF3818BF012001B0704784B041EC6E
:10038000100B8DED020B039A00200021CFF6E071D7
:10039000B1EB420F019006D1FFE70298B0FA80F06E
:1003A00040090190FFE7019800F0010004B0704798
:1003B00081B000EE100A009000994FF0807000EBC1
:1003C0004100B0FA80F0400901B0704781B08DF86B
:1003D00003009DF90300002812D4FFE79DF90310E4
:1003E00001F01F02012090404A094EF28011CEF226
:1003F000000141F82200BFF34F8FBFF36F8FFFE77B
:1004000001B0704781B08DF803009DF9030000280A
:100410000ED4FFE79DF9031001F01F020120904068
:100420004A094EF20011CEF2000141F82200FFE726
:1004300001B070474EF60C50CEF200000068C0F3D9
:100440000220704782B08DF8070000919DF90700E7
:1004500000280AD4FFE7009800019DF907104EF22A
:100460000042CEF2000288540BE0009800019DF893
:10047000071001F00F014EF61452CEF2000288541C
:10048000FFE702B07047000082B08DF807000091CE
:100490009DF9070000280AD4FFE7009800019DF9A4
:1004A00007104EF20042CEF2000288540BE0009892
:1004B00000019DF8071001F00F014EF61452CEF224
:1004C00000028854FFE702B07047000083B002903A
:1004D000029800F0070000904EF60C51CEF2000199
:1004E0000868019001984FF6FF02104001900198B2
:1004F000009A40EA02200022C0F2FA521043019012
:100500000198086003B07047B0B581B000900099C1
:1005100040F2006EC2F2000EDEF80000DEF80420A9
:10052000DEF80830DEF80CC0DEF81040DEF81450BB
:100530004D610C61C1F80CC08B604A600860DEF848
:100540001800DEF81C20DEF82030DEF824C0DEF8CB
:1005500028E0C1F828E0C1F824C00B62CA618861B4
:1005600001B0B0BD82B08DED010ACDED000A019859
:100570000099C90F61F3DF7001909DED010A02B08F
:100580007047000080B588B00690069801900198E9
:1005900058B9FFE74FF0500080F31188BFF36F8F19
:1005A000BFF34F8F0790FFE7FEE7019841F2242148
:1005B000C2F200010968884204D1FFE700208DF8EB
:1005C000170056E001F0FEFF01984069049041F2E7
:1005D0002C20C2F200000068039041F23420C2F2E5
:1005E00000000068029002F019F80498039988420C
:1005F00005D0FFE704980299884204D1FFE7022062
:100600008DF8170034E0049848F6F451C2F2000166
:10061000884218D1FFE70198806A78B9FFE701980E
:1006200090F85800012804D1FFE702208DF8170048
:1006300003E003208DF81700FFE703E002208DF8A8
:100640001700FFE713E0049848F60861C2F20001C2
:10065000884203D0FFE7049820B9FFE704208DF813
:10066000170003E001208DF81700FFE7FFE7FFE721
:10067000FFE79DF8170008B080BD000086B08DED43
:10068000050ACDED040A8DED031A02909DED030AD3
:100690009DED041A30EE410A8DED010A0498009098
:1006A0009DED050A9DED001A30EE410A02990120E8
:1006B0008840013801EE100AB8EEC11A20EE010A96
:1006C0009DED011A80EE010ABDEEC00A10EE100A7F
:1006D00006B0704780B582B000200190F7F7EEFCBD
:1006E000FEF722FAFBF7BEFEFBF73EFEFBF7ECFD42
:1006F000FBF712FEFBF7BAFFFCF706F8FBF7DAFF91
:10070000FCF71EF9FCF73EF9FCF746F8FCF792F807
:1007100000F08EF8FBF786FE00F0DAF8FFE7FEE760
:1007200080B584B00290EFF305800390039820B168
:10073000FFE76FF00500019009E0002001900298AA
:1007400020B1FFE7029802F0B7F8FFE7FFE7019852
:1007500004B080BD80B586B00490EFF305800590AD
:10076000059820B1FFE76FF0050001901BE0002025
:10077000019003F073FD039004980399401A0290CE
:10078000029858B1FFE702990020B0EBD17F05D164
:10079000FFE7029903A802F0C7F803E06FF0030037
:1007A0000190FFE7FFE7019806B080BD80B582B0F9
:1007B00003F038FD0146009158B1FFE70098012889
:1007C0000AD0FFE70098022807D1FFE70220019036
:1007D00012E0032001900FE0FFE740F26050C2F208
:1007E00000000068012803D1FFE70120019002E02A
:1007F00000200190FFE7FFE7019802B080BD0000F4
:1008000080B582B0EFF305800190019820B1FFE739
:1008100003F02EFD009003E003F020FD0090FFE7C1
:10082000009802B080BD00004FF47A70704700005D
:1008300082B0EFF305800190019820B1FFE76FF0DF
:100840000500009014E040F26050C2F20000006821
:1008500048B9FFE740F26051C2F200010120086090
:100860000020009003E04FF0FF300090FFE7FFE72B
:10087000009802B07047000080B584B0EFF30580A7
:100880000390039820B1FFE76FF0050002901BE092
:1008900003F0C8FC0146019140B1FFE7019801282F
:1008A0000CD0FFE70198022803D008E00120029055
:1008B00009E002F0BBFA0020029004E0FFE74FF0ED
:1008C000FF300290FFE7FFE7029804B080BD000010
:1008D00080B582B0EFF305800190019820B1FFE769
:1008E0006FF00500009019E040F26050C2F2000085
:1008F000006801280DD1FFE7FDF784F840F2605150
:10090000C2F200010220086002F020FA00200090EC
:1009100003E04FF0FF300090FFE7FFE7009802B0E0
:1009200080BD000080B584B0EFF30580039003988C
:1009300020B1FFE76FF00500029027E003F072FCA2
:100940000146019140B1FFE70198012818D0FFE767
:100950000198022811D014E00120029003F04CFF0E
:10096000012809D0FFE703F05DFC20B9FFE74FF055
:10097000FF300290FFE7FFE707E00020029004E06D
:10098000FFE74FF0FF300290FFE7FFE7029804B067
:1009900080BD000080B588B0069005910492039355
:1009A0000698029000200190EFF3058007900798C9
:1009B00068B3FFE7029830B1FFE7059818B1FFE789
:1009C000039820B1FFE76FF0030001901EE00020C4
:1009D0000090029805996A4602F08CFF012804D025
:1009E000FFE76FF0020001900FE0009860B1FFE7B1
:1009F0004EF60451CEF200014FF080500860BFF374
:100A00004F8FBFF36F8FFFE7FFE7FFE71FE002980D
:100A100018B1FFE7059820B9FFE76FF003000190D8
:100A200014E002980599039A02F076FE01280CD092
:100A3000FFE7039820B1FFE76FF00100019003E0AA
:100A40006FF002000190FFE7FFE7FFE7FFE7019883
:100A500008B080BD80B588B0069005910492002052
:100A60000390EFF305800790079800286ED1FFE709
:100A7000069800286AD0FFE70598002866D0FFE7AF
:100A80004FF0FF300290049868B3FFE70498806845
:100A9000A0B1FFE70498C06850280FD3FFE704987F
:100AA000006958B1FFE7049840690699059A5143D7
:100AB000884203D3FFE70120029013E00498806886
:100AC00078B9FFE70498C06858B9FFE7049800694F
:100AD00038B9FFE70498406918B9FFE70020029091
:100AE000FFE7FFE702E000200290FFE702980128FD
:100AF0000ED1FFE706980599049A93681269EE46AD
:100B00004FF0000CCEF800C002F02EFB03900AE07C
:100B1000029838B9FFE706980599002202F0EAFA30
:100B20000390FFE7FFE7039878B1FFE7049820B14F
:100B3000FFE704980068019002E000200190FFE7C1
:100B40000398019901F05CFEFFE7FFE7039808B006
:100B500080BD000080B588B0069005918DF8132007
:100B600003930698029000200190EFF30580079010
:100B7000079868B3FFE7029830B1FFE7059818B10E
:100B8000FFE7039820B1FFE76FF0030001901EE03C
:100B900000230093029805996A4602F0E1FC0128BF
:100BA00004D0FFE76FF0020001900FE0009860B101
:100BB000FFE74EF60451CEF200014FF0805008607E
:100BC000BFF34F8FBFF36F8FFFE7FFE7FFE720E033
:100BD000029818B1FFE7059820B9FFE76FF003000E
:100BE000019015E002980599039A002302F0A2FBF8
:100BF00001280CD0FFE7039820B1FFE76FF0010058
:100C0000019003E06FF002000190FFE7FFE7FFE7CC
:100C1000FFE7019808B080BD80B584B002900298CB
:100C20000190EFF305800390039820B1FFE76FF088
:100C3000050000900DE0019820B9FFE76FF0030078
:100C4000009005E000210091019802F015FBFFE7FC
:100C5000FFE7009804B080BD80B586B00490039192
:100C6000049820F001000290049800F00100009028
:100C700000200190EFF305800590059820B1FFE773
:100C80006FF00500019033E0029820B9FFE76FF0A4
:100C9000030001902BE00098A0B1FFE702980399B0
:100CA00002F0C2FF01280CD0FFE7039820B1FFE754
:100CB0006FF00100019003E06FF002000190FFE788
:100CC000FFE713E00298039902F098FE01280CD088
:100CD000FFE7039820B1FFE76FF00100019003E008
:100CE0006FF002000190FFE7FFE7FFE7FFE7FFE794
:100CF000019806B080BD000080B588B00690002045
:100D00000590EFF3058007900798002840F0858054
:100D1000FFE7069820B1FFE706984068049002E0DC
:100D200000200490FFE79DF81000C00718B1FFE70E
:100D30000120039002E000200390FFE7049800F0F8
:100D40000800082868D0FFE74FF0FF3002900698AF
:100D5000C8B1FFE70698806840B1FFE70698C06811
:100D6000502803D3FFE7012002900BE0069880682B
:100D700038B9FFE70698C06818B9FFE7002002906D
:100D8000FFE7FFE702E000200290FFE7029801285A
:100D900012D1FFE7039838B1FFE706988168042075
:100DA00002F08EF9059006E006988168012002F0B5
:100DB00087F90590FFE711E0029870B9FFE7039803
:100DC00028B1FFE7042002F067F9059004E0012054
:100DD00002F062F90590FFE7FFE7FFE7059878B1B9
:100DE000FFE7069820B1FFE706980068019002E04F
:100DF00000200190FFE70598019901F001FDFFE750
:100E0000059840B1FFE7039828B1FFE7059840F047
:100E100001000590FFE7FFE7FFE7059808B080BDF8
:100E200080B586B00490049820F0010003900498E7
:100E300000F00100019000200290EFF30580059082
:100E4000059820B1FFE76FF00500029024E00398B9
:100E500020B9FFE76FF0030002901CE0019858B141
:100E6000FFE7039802F022FC012804D0FFE76FF0AF
:100E700002000290FFE70DE00398002319461A468E
:100E800002F058FA012804D0FFE76FF00200029048
:100E9000FFE7FFE7FFE7FFE7029806B080BD00002D
:100EA00080B58AB00890079108980690069830B1EE
:100EB000FFE79DF81F000006002804D5FFE76FF04C
:100EC000030005903BE04FF0FF300590EFF3058005
:100ED0000990099820B3FFE7002303930493069831
:100EE0000799EC4604AACCF80020012203F0AEF8E2
:100EF000039A069869460A6005AB114603F0A6F806
:100F0000049860B1FFE74EF60451CEF200014FF0B5
:100F100080500860BFF34F8FBFF36F8FFFE70DE086
:100F20000698079901220023029302F0D3FF029A48
:100F3000069805AB114602F0CDFFFFE7FFE70598E5
:100F40000AB080BD80B58CB00A9009910892EFF389
:100F500005800B900B9820B1FFE76FF0050007901C
:100F60007AE09DF82B000006002804D5FFE76FF01B
:100F7000030007906FE09DF824008007002803D548
:100F8000FFE70020059002E00A980590FFE70020A7
:100F900007900898029003F061F90490FFE7059923
:100FA000029B002006AA03F055FA0190019801283F
:100FB0003FD1FFE70A9907980840079006990798DC
:100FC000084307909DF82400C00780B1FFE70A9905
:100FD00007980840884201D1FFE73BE0089820B914
:100FE000FFE76FF00200079034E0FFE70EE00A9899
:100FF0000799084201D0FFE72CE0089820B9FFE7E5
:101000006FF00200079025E0FFE7FFE703F026F905
:101010000499401A039003980299884203D9FFE784
:101020000020029004E003990298401A0290FFE722
:101030000BE0089820B9FFE76FF00200079003E08B
:101040006FF001000790FFE7FFE7FFE70198002836
:10105000A5D1FFE7FFE7FFE707980CB080BD0000D0
:1010600080B582B003F0D4F80190019802B080BD41
:10107000B0B58EB00B900A91099200200690EFF364
:1010800005800D900D98002840F09980FFE70B989F
:10109000002800F09480FFE780200790182005903A
:1010A000002008904FF0FF300490099800284DD0A0
:1010B000FFE70998006820B1FFE7099800680890E9
:1010C000FFE70998806920B1FFE7099880690590DA
:1010D000FFE7059848B1FFE70598382805D8FFE7EE
:1010E00009980079C00718B1FFE700200C9069E06B
:1010F0000998406928B1FFE709984069800807907E
:10110000FFE70998806880B1FFE70998C0685C280C
:101110000BD3FFE70998006938B1FFE709984069E8
:1011200018B1FFE7012004900FE00998806858B9D2
:10113000FFE70998C06838B9FFE70998006918B94E
:10114000FFE700200490FFE7FFE702E000200490A3
:10115000FFE70498012817D1FFE70B980899079A31
:101160000A9BDDF814C0DDF824E0DEF80850DEF854
:101170001040EE46CEF80850CEF80440CEF800C03D
:1011800002F040FE069019E00498B0B9FFE70B9812
:101190000899BDF81C200A9BDDF814C0EE4606AC89
:1011A000CEF80440CEF800C002F0DCFD012803D0E8
:1011B000FFE700200690FFE7FFE7FFE7FFE706985D
:1011C0000C90FFE70C980EB0B0BD000080B586B063
:1011D000049004980390EFF305800590059820B1E2
:1011E000FFE76FF0050002901CE0039820B9FFE7CD
:1011F0006FF00300029014E00398FFF7C3F98DF835
:1012000007009DF80700042806D0FFE700200290A1
:10121000039801F013FC03E06FF002000290FFE777
:10122000FFE7FFE7029806B080BD000080B584B0FC
:101230000390029148F61C60C2F200000068009022
:1012400041F22420C2F200000068043001F0ECF802
:1012500008B9FFE700E0FFE70398013080B9FFE736
:10126000029868B1FFE741F22420C2F20000006852
:10127000011D48F6F450C2F2000001F07BF93DE098
:101280000098039908440190019841F22421C2F288
:101290000001096848600198009988420ED2FFE772
:1012A00041F23420C2F20000006841F22421C2F26F
:1012B00000010968043101F027F91EE041F22C20F9
:1012C000C2F20000006841F22421C2F20001096864
:1012D000043101F019F9019848F68051C2F2000179
:1012E0000968884207D2FFE7019848F68051C2F2A8
:1012F0000001086000E0FFE7FFE7FFE704B080BD02
:1013000080B582B0019001F05DF948F25461C2F2FB
:10131000000108680130086041F22420C2F2000098
:10132000006898B9FFE7019841F22421C2F2000158
:10133000086048F25460C2F200000068012803D13E
:10134000FFE700F021FB00E0FFE71CE048F6E85073
:10135000C2F200000068A0B9FFE741F22420C2F207
:1013600000000068C06A0199C96A884207D8FFE78F
:10137000019841F22421C2F20001086000E0FFE779
:1013800000E0FFE7FFE748F26060C2F2000001689A
:10139000013101600068019948640198C06A48F20F
:1013A0006461C2F200010968884208D9FFE7019828
:1013B000C06A48F26461C2F200010860FFE7019967
:1013C000C86A00EB800241F23C20C2F2000000EB50
:1013D0008200043101F0CEF801F020F948F6E8501F
:1013E000C2F200000068C8B1FFE741F22420C2F257
:1013F00000000068C06A0199C96A88420CD2FFE700
:101400004EF60451CEF200014FF080500860BFF359
:101410004F8FBFF36F8F00E0FFE700E0FFE702B000
:1014200080BD000080B584B001F0CCF848F62060A3
:10143000C2F200000068002840D1FFE748F62050C3
:10144000C2F20000029001F03FF848F63450C2F2B8
:101450000000039001F038F80299039841F2282225
:10146000C2F20002116041F23821C2F200010860AC
:1014700069460020086041F23012C2F2000241F2D7
:10148000D013C2F200030A20102101F06DFE0146C4
:1014900048F62060C2F200000160006860B1FFE71A
:1014A00048F62060C2F20000006846F64521C0F60A
:1014B000010101F0A5F900E0FFE700E0FFE701F01E
:1014C000ADF804B080BD000080B582B0FFE748F2FF
:1014D0005860C2F20000006808B3FFE701F072F83C
:1014E00048F60860C2F20000C068C0680190019828
:1014F000043000F099FF48F25461C2F2000108681C
:101500000138086048F25861C2F2000108680138E9
:10151000086001F083F8019800F08CF8D7E702B07A
:1015200080BD000080B582B0019000910198006CF0
:10153000B8B1FFE70199C8680A6C1044C860019807
:101540008168C068884204D3FFE701990868C860D1
:1015500000E0FFE70098019AD168126CEEF756FFA1
:10156000FFE702B080BD000080B586B00590049111
:101570000392002002900598806B01900598006C02
:1015800078B9FFE70598006848B9FFE705988068D3
:1015900002F0CCFF029005990020886000E0FFE790
:1015A00041E00398B8B9FFE7059A04995068126CB6
:1015B000EEF72CFF059948680A6C104448600599BD
:1015C00048688968884204D3FFE70599086848603D
:1015D00000E0FFE726E0059A0499D068126CEEF768
:1015E00015FF0599C8680A6C801AC86005980168DB
:1015F000C068884206D2FFE7059988680A6C801A9D
:10160000C86000E0FFE70398022809D1FFE70198CE
:1016100020B1FFE701980138019000E0FFE700E00A
:10162000FFE7FFE7FFE7019801300599886302981B
:1016300006B080BD80B582B00090009890F8590047
:1016400040B9FFE70098006B01F00EF8009801F038
:101650000BF81CE0009890F85900012804D1FFE72E
:10166000009801F001F811E0009890F85900022864
:101670000BD0FFE74FF0500080F31188BFF36F8F5E
:10168000BFF34F8F0190FFE7FEE7FFE7FFE702B0F0
:1016900080BD000082B001900198406A38B1FFE738
:1016A0000198006B0068C0F13800009002E0002053
:1016B0000090FFE7009802B07047000082B00190F0
:1016C00041F22820C2F2000000680068B0FA80F001
:1016D0004009019908600198006848B9FFE741F2A4
:1016E0002820C2F200000068C0680068009002E094
:1016F00000200090FFE7009802B0704784B04FF4DC
:10170000C040009042F24860C2F2000001909DF893
:101710000400400788B1FFE7019807300190019865
:1017200020F007000190019A42F24861C2F20001E4
:101730000098891A08440090FFE7019802900299E6
:1017400048F6EC50C2F200000160002141600298AE
:10175000009A10440190019808380190019820F0F7
:1017600007000190019A41F23020C2F200000260AD
:101770000268516002681160029903910199039A0D
:10178000891A51600068039908600398406848F618
:101790007C51C2F2000108600398406848F6745119
:1017A000C2F20001086048F64851C2F200014FF051
:1017B0000040086004B0704780B582B00190FFE738
:1017C000FFF782FE41F23C20C2F2000000680228CE
:1017D0000CD3FFE74EF60451CEF200014FF08050DB
:1017E0000860BFF34F8FBFF36F8F00E0FFE7E7E7BD
:1017F00080B582B00190019868B1FFE7019800239D
:101800008360019803600198C360019819461A46E5
:1018100001F090FD00E0FFE702B080BD80B584B02C
:10182000DDF818C00390029101928DF80330029800
:1018300018B9FFE70698006003E001980699086070
:10184000FFE703980699C86302980699086406980A
:10185000012101F011FD9DF80300069981F84C006B
:1018600004B080BD80B588B0DDF834C0DDF830C08C
:10187000DDF82CC0DDF828C0069005910492039392
:101880000C98006B04998900A522EEF736FE0C989F
:10189000006B049900EB810004380290029820F05C
:1018A000070002909DF80800400758B1FFE74FF08D
:1018B000500080F31188BFF36F8FBFF34F8F0790F5
:1018C000FFE7FEE70598F8B1FFE700200190FFE78A
:1018D00001980F2813D8FFE70598019A805C0C99AE
:1018E000114481F8340005980199405C08B9FFE77C
:1018F00005E0FFE7FFE7019801300190E8E70C9968
:10190000002081F8430004E00C99002081F83400A5
:10191000FFE70A98382803D3FFE737200A9000E052
:10192000FFE70A980C99C8620A980C99C8640C9948
:101930000020009008650C98043000F0DDFD0C9844
:10194000183000F0D9FD00980C9909610A99C1F18D
:1019500038010C9A91610C9949620C9948650C996F
:1019600081F8580002980699039A00F0E7FC0C9958
:1019700008600B9820B1FFE70C980B99086000E015
:10198000FFE708B080BD000080B584B00020039060
:10199000FFE70398372810D8FFE7039800EB800192
:1019A00041F23C20C2F2000000EB810000F08CFD0F
:1019B000FFE7039801300390EBE748F64C50C2F282
:1019C0000000019000F080FD48F66050C2F2000077
:1019D000029000F079FD48F69450C2F2000000F049
:1019E00073FD48F60860C2F2000000F06DFD48F695
:1019F000F450C2F2000000F067FD0199029841F234
:101A00002C22C2F20002116041F23421C2F2000124
:101A1000086004B080BD000083B0029048F6EC502E
:101A2000C2F200000190FFE7019800680299884225
:101A300005D2FFE7FFE7019800680190F4E70198FD
:101A4000009000980199496808440299884209D198
:101A5000FFE702984268019948681044486001987D
:101A6000029000E0FFE70298009000980299496810
:101A7000084401990968884220D1FFE7019800686D
:101A800041F23021C2F20001096888420DD0FFE71F
:101A900001980068426802994868104448600198BB
:101AA000006800680299086007E041F23020C2F245
:101AB0000000006802990860FFE704E001980068F0
:101AC00002990860FFE701980299884204D0FFE775
:101AD00002980199086000E0FFE703B0704700003A
:101AE00080B586B005900491039202930020019086
:101AF0000498059948600598006104980399884204
:101B000016D8FFE703980299401A05998969884217
:101B100003D3FFE70120019009E041F23820C2F22F
:101B2000000000680599043100F0EEFCFFE717E0C3
:101B300003980299884208D2FFE7049802998842E4
:101B400003D3FFE70120019009E041F22820C2F20F
:101B5000000000680599043100F0D6FCFFE7FFE7BC
:101B6000019806B080BD000080B582B0019000F001
:101B700029FD0198806B18B9FFE70120009002E071
:101B800000200090FFE700F049FD009802B080BD02
:101B900080B582B0019000F015FD0198806B01992D
:101BA000C96B884203D1FFE70120009002E00020CA
:101BB0000090FFE700F032FD009802B080BD000009
:101BC00008480068006880F308884FF0000080F340
:101BD000148862B661B6BFF34F8FBFF36F8F00DF1B
:101BE00000BF00BF08ED00E080B586B0049003910F
:101BF00041F22820C2F200000068C068C06801906D
